:020000040800F2
:10000000E0E5012095020008BD7200080D620008BD
:100010005D710008152100083D93000800000000F4
:1000200000000000000000000000000091790008BE
:100030003D2F0008000000003175000815850008FC
:10004000AF020008AF020008AF020008AF020008CC
:10005000AF020008AF020008412F0008AF020008FD
:10006000AF0200084D2F0008592F0008AF0200080A
:10007000512E0008AF020008AF020008AF020008CE
:10008000AF020008AF020008AF02000839210008E3
:100090001921000829210008AF020008652F000877
:1000A000AF020008E1850008AF020008AF020008B7
:1000B000AF020008AF020008AF020008AF0200085C
:1000C000AF020008AF020008AF020008AF0200084C
:1000D000AF020008AF020008AF0200082593000835
:1000E000AF020008AF020008AF020008AF0200082C
:1000F000AF020008AF020008AF020008AF0200081C
:10010000AF020008AF020008AF020008AF0200080B
:10011000AF020008AF020008AF020008AF020008FB
:10012000AF020008AF020008612E0008712E00081F
:10013000AF020008AF020008AF0200086921000802
:100140004921000859210008AF020008AF02000849
:10015000AF020008AF020008AF020008AF020008BB
:10016000AF020008AF020008AF020008AF020008AB
:10017000AF020008AF020008AF0200080000000054
:10018000AF020008AF02000800F002F800F072F8B9
:100190000AA090E8000C82448344AAF10107DA45E2
:1001A00001D100F067F8AFF2090EBAE80F0013F0C2
:1001B000010F18BFFB1A43F001031847C0E4000009
:1001C00000E500000A444FF0000C10F8013B13F06A
:1001D000070408BF10F8014B1D1108BF10F8015BA0
:1001E000641E05D010F8016B641E01F8016BF9D193
:1001F00013F0080F1EBF10F8014BAD1C0C1B09D1EA
:100200006D1E58BF01F801CBFAD505E014F8016B5B
:1002100001F8016B6D1EF9D59142D6D370470000ED
:10022000103A24BF78C878C1FAD8520724BF30C822
:1002300030C144BF04680C607047000000230024F4
:1002400000250026103A28BF78C1FBD8520728BFE6
:1002500030C148BF0B607047752900F0DD8063290D
:1002600000F02D82002070471FB50EF080F81FBDF2
:1002700010B510BD00F038FA1146FFF7F5FF09F090
:1002800003FA00F056FA03B4FFF7F2FF03BC00F0E4
:1002900059FA00000948804709480047FEE7FEE791
:1002A000FEE7FEE7FEE7FEE7FEE7FEE7FEE7FEE726
:1002B00004480549054A064B70470000CD850008F3
:1002C00089010008F0A30120E0E50120F0A501204C
:1002D000E0E1012053EA020C00F069802DE9F04BC7
:1002E0004FF00006002B1FBFB3FA83F503FA05F4A5
:1002F00024FA05F65E4012BF1643B2FA82F502FAFE
:1003000005F4C5F120051EBF22FA05FC44EA0C04E1
:10031000203556EA044C4FEA144418BF641C4FF0D1
:1003200000084FF00009904271EB030C39D300290B
:1003300019BFB1FA81F701FA07F6B0FA80F700FAAF
:1003400007F6C7F120071EBF20FA07FC46EA0C0695
:100350002037B6FBF4FCA7EB0507103F07F01F0B97
:10036000CBF120062CFA06F60CFA0BFB44BFB34681
:100370000026202FA4BF5E464FF0000B5BEA060C60
:1003800008BF4FF0010B19EB0B0948EB0608ABFB5C
:10039000027C06FB02CC0BFB03CCC01B71EB0C01F7
:1003A000C1E70B46024641464846BDE8F08B13B50F
:1003B000084318BF4FF0FF300146AFF30080BDE89F
:1003C0001C40704770B50C460546012A05D02878B8
:1003D000800600D5EA69002302E0012305E05B1CEA
:1003E000934202D2E05C0028F9D1A869E618C01A4D
:1003F000A861286A184428622846AFF3008004E008
:10040000D5E9012114F8010B9047B442F8D32846EE
:10041000AFF3008070BD00002DE9F04106460024D6
:1004200010687529314616A510D0AFF3008000285A
:1004300002DA404213A507E031688A0701D512A508
:1004400002E0490704D511A5012401E0AFF30080C3
:1004500000210A2206F1240709E0B0FBF2FCB0FB00
:10046000F2F302FB1C00303078541846491C002877
:10047000F3D123462A463046BDE8F04100F0BCB82F
:10048000000000002D0000002B00000020000000F4
:10049000032A40F2308010F0030C00F0158011F8B0
:1004A000013BBCF1020F624498BF11F801CB00F888
:1004B000013B38BF11F8013BA2F1040298BF00F8DC
:1004C00001CB38BF00F8013B11F0030300F0258099
:1004D000083AC0F0088051F8043B083A51F804CBC0
:1004E000A0E80810F5E7121D5CBF51F8043B40F886
:1004F000043BAFF30080D20724BF11F8013B11F891
:1005000001CB48BF11F8012B24BF00F8013B00F8D4
:1005100001CB48BF00F8012B704710B5203AC0F05E
:100520000B80B1E81850A0E81850B1E81850A0E8C6
:100530001850203ABFF4F5AF5FEA027C24BFB1E85F
:100540001850A0E8185044BF18C918C0BDE81040A2
:100550005FEA827C24BF51F8043B40F8043B08BFAB
:100560007047D20728BF31F8023B48BF11F8012B72
:1005700028BF20F8023B48BF00F8012B704702F06B
:10058000FF0343EA032242EA024200F002B84FF0BE
:10059000000200B5134694469646203922BFA0E8D3
:1005A0000C50A0E80C50B1F12001BFF4F7AF0907DF
:1005B00028BFA0E80C5048BF0CC05DF804EB8900D0
:1005C00028BF40F8042B08BF704748BF20F8022B13
:1005D00011F0804F18BF00F8012B7047704770472B
:1005E000704710B500F078F8006810BD10B50446EB
:1005F00000F072F8046010BD2DE9F0470D469946F1
:100600009246044600F124080168880604D5E06992
:1006100021F01001216000E00120A84201DD471B0C
:1006200000E00027A1697A1902EB0900081AA0610D
:100630002078C00602D42046AFF30080002608E0F0
:10064000D4E901211AF806009047206A401C761C64
:1006500020624E45F4DB2078C0060AD52046AFF371
:10066000008006E0D4E9012130209047206A401C38
:100670002062381EA7F10107F4DC07E0D4E901216C
:1006800018F805009047206A401C2062281EA5F13A
:100690000105F3DC2046AFF300802078000602D588
:1006A0000220BDE8F0870120FBE710B5436913B1D4
:1006B000AFF3008001E0FFF785FE012010BD127846
:1006C00000F124010A7000224A700122EDE711684E
:1006D0004FF0FF32E9E70000004870478803002030
:1006E00000487047880300207546FFF7F9FFAE46C3
:1006F00005006946534620F00700854618B020B52E
:10070000FFF7D6FDBDE820404FF000064FF0000790
:100710004FF000084FF0000BAC46ACE8C009ACE865
:10072000C009ACE8C009ACE8C00921F007018D465A
:10073000704710B50446AFF300802046BDE8104076
:10074000FFF7A1BD01491820ABBEFEE7260002005D
:1007500070470000B0B52DED028B044600284FF025
:10076000FF0061D00D4600295ED095ED000A95EDA1
:10077000011A95ED022A95ED033A20EE010A22EEC8
:10078000033A21EE011A22EE022A31EE021A30EE6D
:10079000030A31EE011AB7EE008A30EE000A78EE55
:1007A000410A0CF0DDF9B0EE401A95ED000A95ED26
:1007B000012A95ED023A95ED034A20EE030A24EE54
:1007C000022A30EE420A30EE000AB0EEC02AB4EE41
:1007D000482AF1EE10FA84ED011A02DA0BF0BEFE9F
:1007E00001E008F0DFFE84ED020A95ED000A95EDC8
:1007F000011A95ED032A95ED023A20EE020A21EE48
:10080000031A30EE010A23EE031A22EE022A32EE18
:10081000011A31EE011A30EE000A78EE410A0CF0AE
:100820009FF9002084ED000A40B2BDEC028BB0BD00
:1008300070B52DED028B00284FD0B7EE001A81EE77
:10084000000A0D4604464FF07E51002D80ED040A4B
:100850004FF00000C4E90010A060E06000F09F804D
:10086000D5E900600DF0B8FC41EC180B30460DF0F6
:10087000B3FC41EC110BB0EE480AF0EE680A0CF044
:100880006FF851EC100B0CF0EFFD95ED000AB5EE92
:10089000400AF1EE10FA22D195ED010AB5EE400AB8
:1008A000F1EE10FA1BD195ED020AB5EE400AF1EE19
:1008B00010FA14D140F2C560C3F64D7044F62D21F4
:1008C0004AF2564244F2AD73C3F60D41CBF63932CB
:1008D000C3F619730FC4002061E0FF205FE09FEDB5
:1008E000321A00EE100AB4EE410AF1EE10FA1EDCE4
:1008F000B5EE400AF1EE10FA19DB9FED2C2AB4EEAA
:10090000420AF1EE10FA25DCB4EE410AF1EE10FADB
:1009100020DB9FED271AB4EE410AF1EE10FA2CDC31
:10092000B4EE420AF1EE10FA27DB002037E045F67C
:100930006E10C3F67F7045F20C3148F6AB0249F2F7
:100940008553C3F6B011CBF6BB32C3F697530FC431
:10095000002024E040F2C560C3F64D7044F62D211E
:100960004AF2564244F2AD73C3F60D41CBF639322A
:10097000C3F619730FC4002011E040F2C560C3F63E
:100980004D7044F62D214AF2564244F2AD73C3F63F
:100990000D41CBF63932C3F619730FC4002040B2B3
:1009A000BDEC028B70BD00BFDB0FC9BFDB0F49C0C0
:1009B0000000B4C20021C0E900118160704700004E
:1009C000B0B52DED108B8EB0044600284FF0FF001F
:1009D00018BF002904D140B20EB0BDEC108BB0BDE1
:1009E000002AF8D04CF200054EF69E70C2F20105C6
:1009F000C3F627502860C3B193ED00EA93ED01FAE6
:100A0000D3ED028AB5EE40EAF1EE10FA11D1B5EE5F
:100A100040FAF1EE10FA0CD1F5EE408AF1EE10FA40
:100A200007D1204600F094FAD5E7204600F090FA6E
:100A3000D1E792ED000A92ED011A94ED014A94ED8E
:100A4000025A92ED022A94ED036A94ED003A24EEE4
:100A5000407A61EE050A37EE607A62EE060A37EEFA
:100A6000607A60EE030A62EE051A71EEA00A61EE8A
:100A7000061A70EEE10A61EE031A62EE042A22EE13
:100A8000032A21EE041A91ED00DA71EEE21A20EE4B
:100A9000066A31EE021A20EE050A36EE216AD1ED21
:100AA000019AD1ED02AA31EE400AB6EE001AB5EE77
:100AB00040DA27EE015A60EE810A26EE017AF1EE65
:100AC00010FA20EE016A0AD1F5EE409AF1EE10FA22
:100AD00005D1F5EE40AAF1EE10FA00F0EC812DEE12
:100AE0000D0A29EEA91A30EE010A2AEEAA1A30EEF2
:100AF000010A8DED0D6A8DED0C7ACDED0B0A8DEDB1
:100B00000A5A05F085FB2DEE001A8DED071A29EE25
:100B1000801A2AEE800A8DED081A8DED090A2EEE54
:100B20000E0A2FEE0F1A30EE010A28EEA81A30EE48
:100B3000010A05F06DFB94ED001A6EEE00DA6FEE1F
:100B400000AA94ED034A31EE01EA68EE808A94ED42
:100B5000012A94ED023A2AEE8E6A61EE01EA8DEDE9
:100B6000026A28EE8E0A2DEEAE5A26EE046A62EE76
:100B700002BA35EE465A20EE036A36EE055A2DEEDD
:100B8000AB6A32EE02FA36EE055A2AEE8F6A23EE8F
:100B9000066A36EE055A28EE8F6A26EE046A63EE80
:100BA00003FA36EE055A2DEEAF6A24EE048A35EECE
:100BB000465A2DEE886A2DEE8E9A35EE465A29EE6B
:100BC000046A2AEEAE7A37EE066A22EE000A2DEEAD
:100BD0008FAA36EE400A23EE0A6A36EE000A2AEEA3
:100BE000AB6A30EE460A2AEEAF6A73EE039A36EE2F
:100BF000000A28EEA96A24EE066A36EE000A2AEEFA
:100C0000886A30EE460A25EE055A20EE000A35EED7
:100C1000000A21EE02BA21EE035A21EE041A8DEDEC
:100C2000051A22EE031A8DED031A23EE041A8DED38
:100C3000041A34EE041A8DED015A22EE04CA6EEE47
:100C400003CA8DED061A29EE84DA05F0E1FA94ED77
:100C5000013A94ED022A9DED021A29EE024A21EE94
:100C6000031A31EE444A94ED031A28EEAE5A35EEDB
:100C7000044A2AEE015A35EE044A28EEAB5AF7EE42
:100C8000001A34EE454A2AEEA95A81EE800A25EE72
:100C9000015A35EE044A28EEAF5A34EE454A28EEA2
:100CA000885A75EE042A3CEE0C4A9DED075A34EE44
:100CB0006C4A34EE454A3BEE0B5A9DED086A35EE20
:100CC0000D5A35EE465A2FEE056A29EE847AF6EE75
:100CD000007A76EE470A37EEEF6A36EE486A9DED07
:100CE000018A20EE066A3CEE487A27EE227A36EE3A
:100CF000076A36EE6D7A22EE226A66EE073A70EEE9
:100D0000E33ADDED050ADDED034A60EE015A74EECB
:100D1000E00ADDED044A60EE200A7BEE244A64EE30
:100D2000A24A70EEA40A63EE224A70EEEA0A74EE5A
:100D3000E56A66EEA06A77EEEB7A76EEA33A78EE95
:100D40000C6A77EEEF7A60EE266A67EEA27A76EEAC
:100D5000A76A76EEE86A60EE027ADDED068A27EE93
:100D6000A68A38EE23CA68EE843A2EEE058A78EE1B
:100D7000233A3BEEAB8A71EEC81A3FEEAF8A71EEB2
:100D8000C81A9DED098A21EE22AA71EEC81AB1EEA9
:100D9000008A23EE089A21EE899A73EEC93A94EDFF
:100DA000009A2AEE07BA73EE8B3A29EE22BA77EE52
:100DB0008B7A67EEA07A72EEA22A77EEA33A63EE00
:100DC000227A75EEE75A65EEA65A35EEA3DA68EE9A
:100DD000853A6EEE045A73EEE53A62EE085A65EE15
:100DE000A11A73EEE11AF8EE003A60EE233A62EED1
:100DF000235A75EECB5A65EE875A20EE033A71EE10
:100E0000A51A73EE0A5A20EE090A22EE222A65EE8E
:100E1000A05A30EE422A75EEA11A22EE262A23EEBF
:100E2000811A32EE218A2FEE042A29EE854A31EE0C
:100E3000241A34EE022A21EE071A36EE400A32EE68
:100E4000011A20EE200A30EE010A23EE261A31EEB6
:100E5000009A2CEE0C0A2DEE0D1A30EE010A28EE47
:100E6000081A31EE000A29EE091A31EE000A05F0DF
:100E7000CFF995ED004A9DED0A5A20EE0C1ADDEDF2
:100E80000B0A20EE0D2A24EE011A9DED0C7A9DED41
:100E90000D6A20EE083A20EE090A35EE415A24EE9A
:100EA000021A70EEC10A24EE031A24EE000A37EE8D
:100EB000417A36EE406A94ED043A94ED000A94EDDE
:100EC000011A25EE035A94ED022A30EE050A20EEAF
:100ED000835A94ED034A35EE011A27EE035A35EE94
:100EE000022A26EE033A84ED000A84ED011A20EE70
:100EF000000A21EE011A33EE043A30EE010A22EE26
:100F0000021A30EE010A23EE031A30EE010A84EDD4
:100F1000022A84ED033A05F07BF994ED001A94ED72
:100F2000012A94ED023A94ED034A20EE011A20EED4
:100F3000022A20EE033A20EE040A002084ED001A73
:100F400084ED012A84ED023A84ED030A43E50000B2
:100F5000B0B52DED108B044600284FF0FF0018BFF0
:100F6000002900F06981002A00F066814CF200053A
:100F700042F60230C2F20105C3F60750286092ED36
:100F8000000A92ED011A94ED014A94ED025A92ED95
:100F9000022A94ED036A94ED003A24EE407A61EE61
:100FA000050A37EE607A62EE060A37EE607A60EE86
:100FB000030A62EE051A71EEA00A61EE061A70EEDF
:100FC000E10A61EE031A62EE042A22EE032A21EE00
:100FD000041A91ED00CA71EEE21A20EE066A31EEB3
:100FE000021A20EE050A36EE216A91ED01DA91ED42
:100FF00002EA31EE400AB6EE001AB5EE40CA27EE1C
:1010000001BA20EE81AA26EE019AF1EE10FA20EE46
:10101000018A0AD1B5EE40DAF1EE10FA05D1B5EE4B
:1010200040EAF1EE10FA00F0BC802CEE0C0A2DEE36
:101030000D1A30EE010A2EEE0E1A30EE010A05F0FE
:10104000E7F894ED003A94ED025AF1EE001A2CEE16
:10105000001A94ED014A75EE050A63EE212A65EE49
:10106000053A62EEA34A61EE205A74EEA54A64EE98
:10107000045A2DEE002A94ED036A34EE047A62EEEF
:10108000A52A72EEA42A62EE074A32EEE4CA76EE90
:10109000062A64EE214A66EE066A64EEA67A21EE1E
:1010A00022DA77EECD7A23EE03DA2DEE21DA2EEE78
:1010B000000A24EE0DEA33EE033A7EEE277A22EEA2
:1010C00003EA77EECE7AB2EE00EA24EE0E4A77EE2D
:1010D000E47A24EE25FA7FEE277A24EE234A34EED2
:1010E000274A60EE244A34EE84FA2DEE054A21EEBA
:1010F000033A33EE043A25EE0E4A25EE215A65EE08
:10110000264A33EE243A62EE222A33EE623A33EE76
:10111000453A65EE842A32EE833A24EE234A34EED1
:10112000033A20EE050A30EE03DA21EE070A25EE37
:10113000A11A21EE061A31EE400A23EEA11A26EE7C
:10114000011A30EE010A22EE201A30EE41EA2CEEAE
:101150000C0A2FEE0F1A30EE010A2DEE0D1A31EEA9
:10116000000A2EEE0E1A31EE000A05F051F895ED48
:10117000004A20EE0C1A20EE0F2A24EE011A20EE6F
:101180000D3A20EE0E0A3BEE41BA24EE021A3AEE78
:1011900041AA24EE031A24EE000A39EE419A38EEF1
:1011A000408A94ED043A94ED000A94ED011A2BEE76
:1011B000035A94ED022A30EE050A2AEE035A94ED02
:1011C000034A35EE011A29EE035A35EE022A28EEBB
:1011D000033A84ED000A84ED011A20EE000A21EEA4
:1011E000011A33EE043A30EE010A22EE021A30EE12
:1011F000010A23EE031A30EE010A84ED022A84ED7F
:10120000033A05F005F894ED001A94ED012A94EDE7
:10121000023A94ED034A20EE011A20EE022A20EE53
:10122000033A20EE040A002084ED001A84ED012A1E
:1012300084ED023A84ED030A40B2BDEC108BB0BDE0
:10124000B1EE601AB4EE600AF1EE10FAB4EE401A94
:10125000C8BFB0EE600AF1EE10FAC8BFB0EE410AA6
:101260007047000080B540F66810C2F200000068C8
:10127000042108F0B7FC80BD80B54CF24002C2F2F8
:10128000010200201221132300F086F9002080BD06
:1012900080B5012001214FF0FF3208F0E3FC80BD52
:1012A0009FED010A704700BF0000C84380B540F6BB
:1012B0006810C2F200000068082108F093FC80BDAD
:1012C00080B54CF24000C2F20100C21D0120022193
:1012D000062300F061F9002080BD000080B50220E7
:1012E00001214FF0FF3208F0BDFC80BDF0B581B0A8
:1012F00000284FF0FE0700F097800C46002900F010
:1013000093804CF6E036C2F201060546307808B10B
:10131000FD2789E008F004FD40F66811C2F20001E3
:10132000002808607BD000207E21B622EC6200F00D
:101330008FF901201421B62200F08AF91E2000F056
:1013400077FE00201E2100F04DF90020002100F062
:1013500049F91E2865D101200021012400F042F93D
:101360000F2860D1032000F04FFD042000F04CFD59
:1013700041F24952C0F6000200200121002700F08E
:101380002DFE41F26521C0F60001032000F082FD30
:1013900041F2AD21C0F60001042000F07BFD0020E9
:1013A0004021AA2200F054F900204121012200F03E
:1013B0004FF900205321082200F04AF9002058215B
:1013C000042200F045F900207D21042200F040F9BC
:1013D000322000F02DFE01200F21012200F038F90B
:1013E00001201021032200F033F9012016210022F0
:1013F00000F02EF901201821012200F029F9012026
:101400001521802200F024F90A2000F011FE0320AB
:10141000347000F011FD042000F00EFD04E0FE2702
:1014200002E0FC2700E0FC2778B201B0F0BD00002C
:10143000002841D04CF24001C2F20101B1F9012073
:101440009FED1F3A00EE102AB8EEC00A80EE030AA4
:10145000B1F90330B1F905C001EE103A02EE10CA3D
:10146000B8EEC11AB8EEC22A81EE031A82EE032A40
:101470004FF60003CFF6FF7380ED040A4A7C897CA7
:10148000D20042EA51120021B1EB922F80ED051AF1
:1014900080ED062A18BF1A4300EE102AB8EEC00AE3
:1014A000B4EE001A20EE010AB3EE071A30EE010A7C
:1014B00080ED0A0A48B27047FE2148B2704700BF6B
:1014C00000A0AA45C0B34CF24001C2F20101B1F93B
:1014D0000720B1F90930B1F90B1000EE102A01EE26
:1014E000103A9FED172A03EE101AB8EEC00AB8EEB4
:1014F000C11AB8EEC33A80EE020A81EE021A83EEF8
:10150000022A9FED103AC16A91ED014A91ED025A0B
:1015100020EE030A21EE031A22EE032A91ED003A8F
:1015200031EE441A30EE430A32EE452A80ED070AC6
:1015300080ED081A80ED092A6FF00100704700BFA6
:101540006F12034235FA8E3C10B5012000F08CFC7E
:1015500040F66814C2F2000438B90120012100F0FD
:10156000BFFC2068012108F03DFB022000F07CFC5C
:10157000002818BF10BD0220012100F0B1FC206836
:10158000022108F02FFB10BD80B50C2001214FF087
:10159000FF3208F067FB80BD002A08BF704770B5B6
:1015A0001C4615460E4618B1012805D1022000E060
:1015B0000120002100F094FC40F2385146F08000F8
:1015C000C2F20001087000200122002300F016FD85
:1015D000002029462246012300F0E6FCBDE87040C9
:1015E00070470000F0B581B0044601200D46012689
:1015F00000F01EFD14B1012C04D10226304600215A
:1016000000F06EFC40F23856C2F2000645F0800051
:10161000374607F8010B002031460122002301253F
:1016200000F0ECFC002031460222002300F0BCFC5C
:1016300034B1012C09D140F23857C2F2000702251B
:101640002846012100F04CFC3878C0B201B0F0BD52
:10165000B0B5044601F07F0040F23851C2F20001FB
:10166000087001204A70012500F0E2FC14B1012C41
:1016700004D102252846002100F032FC40F2385106
:10168000C2F2000100200222002300F0B7FC24B1C6
:10169000012C18BFB0BD022000E00120012100F0A4
:1016A0001FFCB0BD2DE9F04381B04DF2FC08C2F241
:1016B00001080646D8F8000014460D466421002AA9
:1016C00008BF0A2408F0F8F908B1FB242FE040F223
:1016D0008079C2F20009D9F8000000E0006930B159
:1016E0000178B142FAD14168A942F7D11AE0142039
:1016F00000F00EFC88B1074620461C21002208F0AD
:1017000031F9B86058B1D9F800003C7300243E703C
:101710007D603861C9F8007005E0FE2403E03846BA
:1017200000F06EFBFF24D8F8000008F03BFA60B22E
:1017300001B0BDE8F08300007047000040F2807205
:10174000C2F20002126800E01269002A04BF002001
:10175000704713788342F7D153688B42F4D1906875
:1017600070470000D0E90212081FB0FA80F14FF074
:10177000020008BF0320022A18BF48097047000072
:1017800040F28C524CF68011C2F200020128C2F2E3
:10179000010118BF0022002818BF1146012888BF88
:1017A00000210846704700002DE9F041154640F23F
:1017B0001472C2F200021278012A11D1A5B14DF2C1
:1017C000FC08C2F201080746D8F800000E46642162
:1017D0001C4608F071F958B1FB2040B2BDE8F08119
:1017E000FD2040B2BDE8F081FE2040B2BDE8F081AE
:1017F00038463146FFF7A2FFD8F8001006460846E3
:1018000008F0D0F966B1304629460022234608F098
:1018100065F8002818BF4FF0FF3040B2BDE8F081F6
:10182000FC2040B2BDE8F0812DE9F0478AB040F2DB
:101830001477C2F20007387808B1FD248AE040F23C
:10184000E830C2F200006821FEF7A1FE002400BFCC
:10185000E0B200F03BFA0134012CF9D040F2F8601C
:1018600041F23971C2F20000C0F6000101600020AF
:10187000002408F04BF94DF2FC01C2F201010028EE
:10188000086066D0E8464FF001094046282187F8F5
:101890000090FEF77CFE4CF68016C2F201064FF077
:1018A0000E0A30464146CDE90244CDE90799CDF80C
:1018B00024A0049401F0D8FE304602F0A5FA41F6C7
:1018C000D512C0F600020020062100F051F841F6C2
:1018D0006945C0F60005002000212A4600F048F8BE
:1018E000002001212A4600F043F8002002212A4668
:1018F00000F03EF83046032101F058FE40F28C56CD
:10190000C2F2000630464146CDE9049A01F0ACFE31
:10191000304602F079FA41F69922C0F60002012021
:10192000082100F025F8012000212A4600F020F8C7
:10193000012001212A4600F01BF8012002212A463D
:1019400000F016F83046112101F030FE87F80090C3
:1019500000E0FF2460B20AB0BDE8F08780B540F235
:10196000F862C2F200021268002A18BF904780BDD8
:1019700040F21473C2F200031B78012B1EBFFD233B
:1019800058B270473AB101284FF0FF0398BF0C29B5
:1019900004D958B27047FE2358B2704740F2E83C71
:1019A000C2F2000C342310FB03C0002340F82120B6
:1019B00058B2704780B540F21473C2F200031B782E
:1019C000012B03D1FFF76EFE40B280BDFD2040B277
:1019D00080BD00002DE9F04F93B003A80D300190B9
:1019E0004FF0000A0CAE002005E000BF029800286E
:1019F00000F101004CD15FFA80FB02905846FFF7DE
:101A0000BFFE0028F2D0044609E000BF02F06CFDE2
:101A10000990384603A90022002307F0F3FF20466F
:101A2000002101F0A3FE0028E0D02046002132462C
:101A30000AAB01F0ABFE0028F1D10E980028304629
:101A400018BF043005683046FFF78CFE80462846F4
:101A50004146FFF783FF814658464946FFF76EFE31
:101A60000028DCD00746DDE90F02CDF80CA00028E5
:101A7000CDE908AACDE906AA8DF80C80CDE9045974
:101A80008DF81820C2D101980AA9FEF701FDBDE723
:101A900013B0BDE8F08F00002DE9F04F93B003A81C
:101AA0000D3001904FF0000A0CAE002005E000BFA1
:101AB0000298002800F101004CD15FFA80FB0290EF
:101AC0005846FFF75DFE0028F2D0044609E000BF4B
:101AD00002F00AFD0990384603A90022002307F00E
:101AE00091FF2046012101F041FE0028E0D0204670
:101AF000012132460AAB01F049FE0028F1D10E98CF
:101B00000028304618BF043005683046FFF72AFE2B
:101B1000804628464146FFF721FF81465846494600
:101B2000FFF70CFE0028DCD00746DDE90F02CDF8F8
:101B30000CA00028CDE908AACDE906AA8DF80C80F2
:101B4000CDE904598DF81820C2D101980AA9FEF7F1
:101B50009FFCBDE713B0BDE8F08F00002DE9F04316
:101B600089B0174640F21472C2F200021278012ABC
:101B700004D10446012806D9FF2000E0FD2040B230
:101B800009B0BDE8F08301F0FE001D460E460228B4
:101B900002D00DB9FE20F2E7DDF84080B8F1080F61
:101BA00001D9FF20EBE72046FFF7EAFD98B1814617
:101BB0000020032E0890CDE90600CDE90400CDE910
:101BC0000200019009D8DFE806F0020A0D11019722
:101BD000002100200DE0FE20D1E7FF20CFE7029793
:101BE000002005E001970220002102E00220029778
:101BF0000421CDE903100020002DCDF814808DF8CC
:101C0000180018BFB8F1000F05D001A818302946F8
:101C10004246FEF73DFC484601F04AFE38B101A9B4
:101C200001F118026B46484601F0D4FC28B101A925
:101C3000204600F0A5F80138A1E700209FE700004A
:101C400079B180B582B00A6891F804C04B1D0021BB
:101C5000CDF800C0FFF782FF02B0BDE8804040B27F
:101C60007047FE2040B270472DE9F04389B001ACC7
:101C700004F118090025E84604E000BF002D05F135
:101C8000010520D1EFB23846FFF77AFD0028F5D0E4
:101C9000064600BF384600F027F80028EED130464F
:101CA00001F006FE0028E9D03846214600F02EF863
:101CB0000028E3D0304621464A46434601F08AFCDC
:101CC0000028E7D0DAE709B0BDE8F0834DF2C8217B
:101CD00000EBC010C2F2010101EBC0000021C0F80E
:101CE0000014C0F8041470474DF2C82100EBC01076
:101CF000C2F2010101EBC000D0F80014D0F80404D6
:101D0000081AB0FA80F0400970470000002904BFAB
:101D1000002070472DE9F0414DF2C82C00EBC012B5
:101D2000C2F2010C0CEBC202D2F800E4D2F8043487
:101D30009E451FD002F204452C6800EBC0100CEB4E
:101D4000C00000EB4412640150F804C0D2E90180E5
:101D50005769D2E90364C1E900C8C1E90447C1E990
:101D60000206D2E90620C1E906202868013000F009
:101D70001F002860BEEB030018BF0120BDE8F08102
:101D800001284FF0000238D8B9B32DE9F0474DF2E1
:101D9000C82C00EBC012C2F2010C0CEBC202D2F84C
:101DA0000034D2F804E4013303F01F0373451ED05E
:101DB00002F58069D9F8004000EBC0100CEBC000C0
:101DC00000EB44124FEA441AD1E904C6D1E9007885
:101DD000D1E9025440F80A705661C2E9034CC2E9E5
:101DE0000185D1E90610C2E90610C9F80030B3EB4D
:101DF0000E0218BF0122BDE8F047104670470000F0
:101E000080B508F0C9FE80BD05284FF0FF0211D84B
:101E100001460620DFE801F0080E0E0305070A2040
:101E200002E0172000E0092080B502F011FD002239
:101E3000BDE8804050B2704705284FF0FF0211D82E
:101E400001460620DFE801F0080E0E0305070A2010
:101E500002E0172000E0092080B502F0FDFC00221E
:101E6000BDE8804050B27047062884BF002070470C
:101E700080B54EF27041C0F6000101EBC00252681D
:101E800031F83010104602F023FB0138B0FA80F030
:101E9000400980BDB9B1062882BFFF2040B270471B
:101EA0004EF27042C0F6000232F830C0002000232B
:101EB0002CFA00F2D20709D10E2B03F1010300F135
:101EC0000100F5D908E0FE2040B2704740F25042D0
:101ED000C2F2000242F82010002040B27047000019
:101EE000062882BFFF2040B2704780B50A464EF2F6
:101EF0007041C0F6000101EBC0035B6831F830109F
:101F0000184602F0EBFA0020BDE8804040B270476E
:101F100080B508F051FC80BD00281EBFFF2040B2F4
:101F20007047B7EE001A4CF61430B4EE410AC2F214
:101F30000100F1EE10FAC8BFB0EE410A00689FED53
:101F40000C1AC16AB5EE400A0131F1EE10FAB8BFC1
:101F5000B0EE410A01EE101AB8EE411A20EE010A65
:101F6000BCEEC00A80ED0D0A002040B2704700BFF1
:101F70000000000010B510B1FF2460B210BD4CF697
:101F80001430C2F201000021002403F02BFE60B2E5
:101F900010BD00004CF6BC21C2F20101002818BFA0
:101FA000002108467047000070B510B1FF2040B214
:101FB00070BD1E4614460D46FFF7ECFF0028F5D015
:101FC0002946224616B103F0CFF802E0142303F0AD
:101FD00011F8002818BF012040B270BD002A0FBFC1
:101FE000FE204CF20C03C2F2010303EB40101CBFB5
:101FF00040F82120002040B27047000070B510B1B9
:10200000FF2040B270BD1E4614460D46FFF7C2FFCA
:102010000028F5D02946224616B103F093FB02E0D2
:10202000142303F03BF9002818BF012040B270BD13
:1020300070B5044607F0E8FB0546FF2607F0C6FB2F
:10204000411C05290BD80120884010F0310F0BD11D
:1020500010F0060F0AD0204602F034F911E06FF0BC
:102060000041884218BF002670B270BD4FF47A70EC
:10207000B0FBF5F1B4FBF1F0A14288BF012007F0FD
:102080007BFB002670B270BD2DE9F04107F0BCFB70
:10209000044609F061FF4FF47A784EF21806B8FB57
:1020A000F4F4CEF20006376804FB00F509F054FFA3
:1020B00060433168854208BF394656F8042C01FB5D
:1020C00008F10132B1FBF2F100FB08F0401A00F513
:1020D0007A700021BDE8F08180B582B001680A689D
:1020E000D20614D5002201920A6801924968019132
:1020F000019907F001F840F2944100EBC000C2F2F0
:10210000000101EB8000006A002818BF804702B080
:1021100080BD0000FEE7000080B54CF68010C2F2E2
:10212000010001F0D9FB80BD80B54CF68010C2F2F1
:10213000010001F0D1FB80BD80B54CF68010C2F2E9
:10214000010001F0C9FB80BD80B540F28C50C2F2A5
:10215000000001F0C1FB80BD80B540F28C50C2F29E
:10216000000001F0B9FB80BD80B540F28C50C2F296
:10217000000001F0B1FB80BD4FF0030160B146F2F9
:1021800000420068C4F2000202F58063984208BF72
:102190000121801A08BF0146C8B270472DE9F04FEF
:1021A00081B02DED028B804600284FF0FE0000F03C
:1021B000B7800D46002900F0B380FFF765FFD8E92E
:1021C0000023801A99410CF05CF89FED580A01EE4B
:1021D000100A81EE000A88ED020AFFF755FFC8E9F0
:1021E00000014046294600F0A5F808B1FD2097E01F
:1021F00098F80C0001280AD0002840F090800020B8
:102200009FED4B0AC8F81000C8F8140011E095EDD6
:10221000020A95ED052A95ED031A95ED043A20EE94
:10222000020A22EE011A88ED040A22EE030A88ED62
:10223000051A88ED060A98ED040A08F24C4004F0ED
:1022400009F888ED040A98ED050A08F26C4004F0DC
:1022500001F888ED050A98ED060A08F28C4003F0B3
:10226000F9FF404688ED060A00F0A6F99FED308A96
:1022700040F25C5A6FF00F0640F2AC4940F22C5B22
:102280004FF48077C2F2000A08EB060494ED180AB6
:10229000D4ED380A84ED1C0AD8ED021A08EB0705C4
:1022A0002846B0EE481A05F021F80AEB060080ED4A
:1022B000040AD4ED340AD8ED021A05F1F000B0EEAC
:1022C000481A05F013F808EB0B0084ED240A03F01C
:1022D000C1FF04F2DC5080ED000A94ED100AD4ED49
:1022E0002C0A84ED200AD8ED021A05F5F070B0EE44
:1022F000481A04F0FBFF08EB090084ED280A03F0FC
:10230000A9FF04F2CC50043609F120090BF1200B8F
:1023100007F13C0780ED000AB6D1002000E0FD2067
:1023200040B2BDEC028B01B0BDE8F08F00247449CF
:1023300000000000F0B1F0B581B004460D464FF446
:10234000807700BFE61906F5F07005F0CFF806F1CA
:10235000F00005F0CBF8304605F0C8F83C37B7F58B
:10236000F87FEFD128792073002001B0BDE8F0405C
:1023700040B27047FE2040B270470000F0B581B017
:10238000044600F5B7666025D4F8280496ED010AE6
:102390002844371D04F0A6FBD4F8280496ED050A5E
:1023A0002844203004F09EFB0835802D3E46EBD1BA
:1023B000D4F82804603004F061FAD4F8280480309E
:1023C00004F05CFA01B0F0BD002864D02DE9F047BC
:1023D0002DED088B8246406990F80480B8F1000F1B
:1023E0005CD008EB88009FED6F8A9FED6F9A4FEAF3
:1023F000400900270425B7EE00AABFEE00BA002668
:1024000000242BE0DAF82000DAF84811284490ED97
:10241000000AC81903F01EFF80EE091ADAF87C00E2
:10242000DAF88410304480ED000A0A348819043642
:1024300020371035B4EE4A1AF1EE10FAC8BFB0EEEC
:102440004A1AB4EE4B1AF1EE10FAB8BFB0EE4B1ABE
:1024500038EE018AA14580ED001A21D0DAF8140087
:10246000C06A204404F08EFBDAF81400C06A2044ED
:1024700004F0A2FA0028C5D0DAF8201000F12C0EE2
:102480009EE80850806B01EB860241F82630C2E9D5
:1024900001CED060B6E7FF2040B270479FED418A81
:1024A00000EE108AB8EEC00A88EE000ADAF81400CE
:1024B00030308AED220A04F065FBDAF8140030307F
:1024C00004F07AFA01460AF128005022FEF725F8B6
:1024D000DAF814009AED1C1A90ED020A20EE010AB7
:1024E000B5EE400AF1EE10FA8AED1E0A0BDA9FED06
:1024F0002F1A00BF30EE010AB5EE400AF1EE10FAD5
:10250000F8DB8AED1E0A9AED1E0A9FED281AB4EE3A
:10251000410AF1EE10FA0ADB9FED252A30EE020A9D
:10252000B4EE410AF1EE10FAF8DA8AED1E0A9AF8D2
:10253000500000281CBF31EE400A8AED1E0A9AEDB9
:102540000D0A0AF5A87003F085FE9AED0D1A9FEDAD
:10255000192A8AED200A81EE021AB7EE000AB4EEBB
:10256000401AF1EE10FAC8BFB0EE401ABFEE000AF2
:10257000DAF82000B4EE401AF1EE10FAB8BFB0EE6F
:10258000401A90ED010A90ED052A8AED231A30EEEB
:10259000420A8AED640A0020BDEC088BBDE8F047D2
:1025A00040B270470000000000C0DA45DB0FC940B0
:1025B000DB0FC9C000409C452DE9F04F81B02DEDE7
:1025C000028B86B0077B0446012F3AD1206920F0A8
:1025D00000400BF001FE9FED2A0B55EC106B3246CC
:1025E0002B460BF039FE60BB606920F000400BF019
:1025F000F3FD32462B460BF02FFE10BBA06920F0F6
:1026000000400BF0E9FD32462B460BF025FEC0B929
:1026100094F8D00304F1400C002804BF012084F892
:10262000D0030020C4E90800C4E90A00D4F8AC05CE
:10263000D4F8B015D4F8B425D4F8B8358CE80F0028
:1026400030E2002084F8D0036FF00F0021180A6DEB
:102650000430C1F8BC25F9D1002F00F01382012FFE
:102660001AD0022F40F01E820020C4E90800C4E9FD
:102670000A00C4E91000A06402E200BF00BF00BF6E
:102680009A9999999999B93FCC3B7F669EA0E63F6C
:10269000CD3B7F669EA0E63FD4E9040AA5690BF016
:1026A0009BFD8046284689460BF096FD1FED0A0BE0
:1026B00006465BEC102B5B460F460292CDF814B039
:1026C0000BF01EFA42464B460AF000FF02460B464C
:1026D0000BF016FA8146504688460BF07DFD1FED43
:1026E000140B05468A4653EC102B30463946CDE98B
:1026F00003230BF005FA2A4653460AF0E7FE02468A
:102700000B460BF0FDF902460B46484641460AF0DF
:10271000DDFE41EC100B0AF0FBFB51EC100B0AF054
:10272000A3FE2062D4E90408A5690BF055FD074615
:1027300028468A460BF050FD029A5B4606468946BB
:102740000BF0DEF93A4653460AF0C0FE02460B464D
:102750000BF0D6F9824640468B460BF03DFDDDE995
:10276000032305460F46304649460BF0C9F9024699
:102770000B46284639460BF041FC02460B460BF04F
:10278000BFF902460B46504659460AF09FFE41ECFF
:10279000100B0AF0BDFB51EC100B0AF065FE6062F5
:1027A000D4E90401A56901910BF016FD07462846FE
:1027B00089460BF011FDDDF80880059B4246064670
:1027C0008B460BF09DF902460B46384649460BF006
:1027D00015FC02460B460BF093F9814601988A4698
:1027E0000BF0FAFCDDE9032307460D463046594657
:1027F0000BF086F902460B46384629460BF0FEFBE5
:1028000002460B460BF07CF902460B464846514601
:102810000AF05CFE41EC100B0AF07AFB51EC100B55
:102820000AF022FEA062D4E9040AA5690BF0D4FCE8
:102830000746284689460BF0CFFC059B42460646D4
:102840008B460BF05DF902460B46384649460BF0C5
:10285000D5FB02460B460BF053F98146504688469D
:102860000BF0BAFC0D465946DDF80CA0DDF810B0AF
:102870000746304652465B460BF042F93A462B4635
:102880000AF024FE02460B460BF03AF902460B46CC
:10289000484641460AF01AFE41EC100B0AF038FB9C
:1028A00051EC100B0AF0E0FDE062D4E90480A66967
:1028B0000BF092FC0546304689460BF08DFC5246E3
:1028C0005B4606460F460BF01BF92A464B460AF0BC
:1028D000FDFD41EC180B40460BF07EFC029A059B77
:1028E00005468846304639460BF00AF92A464346E3
:1028F0000AF0ECFD41EC110BB0EE480AF0EE680A6C
:102900000AF02EF851EC100B9FEDB10B53EC102B8D
:10291000CDE900230BF0F4F80AF0A6FD2064D4E919
:1029200004A0A6690BF058FC054630468B460BF018
:1029300053FCDDF80C90049B4A4606460F460BF00C
:10294000DFF802460B46284659460BF057FB41EC90
:10295000180B50460BF040FCDDF80880059B05463F
:102960008A463046394642460BF0CAF82A46534654
:102970000AF0ACFD41EC110BB0EE480AF0EE680A2B
:1029800009F0EEFFDDE9002351EC100B0BF0B8F875
:102990000AF06AFD6064D4E904A0A6690BF01CFC8F
:1029A000054630468B460BF017FC4A46DDF8109082
:1029B00006464B460F460BF0A3F802460B46284648
:1029C00059460BF01BFB41EC180B50460BF004FC76
:1029D0004246DDF8148005468A463046394643466D
:1029E0000BF08EF802460B46284651460BF006FBCC
:1029F00041EC110BB0EE480AF0EE680A09F0B0FFA6
:102A0000DDE9002351EC100B0BF07AF80AF02CFDF5
:102A1000A064D4E904A0A6690BF0DEFB05463046AD
:102A20008B460BF0D9FB039A4B4606460F460BF03C
:102A300067F82A465B460AF049FD41EC180B504600
:102A40000BF0CAFB029A05468A4630463946434691
:102A50000BF056F802460B46284651460BF0CEFACC
:102A600041EC110BB0EE480AF0EE680A09F078FF6D
:102A7000DDE9002351EC100B0BF042F80AF0F4FCF6
:102A8000E0640FE00020C4E90800C4E90A0048F24D
:102A900000000021C4F29D30C4F23421C4E91001C9
:102AA000C4E912019FED4C0A04F14000002100BF6F
:102AB000421892ED001A0431B5EE401AF1EE10FA08
:102AC000BCBF31EE001A82ED001A1029F0D19FED43
:102AD000431A9FED432A9FED433A9FED434A9FEDF2
:102AE000435A4CF230010020C2F201010FE000BF56
:102AF000B1EE476A82ED0C6A97ED006A93ED007AB9
:102B000036EE076A0130042882ED146A57D004EBD0
:102B1000800292ED106A92ED347A01EB800336EE7A
:102B2000476AB4EE416AF1EE10FA83ED006A08DDFF
:102B300036EE026AB4EE416AF1EE10FAF8DC83ED8B
:102B4000006A93ED006AB4EE436AF1EE10FA08DA17
:102B500036EE006AB4EE436AF1EE10FAF8DB83ED6C
:102B6000006AB4EE446AF1EE10FA02F1D0070FDD0C
:102B7000B4EE416AF1EE10FA0ADC166A97ED006ACB
:102B8000166393ED007A36EE076A36EE036AB9E70C
:102B900092ED087AB4EE456AF1EE10FAA8DAB4EED6
:102BA000436AF1EE10FAA3DB82ED0C7A97ED006A2E
:102BB00093ED007A36EE076A36EE016AA2E706B0B8
:102BC000BDEC028B01B0BDE8F08F00BF00BF00BFBD
:102BD00000000000DCA54C400000B443000034437A
:102BE0000000B4C3000034C30000B4420000B4C20B
:102BF000002870D0F0B581B02DED0C8B044604F0A8
:102C000025F89FED399A9FED39AA9FED39BA9FEDCE
:102C100039CA9FED338B9FED38DA0025802600BF3F
:102C2000D4F82804304403F0C7FE183003F0F8FD50
:102C300080EE090AD4F828046719304420EE0A0A05
:102C400087ED340A03F0B8FE183003F0F1FD80EE92
:102C50000B0AD4F828043044203887ED300A03F0FA
:102C6000ABFE183003F0E4FD80EE0C0A07F583603C
:102C700097ED341A90ED002A87ED280A31EE420ACA
:102C800010EE100A0BF0A8FA41EC100BB0EE481A47
:102C9000F0EE681A0AF0BAF851EC100B0AF0E4FBF7
:102CA00000EE100AB5EE400AF1EE10FA05F1040547
:102CB00030EE0D1AB8BFB0EE410A102D06F108062D
:102CC00087ED340AACD10020BDEC0C8B01B0BDE81F
:102CD000F04040B27047FE2040B2704700BF00BFD6
:102CE0000000000000807640DB0F494000003443C4
:102CF0000000A04300401C460000B44390ED001AC1
:102D0000F5EE400AF1EE10FA31EE000A10DDB4EEF5
:102D1000600AF1EE10FAA2BF30EE600A80ED000A00
:102D20007047B5EE400AF1EE10FAB8BF30EE200A57
:102D300080ED000A70470000B5EE401AF1EE10FA7F
:102D400030EE600AD8BF7047B6EE002A21EE022AA4
:102D5000B4EE420AF1EE10FAC4BF30EE410A7047F9
:102D6000B1EE422AB4EE420AF1EE10FAB8BF30EEEC
:102D7000010A704790ED001AB4EE601AF1EE10FAF5
:102D8000C8BFC0ED000A90ED001AB4EE401AF1EE93
:102D900010FAB8BF80ED000A7047000040F204004E
:102DA000C2F20000704700002DE9F04381B040F20C
:102DB0000408C2F20008D8F88451D8F8986105EBED
:102DC00085004000FFF7A4F8C8F8AC01A0B3B0003C
:102DD000FFF79EF8C8F89C0190B3012D20DB4FF05F
:102DE000000C40F2012E4FF0FF390123002100209A
:102DF000D8F8AC615EFA80F759FA80F401EB8101F2
:102E00000130B4FA84F406EB410206F81130C1B285
:102E100064098D4257801371547182F806C0E7DC53
:102E2000D8F8AC11D8F89C0101220A728A744FF0CC
:102E30007E510160002006E0FEF7E2FFFF2002E085
:102E4000FEF7DEFFFF2040B201B0BDE8F0830000D6
:102E500080B54CF60820C2F2010001F0D3F880BD25
:102E600080B54CF6A810C2F2010001F0CBF880BD8D
:102E700080B540F2B450C2F2000001F0C3F880BD4A
:102E8000D0F800C06FF00F024AF6AB2352FA8CF272
:102E9000CAF6AA230146A2FB0330000905A31B5C66
:102EA00040F2FF302CEA00005F2A88BF0430C1E9FD
:102EB0001603704700061016000610168269816A14
:102EC000B2F5005F06D06AB9022912D0012914D0E8
:102ED000D1B90EE0032917D8DFE801F0020B020F89
:102EE0000120704703293CBF012070471CBF002010
:102EF0007047C06AC0F300607047C06AA0F1C0703C
:102F0000B0FA80F0400970470020704780B5D0F8D3
:102F100000C0D0F808E0DCF80000BEF1400F20F45B
:102F20008020CCF800000846CCF8043004BF1046DE
:102F30000A46CCF80800CCF80C2080BD7047000091
:102F400080B5012001F0E8F980BD000080B50820BF
:102F500001F0E2F980BD000080B5102001F0DCF93D
:102F600080BD000080B5202001F0D6F980BD0000B2
:102F700072B600BFFEE7000070B52DED0A8B044667
:102F800000284FF0FF0000F05B810D46002900F0A3
:102F90005781FFF779F8D4E90023801A99410BF0A3
:102FA00070F99FEDA90A01EE100A81EE000A84ED86
:102FB000020AFFF769F82A78C4E9000120461146A1
:102FC00000F04CFA94ED020A95ED011A95ED022AF3
:102FD00004F52F7004F52C7121EE00AA20EE02CA30
:102FE00006F0A8FB94ED091AB0EE409A9FED97BA4F
:102FF00094ED870A39EE011A7AEE010AB0EE4B1A07
:1030000004F12405FFF798FE94ED091AB0EE408A0A
:1030100094ED880A39EE011A7AEE010AB0EE4B1AE5
:10302000FFF78AFE207CB0EE409A022807D00128E4
:103030005ED0002804BF0020C4E99D00EFE004F545
:10304000337004F52D7106F075FBE06894ED063AD7
:1030500090ED4A2A90ED491A84ED050A32EE400AB5
:1030600004F50B7631EE431A84ED080A3046B0EED3
:103070004A0AF0EE4B0A84ED071AFFF73FFE94ED83
:103080008B0AB4EE4B0AF1EE10FA05DB9FED701AD5
:1030900030EE010A86ED000AE16894ED071A91ED21
:1030A000510A91ED502A04F50C7030EE010A72EECF
:1030B000410A84ED8CCAFFF75DFEE06894ED071AC3
:1030C00094ED080A94ED8B2A94ED8C3A007830EE5A
:1030D000020A31EE031A84ED090A84ED0A1A78B364
:1030E0002846B0EE490AF0EE480AFFF743FE34E006
:1030F000E06894ED090A00783AEE000A84ED090AC6
:1031000038B12846B0EE490AF0EE480AFFF732FE21
:103110000CE09FED501AB4EE410AF1EE10FA05DD15
:103120009FED4B1A30EE010A85ED000AE06894ED40
:103130000A0A41783CEE000A84ED0A0A81B917E0D8
:103140009FED441AB4EE410AF1EE10FA05DD9FED51
:10315000401A30EE010A85ED000AE068417839B185
:10316000D0ED500A90ED510A04F12800FFF702FE5D
:103170009FED39AAD4ED021A94ED090AD4EDAC0AF8
:1031800004F13C00B0EE4A1A04F0B0F8D4ED021A93
:10319000D4EDAB0A04F17800B0EE4A1AB0EE408AE2
:1031A00004F0A4F884ED9D0AD4ED021A94ED0A0A05
:1031B000D4EDAD0A04F1B400B0EE4A1A04F096F86A
:1031C000D4ED021AD4EDA90A04F1F000B0EE4A1AC7
:1031D000B0EE409A04F08AF8E06884ED9E0A90F818
:1031E0002C1169B194EDAB2A90ED4C1A94ED9D3AF7
:1031F00038EE422A21EE021A33EE011A84ED9D1AAE
:1032000090F82D1159B194EDA91A90ED4D2A39EE8F
:10321000411A22EE011A30EE010A84ED9E0A94ED65
:103220009D0A04F50D7003F015F884ED9D0A94EDE8
:103230009E0A04F5157003F00DF8002084ED9E0A37
:1032400040B2BDEC0A8B70BD00247449DB0FC9404D
:10325000DB0FC9C0DB0F49400000000010B52DEDA9
:10326000028B002800F08C800446C160002020748E
:1032700004F13C0001F144020121B0EE408A04F067
:10328000EDF8E16804F1780001F124020121B0EECB
:10329000480A04F0E3F8E16804F1B40001F18402A3
:1032A0000121B0EE480A04F0D9F8E16804F1F00019
:1032B00001F164020121B0EE480A04F0CFF8E168A0
:1032C00004F5B47001F1C4020121B0EE480A04F023
:1032D000C5F8E16804F5967001F1A4020121B0EE91
:1032E000480A04F0BBF8E16804F5F07001F5827259
:1032F0000121B0EE480A04F0B1F8E16804F5D2709B
:1033000001F1E4020121B0EE480A04F0A7F8E068F8
:10331000B0EE480AD0F84811C4F81C12D0F84C118D
:10332000C4F82012D0ED4E0A04F50D7002F0D0FF63
:10333000E068B0EE480AD0ED4E0A04F5157002F0D0
:10334000C7FFFEF771FAE068C178012902D11C308D
:1033500003F06CFBE0688178012902D1143003F09E
:1033600065FBE068C17831B90C3003F03DF9E068E5
:103370000C3003F04BF8E068817819B1002009E0C7
:10338000FF2007E0043003F02FF9E068043003F079
:103390003DF8002040B2BDEC028B10BD10B50446D4
:1033A000C068C178012908D11C3003F067FAE068D1
:1033B00094ED9D0A1C3003F095FBE06881780129AB
:1033C00008D1143003F05AFAE06894ED9E0A1430E4
:1033D00003F088FBE0688178E1B9D0F86C1194EDD6
:1033E0009E0AC4F89812D0F87411C4F8A012D0F84C
:1033F0007011C4F89C12D0F86811C4F8941290EDC2
:103400005F1A04F5247120EE010A043084EDA40A49
:1034100003F056F8E068C178002918BF10BDD0F855
:10342000581194ED9D0AC4F88412D0F86011C4F8C4
:103430008C12D0F85C11C4F88812D0F85411C4F87A
:10344000801290ED5E1A04F51F7120EE010A0C3017
:1034500084ED9F0A03F034F810BD0000B0B52DEDE7
:10346000028B58B30446007C0D46884226D004F1F6
:103470003C0004F03BF804F1780004F037F804F164
:10348000B40004F033F804F1F00004F02FF89FEDDD
:103490000D8A04F50D70B0EE480A02F06BFF04F5DA
:1034A0001570B0EE480A02F065FF04F12400FDF744
:1034B00081FAD4E9AC012574C4E90901BDEC028BA1
:1034C000B0BD00BF0000000010B5002859D0044670
:1034D000C068C178012911D11C3003F053FBE068AA
:1034E0001C3003F069FA48B100F108030ECB4069C3
:1034F00004F52F7C8CE80E00C4F8C802E0688178DF
:10350000012911D1143003F03DFBE068143003F0C1
:1035100053FA48B100F108030ECB406904F5337C3F
:103520008CE80E00C4F8D802E068C17889B90C3084
:1035300003F026F9E0680C3002F096FF48B100F184
:103540001C030ECB806A04F52F7C8CE80E00C4F8B7
:10355000C802E068817889B9043003F011F9E068A5
:10356000043002F081FF48B100F11C030ECB806AE9
:1035700004F5337C8CE80E00C4F8D802002040B279
:1035800010BDFF2040B210BD68B18B68D1E900C208
:10359000C0F8AC32C0E9A9C2D1E903234969C0E946
:1035A000AC23C0F8B8124FF0FF30704790F82020DD
:1035B000013A012A04D8006800F11402002004E056
:1035C00000F1240201204FF4802113681943116097
:1035D0007047000010B590F820E0D0F800C0AEF1C0
:1035E000010EBEF1010FDCF808E00ED81EF0E05F1E
:1035F00011D0CEF3016E012000FA0EF018608B6836
:103600007BB1486843EAC0030DE000F124010120CA
:103610004FF4802223E000F1240101204FF4001236
:103620001DE008684305D1E9030403430CEB0E10C9
:10363000C0F88031C0F88441097D012905D100F529
:10364000C2710B6843F480730B605168C0F88C1131
:10365000126800F5C071C0F88821002001220B68B3
:103660001A430A6010BD0000B0B590F82020013A5E
:10367000012A2FD846F20060C4F20000026842F02E
:1036800001020260026822F47C520260D1F814E068
:10369000CC694A6A0368012C43EA022202600EF0F8
:1036A0001F024FF0010303FA02F2C3696FEA020C32
:1036B00023EA0203C36113D02CBBC36803EA0C03E3
:1036C000C360CB688C8844EA034300EBCE042364D8
:1036D0000B4611E0416A41F4802141620120B0BDF6
:1036E000C3681343C3600B688C8844EA034300EB50
:1036F000CE04236401F10C038C681B8843EA044365
:1037000000EBCE04636443688D6943EA0204D1F898
:1037100010E0096A002D08BF03EA0C044460436905
:10372000BEF1000F43EA020408BF03EA0C040129BA
:10373000446102D1C1691143C161016821F00101F5
:1037400001600020B0BD000080B5FEF715FD032824
:1037500008BF80BD40F2E831C2F20001342210FB04
:103760000210006B002818BF804780BD90F8202011
:10377000013A012A84BF0020704700681022002906
:1037800008BF0C22805800F00300704710B590F875
:103790002040013C012C0AD8046871B12469A407B7
:1037A0000ED100F1240101204FF4001276E000F167
:1037B000240101204FF4802270E0E468A40771D056
:1037C000046804EB011CDCF8B0410CF5D87E14F061
:1037D00004049460DCF8B04119BFE4085460640D3F
:1037E0001460DEF800400CF5DA7E04F00204D460C8
:1037F000DCF8B44124075ABFDEF8004004F00F049F
:1038000008241461DEF800400029C4F30724946101
:10381000DEF800404FEA14445461DCF8B8211A7015
:10382000026802EB0112D2F8B8214FEA12225A7054
:10383000026802EB0112D2F8B8214FEA12429A70E4
:10384000026802EB0112D2F8B8214FEA1262DA7074
:10385000026802EB0112D2F8BC211A71026802EB75
:103860000112D2F8BC214FEA12225A71026802EB0F
:103870000112D2F8BC214FEA12429A71026802EB9F
:103880000112D2F8BC214FEA1262DA71006814BF4B
:1038900000F1100100F10C01002020220B681A43F6
:1038A0000A6010BD00F1240101204FF40012F5E779
:1038B00090F820100139012984BF0020704700686A
:1038C000816882688068C1F38061C2F3C06211447C
:1038D000C0F30070084470472DE9F04F81B00446F2
:1038E00000684669D0F804908768D0F80CB0D0F82A
:1038F00010A0D0F81880F10703D1002530071CD4A0
:1039000023E0F90710D00121BA07816009D47807B4
:1039100000F1AA80380700F1B080204600F0A2FA3A
:1039200002E0204600F0B0FA0025F80500F184809E
:10393000F80300F1AA80300707D51BF0100004D06F
:10394000206845F400751021C160700708D51BF090
:10395000080005D020680821C160204600F0FAF96F
:10396000B00706D52068C068800702D0204600F066
:1039700003FA700607D51AF0100004D0206845F449
:10398000806510210161B00608D51AF0080005D045
:10399000206808210161204600F000FAF00606D5F3
:1039A00020680069800702D0204600F009FAB003C1
:1039B00008D519F0100005D020681021416020467C
:1039C00000F010FAF00308D519F0080005D02068BF
:1039D00008214160204600F0B1FA300440F18F80A8
:1039E0005FEA497040F1888006F4807008EA102090
:1039F00028435FEA8871014648BF41F00201B205E1
:103A000058BF01465FEA48700D4648BF45F00405BF
:103A1000700558BF0D4630056ED518F070006BD09C
:103A200010380009052862D8DFE800F00353565922
:103A30005C5F45F008055AE020684FF48071BA05D4
:103A400081600AD4780512D4380519D4204600F0D4
:103A50002DFAF8037FF56FAF17E0204600F038FA33
:103A6000F8037FF568AF10E04FF400655DE705F5FA
:103A70000055F8037FF55FAF07E04FF4805554E73A
:103A800005F58045F8037FF556AF20684FF4803187
:103A9000BA0381600AD478030FD4380313D42046C4
:103AA00000F028FA30073FF548AF4EE7204600F017
:103AB00033FA30073FF541AF47E705F500453007DA
:103AC0003FF53BAF41E705F5803530073FF535AFB2
:103AD0003BE745F010050AE045F0200507E045F01A
:103AE000400504E045F0800501E045F4807520685C
:103AF000816921F0700181612068042141602DB14C
:103B0000606A284360622046FFF71EFE01B0BDE8F0
:103B1000F08F0000B0B5C8B1044690F8200010B98D
:103B2000204600F071F82068016841F00101016051
:103B300000F0DAFC054600BF20684168C90707D1DC
:103B400000F0D2FC401B0B28F6D312E00120B0BDE0
:103B5000016821F00201016000F0C6FC054600BFCB
:103B60002068416889070DD500F0BEFC401B0B287A
:103B7000F6D3606A052140F400306062012084F8C9
:103B80002010B0BD217E0268012922F0800208BF0A
:103B900080320260617E0268012922F0400208BF83
:103BA00040320260A17E0268012922F0200208BF93
:103BB00020320260E17E0268012922F0100218BF63
:103BC00010320260217F0268012922F0080208BF3A
:103BD00008320260617F0268012922F0040208BFF6
:103BE00004320260D4E901C2D4E9033561691A43A1
:103BF0002A431143ACF101021143C16100200121AC
:103C0000606284F82010B0BD70B586B0006846F6DA
:103C10000002C4F2000200219042CDE90411CDE976
:103C20000211019137D046F20041C4F200018842EE
:103C300040F08D804CF20801C2F201010A6843F69F
:103C40004000C4F20200531C0B6052B900210091E5
:103C5000016841F000710160016801F0007100919C
:103C600000990021009150F8101C152441F0080122
:103C700040F8101C50F8100C142500F008000090BB
:103C800000980320019040F20040C4F2020000F5C9
:103C90000060132638E043F64000C4F202000091B1
:103CA000016841F080610160016801F0806100916C
:103CB00000994CF20801C2F201010A68531C0B6022
:103CC00052B900210091016841F000710160016862
:103CD00001F00071009100990021009150F8101C32
:103CE000412441F0020140F8101C50F8100C40250E
:103CF00000F00200009000984FF48250019040F2D2
:103D000000403F26C4F202000221029100210391EB
:103D1000032104910921059101A900F00BFB304614
:103D20000521002200F09CFD304600F095FD28465C
:103D30000521002200F094FD284600F08DFD20466C
:103D40000521002200F08CFD204600F085FD06B024
:103D500070BD000080B5FEF70FFA032808BF80BDD4
:103D600040F2E831C2F20001342210FB0210C069B7
:103D7000002818BF804780BD80B5FEF7FDF90328F5
:103D800008BF80BD40F2E831C2F20001342210FBCE
:103D900002108069002818BF804780BD80B5FEF7FB
:103DA000EBF9032808BF80BD40F2E831C2F2000100
:103DB000342210FB0210406A002818BF804780BDE3
:103DC00080B5FEF7D9F9032808BF80BD40F2E8317D
:103DD000C2F20001342210FB0210006A002818BF52
:103DE000804780BD80B5FEF7C7F9032808BF80BDB6
:103DF00040F2E831C2F20001342210FB0210806A66
:103E0000002818BF804780BDB0B5044690F8200058
:103E100001281DD1022084F820002068016821F0CB
:103E20000101016000F060FB054600BF20684068AA
:103E3000C00713D000F058FB401B0B28F6D3606A74
:103E400040F400306062052084F820000120B0BDFD
:103E5000606A40F4002060620120B0BD0020606212
:103E6000B0BD000080B5FEF787F9032808BF80BD0C
:103E700040F2E831C2F20001342210FB0210C068A7
:103E8000002818BF804780BD80B5FEF775F903286C
:103E900008BF80BD3421484340F2E831C2F200013E
:103EA0000858002818BF804780BD000080B5FEF785
:103EB00063F9032808BF80BD40F2E831C2F2000177
:103EC000342210FB02100069002818BF804780BD13
:103ED00080B5FEF751F9032808BF80BD40F2E831F4
:103EE000C2F20001342210FB02104068002818BF03
:103EF000804780BD80B5FEF73FF9032808BF80BD2D
:103F000040F2E831C2F20001342210FB0210406995
:103F1000002818BF804780BD80B5FEF72DF9032823
:103F200008BF80BD40F2E831C2F20001342210FB2C
:103F300002108068002818BF804780BD80B5FEF75A
:103F40001BF9032808BF80BD40F2E831C2F200012E
:103F5000342210FB0210C06A002818BF804780BDC1
:103F600070B5866D044600F0BFFA94F8351002294A
:103F700025D105462068216C026822F016020260F5
:103F8000426922F08002426109B9A16C19B101684D
:103F900021F008010160016821F00101016000BF0A
:103FA00020680068C0070ED000F09EFA401B06286B
:103FB000F6D320206065032084F835000CE08020D3
:103FC0006065012008E0E06D3F2101FA00F0B0607B
:103FD000012084F835000020002184F8341070BDE1
:103FE00090F83510022909D1052180F835100068B4
:103FF000016821F0010101600020704780214165C6
:1040000001207047F0B581B004460020009040F2D6
:104010000000C2F200000268D4E9166048F2B5134D
:1040200037680821C1F64E3381403942A2FB03258F
:104030000CD0226813685B0708D5136823F00403CB
:104040001360B160616D41F0010161650121814042
:10405000394208D022685269120604D5B160616DF8
:1040600041F00201616504218140394208D0226893
:104070001268920704D5B160616D41F00401616579
:1040800010218140394215D020680268120711D5ED
:10409000B16002680168520306D4C90506D40168FC
:1040A00021F00801016001E0080342D4216C09B14C
:1040B00020468847E16D202000FA01F23A4244D0C0
:1040C00020680368DB0640D5B26094F8353002689A
:1040D000052B1ED122F016020260426922F08002F6
:1040E0004261226C0AB9A26C1AB1026822F008027D
:1040F00002603F208840B060012084F83500216DC7
:104100000020002984F8340040D02046884701B0C0
:10411000F0BD0168520310D4C90512D4016821F022
:1041200010010160012084F83500002084F834007B
:1041300007E0A16C0029BBD1BCE7080301D4616C86
:1041400000E0E16B09B120468847606DF0B1606D19
:10415000C00717D0052084F835002068A90A026836
:1041600022F00102026000BF009A01328A420092EE
:1041700002D80268D207F7D1012084F83500002068
:1041800084F83400E16C09B12046884701B0F0BDE5
:104190002DE9F041044600F0A7F9C4B1054602201C
:1041A00084F835000020216884F83400086820F085
:1041B0000100086026683068C0070BD000F094F951
:1041C000401B0528F6D903212022032042E00120CC
:1041D000BDE8F081306848F23F01CFF21001251DA3
:1041E00000EA010C2ECDD4E9050E41EA0C01114381
:1041F00019432943D4E90778084340EA0E01606A6D
:104200003943042841EA080103D1D4E90B231143BF
:10421000194331607169042821F0070141EA000562
:104220000CD1D4E90A1045EA010538B12046FEF761
:1042300045FE18B10121402201200BE020467561A6
:10424000FEF71EFEE16D3F2202FA01F181600022BD
:1042500001210020626584F83510BDE8F08100007E
:10426000B0B5044690F83400012828D0012084F825
:104270003400A56D94F8350001281DD1022084F882
:104280003500002060652046FEF740FEE26D3F23CA
:10429000206803FA02F2216CAA60026842F016025A
:1042A000026019B1016841F008010160016841F044
:1042B000010101600020B0BD002084F8340002201C
:1042C000B0BD0000B0B5044600F00EF9054640F25E
:1042D0007C30C2F200000078611C18BF044400BFAB
:1042E00000F002F9401BA042FAD3B0BD70B540F215
:1042F000504604460025C2F2000603E00135102DA9
:1043000008BF70BD24FA05F0C007F7D056F82500A5
:10431000002818BF8047F1E780B543F61441C4F286
:1043200001010A68024208BF80BD0860FFF7DEFF96
:1043300080BD00002DE9F04F83B000F13E4202F154
:10434000FF724FEAB22241F600470192C4F202071F
:1043500008224FF0010E00254FF0000A4FF0000830
:10436000B84208BF072200920AE000BF08F1010826
:104370000AF1040AB8F1100F05F1020500F0A4805B
:104380000C680EFA08FB14EA0B09EFD04C6804F035
:10439000030CACF1010EBEF1010F11D803228768A6
:1043A00002FA05F6CA68B743AA403A4382604268F7
:1043B000C4F3001722EA0B0207FA08F73A434260F7
:1043C000BCF1030F1CD0C26803238E6803FA05F703
:1043D000BA4306FA05F73A43BCF1020FC2600FD1A7
:1043E0006FF0030202EA580202440AF01C060F238F
:1043F000176A03FA06F40B69A743B3403B43136201
:10440000026803234F68AB409A4307F00303AB40B5
:104410001A4317F4403F4FF0010E0260A6D000226D
:1044200043F644030292C4F202031A6843F60044BE
:1044300042F480421A601A68C4F2010402F4804215
:104440000292029A28F003024FF6084B2244CFF65C
:10445000FF7B52F80B300AF00C070F26BE4023EA10
:10446000060C019B009E072B38BF1E4606FA07F775
:1044700047EA0C0342F80B30A2684B6842EA09078E
:1044800043F60C4CDE0258BF22EA0907A760C4F2CB
:10449000010CDCF800209E0242EA090758BF22EA1C
:1044A0000907CCF8007062689E0342EA090758BF0A
:1044B00022EA090767602268DB0342EA090358BF62
:1044C00022EA0903236051E703B0BDE8F08F000042
:1044D0000069084018BF012070470000002A08BF8B
:1044E00009048161704700004DF6DC20C2F2010032
:1044F00000687047F0B581B0B0B3044690F83D0055
:1045000028B9002084F83C00204600F0BFF82420A1
:1045100084F83D002068016821F001010160016814
:1045200041F400410160016821F40041016000F0A4
:1045300061FA48F28041C0F21E0140F6001265683F
:1045400088424FF00001C0F23D0248F2A16C4FF0EA
:10455000000338BF01219042C0F2010C38BF012393
:10456000654538BF0B4613B1012001B0F0BD4DF6D3
:104570008361C4F21B31A0FB011221684FEA924E05
:104580004B684FF4967623F03F0343EA92434B6027
:1045900044F6D3530F6A0EFB06F6C1F26203A6FB84
:1045A000033627F03F03B709654538BF970C7A1CDF
:1045B0001A430A62CA6948F2A0674CF6FF73C0F258
:1045C0000107BD4222EA030C0AD801386A00B0FB99
:1045D000F2F001306FF31F30042898BF04202BE065
:1045E000A368A0F1010E9BB119206843BEFBF0F057
:1045F0000422013062F31F30000512D09BB1192054
:104600006843BEFBF0F00422013062F31F3011E07A
:1046100005EB4500BEFBF0F001306FF31F300005E5
:10462000ECD1012008E005EB4500BEFBF0F00130C5
:104630006FF31F3040F4004040EA0C00C861086886
:10464000D4E9072320F0C0001043184308608868AD
:1046500048F2FF3204F10C0790438CCF184310430B
:10466000A6698860C86820F0FF0038433043C860FE
:10467000086840F00100086000202021206484F8D0
:104680003D10206384F83E0001B0F0BDB0B586B0A7
:10469000006845F60001C4F2000100248842CDE91B
:1046A0000444CDE90244019431D045F20041C4F202
:1046B0000001884254D1002443F630050094C4F22E
:1046C0000205286801A940F002002860286800F06F
:1046D0000200009000984FF4407001901220CDE944
:1046E0000204032004900420059040F20040C4F22C
:1046F0000200FFF71FFE0094286940F400102861B3
:10470000286900F400100090009806B0B0BD43F690
:1047100030050094C4F202052868122140F0200000
:104720002860286800F02000009000980320019085
:1047300004900420059040F20040C4F20200CDE94C
:10474000021400F5805001A9FFF7F4FD00942869D8
:1047500040F480002861286900F4800000900098EF
:1047600006B0B0BD40F27C304DF6DC21C2F2000054
:10477000C2F2010100780A68104408607047000026
:1047800080B543F60040C4F20200016841F40071B4
:104790000160016841F480610160016841F4807149
:1047A0000160032000F06CF80F2000F005F800F025
:1047B0002BF8002080BD0000B0B540F27C32C2F280
:1047C000000240F200011278C2F200014FF47A7345
:1047D0000968B3FBF2F20446B1FBF2F1084601F0BE
:1047E0005DF80F2C4FF001050CD858B94FF0FF3091
:1047F00021460022002500F033F840F28030C2F25A
:10480000000004602846B0BD80B582B0002043F6A9
:1048100040010190C4F202014A6842F480424A60B9
:104820004A6802F480420192019A009008680022CE
:1048300040F08050086008680F2100F08050009020
:1048400000986FF0010000F00BF802B080BD00008E
:1048500080B504F08DFD80BD80B504F09DFD80BD68
:1048600070B514460D46064604F0A6FD29462246BC
:1048700002F026FD0146304604F0A6FD70BD0000A2
:1048800080B504F0BBFD80BD2DE9F041002800F0AB
:104890008B8043F60808C4F202080446D8F8F803EF
:1048A0000D4600F00700884207D288F8F853D8F880
:1048B000F80300F00700A84276D12068810717D5D9
:1048C000410705D5D8F8001041F4E051C8F80010B0
:1048D000010705D5D8F8001041F46041C8F8001070
:1048E000D8F80010A26821F0F0011143C8F80010B8
:1048F000C0073FD1D8F8F80300F00700A84207D955
:1049000088F8F853D8F8F80300F00700A8424BD114
:104910002068410707D5D8F80010E26821F4E0517B
:104920001143C8F80010000708D5D8F80000216925
:1049300020F4604040EAC100C8F8000000F07EF8B2
:10494000D8F800104EF25842C1F30311C0F600022D
:10495000515C40F2000220FA01F140F28030C2F2D4
:1049600000000068C2F200021160FFF725FF00207E
:10497000BDE8F0816068811E022907D258F8081C42
:1049800089015CBF0120BDE8F08110E0012807D15A
:1049900058F8081C89035CBF0120BDE8F08106E0DF
:1049A00058F8081C890702D40120BDE8F081D8F826
:1049B000001021F003010843C8F80000FFF794FD40
:1049C000064641F2883700BFD8F80000616800F061
:1049D0000C00B0EB810F8DD0FFF786FD801BB84235
:1049E000F2D90320BDE8F08140F20000C2F20000DD
:1049F0000068704780B5FFF7F7FF43F60801C4F27F
:104A0000020109684EF26842C1F38221C0F6000239
:104A1000515CC84080BD000080B5FFF7E5FF43F65C
:104A20000801C4F2020109684EF26842C1F3423142
:104A3000C0F60002515CC84080BD000010B543F6CE
:104A40000404C4F20204606800F00C0008280AD0D4
:104A5000042819BF42F20040C0F2F40041F60030D1
:104A6000C0F2B70010BD206821682368490241F6F2
:104A70000031C0F2B70100F03F02C3F388105CBF01
:104A800042F20041C0F2F401A1FB00010023FBF758
:104A900021FC21680222C1F3014102EB4101B0FB7C
:104AA000F1F010BD2DE9F04182B0002800F0A280A5
:104AB0000446007843F60006C007C4F2020643D05D
:104AC000B06800F00C00042805D1306880033BD5A5
:104AD0006068C8BB8EE0B06800F00C00082802D106
:104AE00070684002F1D46568B5F5A02F0AD0B5F51D
:104AF000803F0BD0306820F480303060306820F484
:104B0000802006E0306840F480203060306840F457
:104B100080303060FFF7E8FC002D054611D000BF63
:104B20003068800310D4FFF7DFFC401B6428F7D9FE
:104B300022E100BFFFF7D8FC401B64284FF00300C0
:104B400055D830688003F5D4207880071AD5B0682E
:104B500010F00C0F09D0B06800F00C00082840F0ED
:104B60008A807068400200F186803068800702D534
:104B7000E06801283ED13068216920F0F80040EA61
:104B8000C10030602078000738D4207840074CD42A
:104B9000A5695DB3B06800F00C00082840F09E8065
:104BA000012D27D07068E16900F480028A4221D18A
:104BB000216A00F03F028A421CD147F6C071626A46
:104BC0000140B1EB821F15D1A26A0023CFF6FF731B
:104BD00003EBC23200F440316FF30F02914209D16E
:104BE000E16A00F07060B0EB016F03D1002002B009
:104BF000BDE8F081012002B0BDE8F08160690028C5
:104C000040F20000C4F2472057D00121C0F8801EB6
:104C1000FFF76AFC054600BF706F8007B5D4FFF749
:104C200063FC401B0228F7D9A6E0306C10F08058D6
:104C30000AD100200190306C40F080503064306C1C
:104C400000F080500190019847F20007C4F200077D
:104C50003868C00524D4386840F480703860FFF7A5
:104C600043FC05463868C0051AD4FFF73DFC401BDD
:104C70000228F7D980E0E068002851D00020C4F273
:104C8000472001210160FFF72FFC054630688007AF
:104C90003FF571AFFFF728FC401B0228F6D96BE007
:104CA000A568052D50D0012D52D0306F20F00100A5
:104CB0003067306F20F004004DE00021C0F8801E06
:104CC000FFF712FC054600BF706F80077FF55DAFF0
:104CD000FFF70AFC401B0228F6D94DE00027C4F27A
:104CE000472700203866FFF7FFFB022D05460BD152
:104CF0003068800158D5FFF7F7FB401B02284FF0C2
:104D00000300F5D973E700BF306880017FF56EAF0F
:104D1000FFF7EAFB401B02284FF00300F4D966E7D7
:104D20000020C4F2472000210160FFF7DDFB0546AB
:104D3000306880077FF526AFFFF7D6FB401B0228BF
:104D40004FF00300F4D952E7306F40F004003067B1
:104D5000306F40F001003067FFF7C6FB002D0546BD
:104D600041F2883714D000BF306F800713D4FFF7AB
:104D7000BBFB401BB842F7D9032002B0BDE8F0816D
:104D8000FFF7B2FB401BB8424FF003003FF62FAFD6
:104D9000306F8007F4D4B8F1000F7FF4F9AE306CB7
:104DA00020F080503064F3E604F11C052FCD084359
:104DB0000021CFF6FF7140EA821001EBC3316FF39F
:104DC0000F0140EA05600843706001203866FFF774
:104DD0008BFB0446306880013FF508AFFFF784FB8A
:104DE000001B02284FF00300F4D900E780B502F061
:104DF0004FFD022808BF80BD4CF20C01C2F2010138
:104E000001EB40108069002818BF804780BD00007A
:104E100070B538B10446406A30B10020206104F119
:104E2000140007E0012070BD6068B0F5827F03D0F8
:104E300004F11C00002101600026A66294F85100D4
:104E400020B9204684F8506000F03CF8022084F835
:104E5000510094E80F0001F48271056802F40442E5
:104E600025F040050560114403F4006223691144F4
:104E700003F002026369114403F00102A369E569CA
:104E8000114403F40072114405F03802256A1144FC
:104E900005F08002A56A114305F400521143016038
:104EA000626A042101EA134102F0100211444160D8
:104EB000C16921F40061C1610120666584F8510077
:104EC000304670BD2DE9F04F87B0044643F200072D
:104ED0000068C4F201070026B8420696CDE90466D0
:104EE0000396029602D007B0BDE8F08F43F630007B
:104EF0000196C4F20200416902AD41F48051416162
:104F0000416946F2404801F48051019101990196AE
:104F100001684FF0020941F00201016001684FF0A1
:104F2000030A01F0020101910199019601684FF015
:104F3000050B41F0010101600068294600F0010005
:104F4000019001981820029007F55440C4F202081D
:104F5000CDE90396CDF814A0CDF818B0FFF7EAF923
:104F60008020CDE9020904A880E8400C07F55040F4
:104F70002946FFF7DFF94CF6A815C2F201054FF4F8
:104F800040304FF0C0674FF48069C5E908062846F5
:104F9000C5E90087C5E90266C5E90496C5E9066664
:104FA000FFF7F6F8002818BFFDF7E2FFE564AC63F1
:104FB00040F2B45508F11800C2F200054021C5E9DD
:104FC000000705F10800002280E806024FF40030D7
:104FD000C5E908022846C5E90522EA61FFF7D8F8C5
:104FE000002818BFFDF7C4FFA564AC6307B0BDE897
:104FF000F08F00002DE9F04182B0044690F8510096
:10500000012815D10E4600294FF0010060D0174647
:10501000002A5DD060681D46B0F5827F02D1A0688D
:10502000002858D0FFF760FA94F85010012903D1F6
:10503000022002B0BDE8F0818046012084F85000D3
:10504000042084F8510000206065A663A787E787E5
:105050002063A086E086A1682064B1F5004F6064FB
:1050600008D12068016821F040010160016821F445
:105070008041016020680168490603D4016841F05D
:1050800040010160E168E08F91B3002855D06E1CAB
:105090000BE000BFC068A16B21F8020BA163E08F99
:1050A0000138E087E08F002847D020688168C90771
:1050B000F0D1FFF719FA002EF4D0A0EB0800A842B7
:1050C000F0D3012084F85100002084F85000032020
:1050D00002B0BDE8F081042084F85100204631463A
:1050E00032463B46009500F09FF902B0BDE8F081E2
:1050F00018B36E1C0BE000BF007BA16B0870A06BA7
:105100000130A063E08F0138E087E08FA8B120680C
:105110008168C907F0D1FFF7E7F9002EF5D0A0EBC1
:105120000800A842F1D3012084F85100002084F83F
:105130005000032002B0BDE8F081204629464246D7
:1051400002F018FB00281CBF20206065012084F8B5
:105150005100002084F85000606D002818BF012025
:1051600002B0BDE8F081000010B5044690F851008F
:1051700001281CBF022010BD13460A4600294FF02B
:10518000010018BF002B00D110BDA06858B961689C
:10519000B1F5827F07D1042084F8510020461146E2
:1051A00000F03EFA10BD94F85010012904BF02200F
:1051B00010BD012184F85010042184F85110002101
:1051C000B0F5004F6165A263A387E387C4E91011BE
:1051D000A186E18608D12068036823F040030360BC
:1051E000036823F480430360E06C47F21D6E47F2CE
:1051F0004163C0F6000EC0F60003C0E90F3E47F25F
:10520000F953C0F60003D4F800C0C0E91331E38FAE
:105210000CF10C01FFF724F840B1606D40F0100074
:105220006065002084F85000012010BD21680868E6
:10523000400603D4086840F040000860002084F86D
:1052400050004A6842F020024A604A6842F0010277
:105250004A6010BD80B502F01BFB022808BF80BD6C
:105260004CF20C01C2F2010101EB40104068002831
:1052700018BF804780BD000080B502F009FB0228FE
:1052800008BF80BD4CF20C01C2F2010101EB4010DD
:105290000069002818BF804780BD00002DE9F0415B
:1052A00082B01D4616460F460446FFF71DF994F8D6
:1052B000511001290DD18046002F4FF0010018BF79
:1052C000002E02D102B0BDE8F08194F85000012810
:1052D00003D1022002B0BDE8F081012084F8500023
:1052E000032084F85100002060652763A686E686C7
:1052F000A063A087E087A168C4E91000B1F5004F62
:1053000008D12068016821F040010160016841F482
:105310008041016020680168490603D4016841F0BA
:10532000400101606168731EE268B1FA81F1B3FA6D
:1053300083F349095B09B2F5006F41EA030124D107
:1053400039B1216B0988C160B81C2063E08E013837
:10535000E086E08E002846D06E1C09E0216B31F813
:10536000022BC2602163E08E0138E086E08ED0B36C
:10537000206881688907F1D4FFF7B6F8002EF5D0D0
:10538000A0EB0800A842F1D323E039B139780173CA
:10539000206B01302063E08E0138E086E08E10B390
:1053A0006E1C0AE0216B09780173206B01302063C9
:1053B000E08E0138E086E08EA8B120688168890718
:1053C000F0D4FFF791F8002EF5D0A0EB0800A8422A
:1053D000F1D3012084F85100002084F8500003200C
:1053E00002B0BDE8F08120462946424602F00AFAA2
:1053F00000281CBF20206065A06838B900200190FB
:105400002068C1680191806801900198012084F8AA
:105410005100002084F85000606D002818BF012062
:1054200002B0BDE8F08100002DE9F04381B01E46D6
:1054300015460F460446FFF757F894F85110814679
:10544000012909D06068B0F5827F14D104294FF09A
:10545000020007D1A16829B9002F4FF0010018BF41
:10546000002D02D101B0BDE8F083002EFAD094F8EF
:105470005000012803D1022001B0BDE8F0830120D3
:1054800084F8500094F85100002104281CBF052026
:1054900084F851006165A563E687A6872763E686E1
:1054A0002068A686216461640168490603D4016806
:1054B00041F0400101606168731EE268B1FA81F158
:1054C000B3FA83F3DDF8208049095B09B2F5006F78
:1054D00041EA030139D139B1216B0988C160B81C97
:1054E0002063E08E0138E086012608F1010500BF47
:1054F000E08E10B9E08F00286CD0206881688907A1
:105500000CD5E18E012E09D141B1216B002631F875
:10551000022BC2602163E18E0139E1868168C907EF
:105520000AD0E18F41B1C068A16B012621F8020BBE
:10553000A163E08F0138E087FEF7D6FF002DD7D0BA
:10554000A0EB09004045D3D33AE039B13978017373
:10555000206B01302063E08E0138E086012608F1DF
:10556000010500BFE08E08B9E08F98B3206881681C
:1055700089070DD5E18E012E0AD149B1216B002694
:1055800009780173206B01302063E08E0138E086DA
:1055900020688168C9070BD0E18F49B1C068A16B51
:1055A00001260870A06B0130A063E08F0138E0870E
:1055B000FEF79AFF002DD5D0A0EB09004045D1D3CE
:1055C000012084F85100002084F85000032001B02D
:1055D000BDE8F083204641464A4602F013F940B147
:1055E00020206065002084F85000012001B0BDE853
:1055F000F083A06838B9002000902068C16800914D
:10560000806800900098012084F85100002084F800
:105610005000606D002818BF012001B0BDE8F08384
:1056200070B5044690F85100012806D100294FF0CA
:10563000010018BF002A0CD170BD6568B5F5827FE6
:105640000ED104284FF00200F6D1A568002DEDD050
:10565000F2E7002B08BF70BD94F85000012801D17B
:10566000022070BD012084F8500094F851000026FB
:1056700004281CBF052084F8510066652163A386B9
:10568000E386A263A387E387C4E9106694F8510018
:1056900047F21D6147F23563C0F60001C0F6000312
:1056A000042808BF0B4647F2416047F21971C0F663
:1056B0000000C0F6000108BF0146E06C2568C0E9A3
:1056C0000F1347F2F951C0F60001C0E91316E38F3A
:1056D00005F10C01FEF7C4FD38B1606D40F010001B
:1056E0006065012084F8506070BD2268216BA06C59
:1056F000536843F001035360C0E90F66C0E91366C5
:10570000E38E0C32FEF7ACFD40B1606D40F010004E
:105710006065002084F85000012070BD2168086891
:10572000400603D4086840F040000860002084F878
:1057300050004A6842F020024A604A6842F0020281
:105740004A6070BD10B5044690F8510001280AD196
:1057500000294FF0010018BF002A00D110BD94F8B5
:105760005000012801D1022010BD012084F8500012
:105770000320002384F8510063652163A286E2863A
:10578000A363C4E91033A387E387A068B0F5004F93
:1057900008D12068026822F040020260026842F4E8
:1057A00080420260A06C47F2296C47F2A962C0F601
:1057B000000CC0F60002C0E90F2C47F2F952C0F607
:1057C0000002D4F800E0C0E91323E38E0EF10C02CE
:1057D000FEF746FD40B1606D40F0100060650020AE
:1057E00084F85000012010BD21680868400603D4E9
:1057F000086840F040000860002084F850004A68C3
:1058000042F020024A604A6842F002024A6010BD3B
:1058100080B502F03DF8022808BF80BD4CF20C01B3
:105820004001C2F201010858002818BF804780BD1E
:1058300080B502F02DF8022808BF80BD4CF20C01A3
:10584000C2F2010101EB4010C068002818BF804778
:1058500080BD000080B502F01BF8022808BF80BDA3
:105860004CF20C01C2F2010101EB401080680028EB
:1058700018BF804780BD000080B502F009F80228FB
:1058800008BF80BD4CF20C01C2F2010101EB4010D7
:105890004069002818BF804780BD000080B502F035
:1058A00021FE80BD7047000070470000002804BF43
:1058B0000120704710B5044690F83D0028B900203B
:1058C00084F83C00204600F01FF8022084F83D00D8
:1058D0002068211D02F08CFE012084F8460084F827
:1058E0003E0084F83F0084F8400084F8410084F8CA
:1058F000420084F8430084F8440084F8450084F8AA
:105900003D00002010BD000080B582B0006844F268
:105910000041C4F20101884201D002B080BD0020E4
:10592000019043F64400C4F202000168002241F4F1
:10593000003101600068052100F4003001900198F9
:105940001920FEF78DFF1920FEF786FF02B080BDFB
:1059500070470000B0B504460068C168026902EAF9
:105960000105A9071DD4680731D4280747D4E806E4
:105970005CD4E80773D128067BD4680606D5206876
:105980006FF040010161204600F0C0F9A80658BF41
:10599000B0BD20686FF0200101612046FFF784FF51
:1059A000B0BD6FF00201016101212177806980079C
:1059B00003D02046FFF7CCFF05E0204600F092F828
:1059C000204600F00DF9002020776807CDD520682B
:1059D0006FF00401016102212177806910F4407F9A
:1059E00003D02046FFF7B4FF05E0204600F07AF828
:1059F000204600F0F5F8002020772807B7D520686A
:105A00006FF00801016104212177C069800703D08C
:105A10002046FFF79DFF05E0204600F063F8204692
:105A200000F0DEF800202077E806A2D520686FF0AD
:105A30001001016108212177C06910F4407F03D073
:105A40002046FFF785FF05E0204600F04BF8204692
:105A500000F0C6F800202077E8073FF48CAF2068FC
:105A60006FF001010161204600F04EF928067FF534
:105A700084AF20686FF0800101612046FFF712FFBC
:105A800068067FF583AF7AE780B586B044F20041BF
:105A90000068C4F20101002288420592CDE9032288
:105AA0000292019201D006B080BD43F63000009210
:105AB000C4F20200036843F020030360006800F0B2
:105AC000200000900098402001900220CDE90202C1
:105AD0000320059001F5504001A90492FEF72AFC2D
:105AE00006B080BD70470000B0B5044690F83C0099
:105AF000012804BF0220B0BD0D464FEAB2010120CB
:105B0000032984F83C0037D8DFE801F0020A1222AA
:105B10002068294602F014FE206850F8181F0EE095
:105B20002068294602F03EFE206850F8181F16E053
:105B30002068294602F06CFE206850F81C1F41F0D6
:105B400008010160016821F00401016029690FE08A
:105B50002068294602F090FE206850F81C1F41F48E
:105B600000610160016821F4806101602969090216
:105B70000268114301600020002184F83C10B0BD90
:105B8000002804BF0120704710B5044690F83D007E
:105B900028B9002084F83C00204600F01FF80220BD
:105BA00084F83D002068211D02F022FD012084F8C8
:105BB000460084F83E0084F83F0084F8400084F8F2
:105BC000410084F8420084F8430084F8440084F8DB
:105BD000450084F83D00002010BD00007047000023
:105BE0007047000010B5044641B1082909D00429C6
:105BF00014BF04F1410004F13F0004E004F13E0051
:105C000001E004F14000007801281CBF012010BD14
:105C1000022041B1082909D0042914BF84F84100A9
:105C200084F83F0004E084F83E0001E084F840007E
:105C30002068012202F072FD206841F2FF71C4F277
:105C4000000188420FDC40F2FF71C4F2000188427B
:105C500017DCB0F1804F49D040F20041C4F200019E
:105C6000884243D049E040F2FF32C4F20102904240
:105C700014DC41F60003C4F20003984236D000233E
:105C800014E040F60001C4F2000188422ED040F634
:105C90000041C4F20001884228D02EE044F2000303
:105CA000C4F20103984221D040F20043C4F2010340
:105CB000984222D1436C884243F400434364C2DDDE
:105CC000904207DC41F60001C4F2000188420DD089
:105CD000002107E044F20001C4F20101884205D02E
:105CE00040F20041C4F20101884206D1816801F00E
:105CF0000701062904BF002010BD016841F0010121
:105D00000160002010BD00007047000070470000D7
:105D10007047000080B503F0EFF9042808BF80BD8C
:105D200040F2944100EBC000C2F2000101EB8000A0
:105D30000069002818BF804780BD0000B0B582B060
:105D4000036804461868D9685A6900F02F05202DA9
:105D500001F0200505D125B1204603F0E7F902B096
:105D6000B0BD5FEA007C1EBF02F0010E01F490722C
:105D700012EB0E024AD1226B0840C1063DD5012A22
:105D80003BD100200190186801905868019001985B
:105D90005869400642D4A08DE18DE28D002A1CBFD7
:105DA000401A5FEA004101D102B0B0BD216851E85C
:105DB000031F226821F4907142E80313002BF5D1F0
:105DC000216851E8051F226821F0010142E805130E
:105DD000002BF5D1202184F842100021216300BF5F
:105DE000216851E8031F226821F0100142E80313E3
:105DF000002BF5D10221616354E0010654D4400622
:105E0000D2D5204603F06CF902B0B0BDC20718BF6E
:105E100011F480725DD1420761D467E0E06B0168E4
:105E200049688AB2002A44D0A38D9A4241D2E185C2
:105E3000C069B0F5807F30D0206850E8030F21683A
:105E400020F4807041E80302002AF5D1206850E870
:105E5000050F216820F0010041E80502002AF5D174
:105E6000206850E8050F216820F0400041E8050255
:105E7000002AF5D1202084F842000020206300BFD2
:105E8000206850E8030F216820F0100041E8030269
:105E9000002AF5D1E06BFEF763F802206063A08D65
:105EA000E18D401A81B20FE0204603F011FA02B0F2
:105EB000B0BDA18D91427FF477AFC069B0F5807F0E
:105EC0007FF472AF022060632046FFF721FF02B02B
:105ED000B0BD626C42F001026264420706D5BEF1B9
:105EE000000F03D0626C42F002026264820706D5A2
:105EF000BEF1000F03D0626C42F004026264BCF198
:105F0000000F06D55EEA050203D0626C42F008027B
:105F10006264626C002A3FF447AF0840800602D5F5
:105F2000204603F003F920684069616C00F04000EE
:105F300001F00801401827D0204603F0A9F8206896
:105F4000406940061BD500BF206850E8050F216856
:105F500020F0400041E80502002AF5D1E06B70B165
:105F600049F28101C0F600010165FEF739F8002809
:105F70003FF41AAFE06B016D884702B0B0BD204618
:105F8000FFF7C8FE02B0B0BD2046FFF7C3FE0020F9
:105F9000606402B0B0BD0000002804BF012070475B
:105FA00010B5044690F8410028B9002084F840005C
:105FB000204600F021F8242084F841002068C168C0
:105FC00021F40051C160204603F014F920680169F2
:105FD00021F490410161416921F02A014161C168C8
:105FE00041F40051C16000202021606484F8411018
:105FF00084F84210606310BD2DE9F04387B0044679
:10600000216844F20042C4F2000200209142CDE92E
:106010000500CDE9030002904ED044F60000C4F222
:106020000000814274D041F20000C4F201008142BC
:1060300040F0C180002643F630000196C4F2020011
:106040004169002441F0100141614169C4F2020438
:1060500001F01001019101990196016802AD41F032
:106060000201016001684FF0020801F00201019194
:106070000199019601684FF0030941F001010160A7
:106080000068072700F0010001900198802002902D
:1060900004F580602946CDE90386CDF81490069773
:1060A000FEF748F94FF40070CDE90208CDE9046924
:1060B00006972046294626E043F630010190C4F2B7
:1060C00002010A6942F400320A610A6902F40032EC
:1060D0000192019A01900A6842F008020A60096878
:1060E00001F0080101910199602102910221CDE99D
:1060F000031003200590072006900020C4F2020040
:1061000000F5406002A9FEF715F907B0BDE8F0837D
:10611000002643F630000196C4F20200016941F402
:1061200080210161016901F48021019101990196A9
:10613000016841F004010160006802A900F0040058
:10614000019001984FF4406002900220CDE90306CF
:1061500003200590072006900020C4F2020000F5FD
:106160000060FEF7E7F84CF6082546F22800C2F278
:106170000105C4F202004FF000614FF480624FF459
:10618000807385E843002846C5E90362C5E90566D2
:10619000C5E907366E62FDF7FBFF002818BFFCF764
:1061A000E7FE272005210022E563AC63FEF758FBDC
:1061B0002720FEF751FB07B0BDE8F08380B502F061
:1061C0009BFF042808BF80BD40F2944100EBC00053
:1061D000C2F2000101EB8000C068002818BF8047B0
:1061E00080BD000080B502F087FF042808BF80BD95
:1061F00040F2944100EBC000C2F2000101EB8000CC
:106200004068002818BF804780BD0000FEE70000FE
:1062100045F6DF1110EE100AC5F63771B6EE001A1A
:10622000A1EB600020EE011A00EE100A21EE002A18
:1062300022EE002AB7EE083A33EE422A22EE000A96
:1062400021EE001A20EE011A33EE411A20EE010A67
:106250007047000010B52DED088B88B3B0EE408A72
:1062600090ED010A90ED069A90ED021A90ED07AAC2
:1062700029EE000A38EE400A2AEE011A30EE41BA41
:1062800004461BEE100A03F06BF8002808BFB0EEBE
:106290004B8A94ED030A94ED041A94ED052A20EE3E
:1062A000080A29EE011A30EE010A2AEE021A30EE2F
:1062B000010A84ED068A84ED079ABDEC088B10BDB7
:1062C0009FED020ABDEC088B10BD00BF000000006E
:1062D000002808BF704710B5F5EE400A0446C0ED2F
:1062E000000A0020F1EE10FAA061E0612EDD80EEE0
:1062F000200A9FED1E1A81EE000A06F047FE9FED70
:106300001C1AB7EE002A20EE011A31EE023A20EEF6
:10631000000ABFEE005A30EE033A30EE055A32EE74
:10632000411A80EE034A35EE055A30EE010A85EE39
:10633000035A80EE030A34EE041A84ED034A84ED16
:10634000041A84ED054A84ED015A07E04FF07E51AE
:106350009FED050AC4E903106061606084ED020AE4
:10636000BDE81040704700BF00000000DB0F49404F
:10637000F304B53F10B52DED048B10B3B0EE408A99
:1063800090ED030A90ED041A90ED052A30EE010A13
:1063900030EE020A88EE009A044619EE100A02F066
:1063A000CFFF00282046B0EE480A08BFB0EE489A5A
:1063B00084ED069A84ED079AFFF74CFFBDEC048B41
:1063C00010BD9FED020ABDEC048B10BD0000000063
:1063D000B0B5012802D9FF2040B2B0BD4CF2600533
:1063E000C2F20105044655F8200060B98820FBF789
:1063F0008FFD002845F82400EDD08821FAF7C7F872
:1064000055F824000470002040B2B0BD80B584B0BF
:10641000D8B100F029F8014600284FF0FC0015D053
:106420008A888DF80C00009208228DF804204FF025
:10643000FF32CDF80520029208786946FBF700FC90
:10644000002818BF4FF0FF3000E0FE2040B204B03B
:1064500080BD000001288FBF00204CF26001C2F215
:10646000010151F8200070472DE9F04128B305786B
:1064700080462846FFF7EEFFF8B1014690F8840009
:10648000D8B10A1D002309E00126002E08BFBDE88F
:10649000F08191F884600133B3420ED252F8234068
:1064A000002CF1D02678AE42EED16688B8F80270A2
:1064B000BE42E9D100262046E7E70020BDE8F08192
:1064C00010B50C46014600284FF0FE0018BF002C06
:1064D00001D140B210BD0846FFF7C6FF20B12146EA
:1064E00000F0D4F840B210BDFC2040B210BD000056
:1064F000B0B52DED028B00286BD00D46002968D079
:106500000446B5F801009FED340A0004DFED330ABC
:1065100000BA102104F078FA84ED070AE8782979A6
:10652000000140EA1110BBEE0E0AF3EE0E0A0C2138
:1065300004F06AFA84ED080A2879697900F00F00FE
:10654000B0EE408A41EA0020BAEE080AF2EE080AEC
:106550000C2104F059FA84ED090AA87994ED071A80
:1065600002EE100AB5EE401AB8EE422AF1EE10FA29
:1065700084ED0A2A0BDA9FED1A2A00BF31EE021AC7
:10658000B5EE401AF1EE10FAF8DB84ED071A94ED3F
:10659000071A9FED132AB4EE421AF1EE10FA0ADB45
:1065A0009FED103A31EE031AB4EE421AF1EE10FAF2
:1065B000F8DA84ED071AE07958B132EE411AB1EEFB
:1065C000482AB1EE400A84ED071A84ED082A84EDCA
:1065D000090ABDEC028BB0BDDA0F49C1DA0F49419F
:1065E000DB0FC940DB0FC9C070B538B10446007875
:1065F000FFF7EEFE28B1FF2040B270BDFE2040B292
:1066000070BD2078FFF726FF0028F4D090F8842092
:1066100005469AB1281D002105E000BF95F88420A9
:10662000013191420AD250F82120002AF6D0528836
:1066300063889A42F2D1FD2040B270BD1F2ADAD899
:106640003020FBF765FC0028D5D030210646F9F74D
:106650009EFF20686168C6E900010020E27930727F
:106660002078618832760322FBF7A4F918B130460E
:10667000FBF7C6FBBFE795F8840005EB800101300E
:1066800085F88400002040B24E6070BD2DE9F043D3
:1066900081B02DED028B84B0044600284FF0FE003F
:1066A0005ED00D4600295BD095ED020ADFED300A81
:1066B0009FED301A102002F0CFFF95ED010A8046C1
:1066C000FBEE0E0AB3EE0E1A0C2002F0C5FF9FED92
:1066D0002A8A95ED030A9FED291A0646F0EE480A2C
:1066E0000C2002F0B9FF95ED040A8146B1EE041AC0
:1066F000F0EE480A0C2002F0AFFF95ED000A0546C7
:10670000FAEE080AB2EE081A0C2002F0A5FF3209D0
:106710004FEA1923A7888DF8072022784FEA18211D
:1067200043EA0613060A46EA05162D0900970827CC
:106730008DF805108DF80C00694610468DF8047030
:106740008DF806808DF808308DF809908DF80A5084
:106750008DF80B60FBF774FA002818BF4FF0FF307C
:1067600040B204B0BDEC028B01B0BDE8F08300BFC5
:10677000DA0F49C1DA0F4941000000000000FA4376
:10678000F0B587B0A0B3077805463846FFF762FE3C
:10679000A8B390F8841069B3011D002205E000BF82
:1067A00090F8843001329A4224D251F82240002CD1
:1067B000F6D063886E88B342F2D1F4B169886D4631
:1067C00038462A460023FAF7EFFFD0B1FBF75CFC0E
:1067D000D4E90423801A48F2A162C0F2010299416F
:1067E000801A71F1000024BF00202072FF2014E005
:1067F000FE2012E00024002CE0D1FC200DE0FC2063
:106800000BE001202072FBF73FFCC4E9040105F115
:106810000D012046FFF76CFE002040B207B0F0BD2E
:10682000002814BF90ED050AB8EE000A704700007A
:10683000002814BF90ED060AB8EE000A7047000069
:10684000B0B5012802D9FF2040B2B0BD40F2545586
:10685000C2F20005044655F8200060B94820FBF755
:1068600057FB002845F82400EDD04821F9F78FFEAA
:1068700055F824000470002040B2B0BDB0B584B01B
:1068800048B304780546204600F064F828B36988C8
:10689000A1F201210A295BD8012202FA01F10A07BB
:1068A0001DD111F0F00F30D040F2FF1100910821FE
:1068B0008DF804100A3000216A4600BF00EB410346
:1068C0005B7802EB41056B7110F81130013104293E
:1068D000AB71F3D131E0FE2037E0FC2035E04FF41E
:1068E0000071009108218DF80410023000216A46E1
:1068F00000EB41035B7802EB41056B7110F811303E
:1069000001310429AB71F3D117E040F2FF2100916E
:1069100008218DF80410123000216A4600EB410373
:106920005B7802EB41056B7110F8113001310329DE
:10693000AB71F3D10020ADF80B0069462046FBF7A0
:106940007FF9002818BF4FF0FF3040B204B0B0BD4F
:10695000FF20FAE701288FBF002040F25451C2F215
:10696000000151F82000704748B102280BD00128DF
:1069700014BF4FF6FF704FF4804000B2704742F2F0
:10698000107000B2704747F2305000B270470000FC
:10699000022905D2A0F2012189B2072909D805E010
:1069A00007D1A0F2052189B2052902D8013840B2E9
:1069B0007047FF2040B27047F0B581B008B307467A
:1069C0000078FFF7C7FFE0B1014690F84400C0B17E
:1069D00001F11802002306E0012585B191F8445029
:1069E0000133AB420DD252F82340002CF4D065881D
:1069F0007E88B542F0D100252046002DEED101B0B1
:106A0000F0BD002001B0F0BD022884BFB7EE000A3F
:106A1000704740B202A101EB800090ED000A704780
:106A2000000010422CA099410000803F70B538B1A1
:106A300004460078FFF704FF28B1FF2040B270BD84
:106A4000FE2040B270BD2078FFF784FF0028F4D00C
:106A500090F8442005469AB105F11800002104E0A1
:106A600095F84420013191420AD250F82120002AA1
:106A7000F6D0528863889A42F2D1FD2040B270BDB0
:106A80000A2ADAD85020FBF743FA0028D5D0064668
:106A900020686168C6E9000106F118002821F9F7AD
:106AA00076FD62792078618886F828200322FAF73B
:106AB00081FF18B13046FBF7A3F9BEE795F8440013
:106AC00005EB8001013085F84400002040B28E6162
:106AD00070BD000080B59FED020A00F003F880BD94
:106AE0000000000070B52DED048B00283ED0054657
:106AF0000078B0EE408AFFF72DFFC8B3B7EE000A6A
:106B0000B4EE408AF1EE10FAC8BFB0EE408ABFEE94
:106B1000000AB4EE408A0446F1EE10FAB8BFB0EEB7
:106B2000408A6879B1EE489A0028284608BFB0EE3E
:106B3000489AFFF741FFE8B12E7968883146FFF7A0
:106B400027FF002818D405463046FFF70DFF00EE5A
:106B5000100AB8EEC00A29EE000ABDEEC00A10EE17
:106B6000100A04EB45014880002006E0FE2004E006
:106B7000FC2002E0FC2000E0FF2040B2BDEC048BD2
:106B800070BD00002DE9F04F87B0002852D00446B8
:106B90000078FFF7DFFE00284ED0054690F844004D
:106BA00000284BD005F11806E8464FF0010A40F2E4
:106BB000E93B4FF0000908E00121002941D095F898
:106BC000441009F1010989453AD256F82970002F7D
:106BD000F2D07A8861888A42EED12078424600233A
:106BE000FAF7E2FD70B1FBF74FFAD7E90823801AF4
:106BF0009941B0EB0B0071F1000016D300203876FC
:106C0000FC2013E087F818A0FBF73EFAC7E908015B
:106C10003846414600F0A4FA07F108030FCB07F10C
:106C20002C0C8CE80F00002000E0FF200021002940
:106C3000C5D106E0FE2004E0FC2002E0FC2000E0DC
:106C4000FC2040B207B0BDE8F08F00002DE9F04114
:106C500000254FF0000804E0B8F1000F08F101082A
:106C60001ED15FFA88F0FFF775FE0028F4D00446C5
:106C700090F844000028EFD004F11807002604E043
:106C800094F8440001368642E6D257F826000028E0
:106C9000F6D0FFF777FF002818BF4FF0FF35EFE77A
:106CA00068B2BDE8F081000010B54CF6801046F2E5
:106CB0000041C2F20100C4F20001032200234FF0A0
:106CC000807480E80E0000F10C014FF4102C4FF49A
:106CD000001E81E8085084618383FCF71BFF0028B5
:106CE00018BFFCF745F910BD10B540F28C5046F6C0
:106CF0000001C2F20000C4F20001032200234FF0A1
:106D0000807480E80E0000F10C014FF4102C4FF459
:106D1000001E81E8085084618383FCF7FBFE002895
:106D200018BFFCF725F910BD80B582B0002043F6EE
:106D300030010190C4F202010A6842F400120A60B4
:106D40000A6802F400120192019A00900868002279
:106D500040F4800008600868052100F4800000907D
:106D600000980C20FDF77CFD0C20FDF775FD3A2006
:106D700005210022FDF774FD3A20FDF76DFD3B2053
:106D800005210022FDF76CFD3B20FDF765FD02B0FB
:106D900080BD000080B548F2D9404EF2D852C0F60E
:106DA0000000C0F60002002102F0BEFF4CF260615C
:106DB000C2F20101086048F6C9004EF23852C0F62E
:106DC0000000C0F60002002102F0AEFF80BD00000E
:106DD0002DE9F04786B0002043F630010590CDE95B
:106DE0000300CDE901000090C4F202010A6800240A
:106DF00042F002020A600A68C4F2020402F00202CF
:106E00000092009A00900A6804F5C05742F001020F
:106E10000A600A68402602F001020092009A00907F
:106E20000A6842F008020A600A6802F0080200924A
:106E3000009A00900A6842F004020A600A6802F0B0
:106E400004020092009A00900A6842F020020A6050
:106E50000A6802F020020092009A00900A6842F04C
:106E600080020A600A6802F080020092009A009094
:106E70000868002240F0400008600868402100F0E7
:106E80004000009000983846FDF728FB204610216E
:106E900001224FF010090125FDF720FB04F5806861
:106EA000404601210122FDF719FBCDE9016501AE44
:106EB00038463146CDE90355FDF73CFA08200190EC
:106EC0004FF4041A38463146CDE902A5FDF732FAEF
:106ED00020463146CDE9015A0395FDF72BFA2046AD
:106EE0003146CDE90195CDE90355FDF723FA302070
:106EF000CDE9010A04F5006031460395FDF71AFA61
:106F000040463146CDE90155CDE90355FDF712FA6A
:106F1000062005210022FDF7A3FC0620FDF79CFCBE
:106F2000092005210022FDF79BFC0920FDF794FCB8
:106F30000A2005210022FDF793FC0A20FDF78CFCB6
:106F4000172005210022FDF78BFC1720FDF784FC9C
:106F500006B0BDE8F087000080B540F2146045F24D
:106F60000041C2F20000C4F2000148F2A062002316
:106F70004FF4804CC0F2010280E80E00C0E9033CEF
:106F8000C0E90533C0E90733FDF7B4FA002818BF9C
:106F9000FBF7EEFF80BD000080B54CF6682045F69B
:106FA0000001C2F20100C4F2000148F2A062002315
:106FB0004FF4804CC0F2010280E80E00C0E9033CAF
:106FC000C0E90533C0E90733FDF794FA002818BF7C
:106FD000FBF7CEFF80BD0000B0B54CF6BC2043F2FD
:106FE0000001C2F20100C4F201014FF482720023D9
:106FF00080E80E0000F10C014FF0020C4FF0010E82
:107000004FF40074182581E808500A21C0E90645AC
:10701000C0E90833C0E90A31FDF7FAFE002818BFBD
:10702000FBF7A6FFB0BD000080B588B04CF6143069
:1070300044F200420021C2F20100C4F2010241F216
:1070400088330791CDE90511CDE90311CDE901118F
:10705000C0E90021C0E9021301618161FEF726FC4D
:10706000002818BFFBF784FF4CF61430C2F2010071
:10707000FEF786FD002818BFFBF77AFF602001901D
:107080000020CDE9020005904CF61430C2F2010058
:1070900001A90022FEF728FD002818BFFBF768FFB2
:1070A0004CF61430C2F20100FEF7EEFC08B080BDD1
:1070B00080B540F2686041F20001C2F20000C4F203
:1070C000010100234FF00C0C4FF4E13280E80E0078
:1070D000C0E90333C0E905C3C361FEF75DFF0028C3
:1070E00018BFFBF745FF80BD80B54CF65C3044F21D
:1070F0000041C2F20100C4F2000100234FF00C0C69
:107100004FF4E13280E80E00C0E90333C0E905C363
:10711000C361FEF741FF002818BFFBF729FF80BDC0
:1071200080B540F2B06044F60001C2F20000C4F243
:10713000000148F2A06200234FF0040CC0F20102EB
:1071400080E80E00C0E90333C0E905C3C361FEF760
:1071500023FF002818BFFBF70BFF80BDFEE70000F0
:107160002DE9F0478846B1F80D10044608BA4FEAF9
:107170001049B8F811002679B8F80F1005BA304652
:1071800091FAB1FAFFF7F0FB07463046FFF73CFCF7
:1071900001EE109A9FED453AB8EE412A9FED441A50
:1071A00022EE032A22EE014A02EE10AA15FB27F076
:1071B000B8EEC23A02EE100AA0799FED3E5AB8EE40
:1071C000C22A22EE052A48B1B4F84000A9EB00001B
:1071D000B0F5805F0CDD4FF0FF300DE00020A4F82B
:1071E0004090C4E9110084ED024A84ED033A1CE0AA
:1071F00010F5805F03DA0120616C0844606494ED4F
:10720000115A83EE003AB8EEC55A25EE015A34EE13
:10721000054A84EE004AA4F8409020EE022A84ED4C
:10722000033A84ED124A84ED024A94ED020A84ED99
:10723000042AB5EE400AF1EE10FA08DA30EE010A3F
:10724000B5EE400AF1EE10FAF8DB84ED020A94ED97
:10725000020AB4EE410AF1EE10FA0ADB9FED162A9B
:1072600030EE020AB4EE410AF1EE10FAF8DA84EDDB
:10727000020A94F8280078B131EE400A84ED020A3F
:1072800094ED030A94ED041AB1EE400A84ED030A6A
:10729000B1EE410A84ED040A98F8130000EE100ADA
:1072A000B8EE400A84ED050ABDE8F0870000003919
:1072B000DB0FC94000008038DB0FC9C0FEE70000CB
:1072C00000F0070080F00703042B28BF04234FF0D1
:1072D000FF3C03380CFA03F338BF00209943814088
:1072E0000CFA00F022EA000008437047B0B52DED1B
:1072F0000A8B044610EE100AB0EE618AB0EE419A95
:10730000B0EE60AAB0EE40BA02F022F8002800F019
:107310009C801AEE100A02F01BF8002800F09580FD
:1073200019EE100A02F014F8002800F08E8018EE12
:10733000100A02F00DF8002800F087806068B0EEB7
:107340004B0A90ED071AF0EE4A0AFBF7F5FC60686D
:10735000B0EE40BA90ED001A04F11C0020EE01CA14
:1073600021EE0A0AFEF776FF207888B1012811D1B4
:1073700094ED051A94ED022A30EE411AB4EE428AD9
:10738000F1EE10FAC8BFB0EE482A81EE029A01E091
:107390009FED309A19EE100A84ED04BA84ED050AC7
:1073A00001F0D6FF65689FED2B0A002808BFB0EEFC
:1073B000409A95ED010A95ED032A2CEE000A29EE7C
:1073C000022A95ED021A30EE42AA94ED030A9FEDCF
:1073D000229A2CEE082A32EE008AB4EE491AF1EE17
:1073E00010FA28EE01BA1ADD18EE100A01F0B0FF0B
:1073F000A8B13AEE0B0A95ED051AB0EEC00AB4EE4C
:10740000410AF1EE10FA0ADC95ED040AB0EEC81A52
:10741000B4EE401AF1EE10FAD8BF84ED038A3AEECA
:107420000B8A18EE100A01F093FF70B1D5ED050A32
:10743000F4EE490AF1EE10FA05DDB0EE480AF9F76C
:10744000FFFEB0EE408A84ED068A94ED060ABDEC9C
:107450000A8BB0BD00000000BD37863570B52DED3C
:10746000048B90B3044650681646B0EE408A0D4631
:1074700001F06EFF58B3B06801F06AFF48B3F068DE
:1074800001F066FF38B3306901F062FF28B370691C
:1074900001F05EFF18B3B7EE000A80EE089A66604E
:1074A00019EE100A01F054FFD8B1D6ED060A04F126
:1074B0001C00B0EE480A84ED029AFEF709FF204650
:1074C000257000F013F800200CE0FF200AE0FF20F8
:1074D00008E0FF2006E0FF2004E0FF2002E0FF209C
:1074E00000E0FF2040B2BDEC048B70BD10B568B168
:1074F00000F11C0100249FED070AC0E90344C0E924
:1075000005440846FEF736FF60B210BDFF2460B2A6
:1075100010BD00BF0000000000280EBFFF210021A9
:10752000C16048B270470000000000000000000089
:10753000EFF30980BFF36F8F154B1A681EF0100F21
:1075400008BF20ED108A20E9F04F10602DE90900F6
:107550004FF0500080F31188BFF34F8FBFF36F8F50
:1075600003F0C0FD4FF0000080F31188BDE8090072
:1075700019680868B0E8F04F1EF0100F08BFB0ECB3
:10758000108A80F30988BFF36F8F704700BF00BF78
:107590008CCC012040F2B062C2F200021268536942
:1075A00043F04003536146F22802C4F2020213681A
:1075B00043F0100313604CF60822C2F20102126875
:1075C000136823F0010313601368DB0707D000BFC3
:1075D000136823F0010313601368DB07F8D144F646
:1075E0000403C4F200039360D0605160106840F05F
:1075F000010010607047000080B5806B01684A6828
:1076000022F003024A60416D41F010014165012101
:1076100080F85110FDF7EAFB80BD000080B5806B5B
:10762000FDF72AFE80BD000080B5806BFEF700F9F3
:1076300080BD000080B5806BFEF71EF980BD0000A4
:10764000B0B5846B0546FCF74FFF29680968C9058A
:1076500026D402462068A168436823F020034360D3
:1076600031B96168B1F5827F02D16FF0030101E0A9
:107670006FF001014368194041602046642100F029
:1076800079F800281CBF202060650020E0870120D9
:1076900084F85100606D18B12046FDF7A7FBB0BD1E
:1076A0002046FDF7D7FDB0BDB0B582B0846B05466E
:1076B000FCF71AFF29680968C90528D40246206822
:1076C000416821F020014160416821F002014160E0
:1076D0002046642100F096F818B1606D40F020005B
:1076E0006065A06838B9002001902068C1680191E8
:1076F0008068019001980020E086012084F8510004
:10770000606D20B12046FDF771FB02B0B0BD204690
:10771000FEF77EF802B0B0BDB0B5846B0546FCF74D
:10772000E3FE29680968C9051FD40246206841683C
:1077300021F0200141602046642100F063F818B177
:10774000606D40F0200060652068416821F0030111
:1077500041600020E086E087012084F85100606DE0
:1077600018B12046FDF742FBB0BD2046FEF772F887
:10777000B0BD0000B0B582B0044640680B46B0F51D
:10778000827F20D1A168B1F5004F02D0B1F5806FA2
:1077900004D121680D6825F040050D60B0F5827FA9
:1077A00011D1A068B0F5806F1DD100922046012153
:1077B0000022002500F076F890B1606D032540F0BE
:1077C000200060650CE00092204601210022002587
:1077D00000F068F820B1606D032540F0200060657E
:1077E000284602B0B0BD009220468021002200252C
:1077F00000F058F80028F3D0606D032540F0200019
:107800006065EDE770B582B00D4616460221012293
:107810002B460446009600F045F838B1606D03250C
:1078200040F020006065284602B070BD40F20000C4
:10783000C2F20000006849F68171C1F25E61A0FBEE
:107840000101480D4FF47A71484301906068B0F52A
:10785000827F0FD12046802100222B4600960025F2
:1078600000F020F80028DED0606D032540F02000F5
:107870006065D8E7019840B101980138019020680F
:1078800080680006F6D40025CDE70025CBE7000090
:10789000006843F20001C4F20101401A18BF012040
:1078A000400070472DE9F04782B00A9C9846154683
:1078B0000E468146FCF718FE201A00EB0804FCF780
:1078C00013FE40F20001C2F200010968C1F3CB319E
:1078D00061430191D9F8001089683140891BB1FAE0
:1078E00081F14909A94203D1002002B0BDE8F08727
:1078F000824608F101070CE0019801380190D9F89F
:10790000000080683040801BB0FA80F04009A84237
:10791000EAD0002FF3D0FCF7E7FDA0EB0A00A0426D
:1079200004D201980028E7D10024E8E7D9E9000152
:107930004268B1F5827F22F0E00242600BD1D9F8B3
:107940000810B1F5004F02D0B1F5806F03D1016886
:1079500021F040010160D9F82810B1F5005F07D18E
:10796000016821F400510160016841F40051016097
:10797000012089F85100002089F85000032002B04E
:10798000BDE8F087000000000000000000000000DB
:10799000074B19680868B0E8F04F80F30988BFF317
:1079A0006F8F4FF0000080F31188704700BF00BF59
:1079B0008CCC012080B501F019FD80BD90ED000A4E
:1079C00091ED001AB7EE002A30EE011AB4EE421A19
:1079D000F1EE10FAD8BF704782EE011A20EE010ACC
:1079E00080ED000A91ED000A21EE000A81ED000A07
:1079F00070470000B0B52DED048B10B30446B0F80D
:107A0000A00000B394ED011A94ED272A9FED278A78
:107A1000D4ED1E0A94ED310A31EE429AB0EE481AC6
:107A20000D46FBF789F96169B7EE001A91ED042A5A
:107A300081EE022AB4EE429AF1EE10FA05DA002045
:107A40002FE0FF202DE0FF202BE0B4EE410AF1EE05
:107A500010FA4FF0000024DCEA7812B3606804F1F9
:107A6000C405C4F89C0091ED030A2846B8EE400A0C
:107A700088EE000AF0EE480AFBF740F9606990F8DA
:107A80003400012807D195ED000A9FED091A30EE68
:107A9000010A85ED000AB4F8A0000138A4F8A0009E
:107AA000002040B2BDEC048BB0BD00BFDB0FC9406D
:107AB000EBAB2B3C68B141690978012900D029B9A9
:107AC0004DF66E31C3F63671C0F8C010002040B2DA
:107AD0007047FF2040B27047B0B52DED028B0546D0
:107AE00000284FF0FF0026D00C4621B3FAF7CCFA5D
:107AF00006F0C7FB9FED128A00EE100A80EE080A1E
:107B000085ED010AFAF7C0FAD5E90223801A9941F6
:107B100006F0B7FB00EE100A80EE080A85ED040AB5
:107B2000FAF7B2FA2278C5E90201284621462A70FE
:107B300000F034F9002040B2BDEC028BB0BD00BFB4
:107B4000002474492DE9F04F81B02DED028B0446DD
:107B500000284FF0FF0000F096800D46002900F04D
:107B60009280B5EE400AB0EE408AF1EE10FA40F392
:107B70008A802F796561BE003046FAF7C9F9C4F8EA
:107B8000A4003046FAF7C4F9C4F8A8003046FAF762
:107B9000BFF9C4F8AC003046FAF7BAF9C4F8B0003F
:107BA0003801FAF7B5F920623046FAF7B1F9E06723
:107BB0003046FAF7ADF9C4F88400C7EB0710860029
:107BC0003046FAF7A5F9C4F8C8003046FAF7A0F92C
:107BD0007E01C4F8CC003046FAF79AF9C4F848019F
:107BE0003046FAF795F9216AC4F84C01E1B1E16F2A
:107BF000D1B1D4F88410B9B1D4F8A410A1B1D4F89B
:107C0000A81089B1D4F8AC1071B1D4F8B01059B142
:107C10006169C96A41B1D4F8C81029B1D4F8CC104F
:107C2000002918BF002834D1206AFAF7E9F8E06F7C
:107C3000FAF7E6F8D4F88400FAF7E2F8D4F8A400EA
:107C4000FAF7DEF8D4F8A800FAF7DAF8D4F8AC00BE
:107C5000FAF7D6F8D4F8B000FAF7D2F86069C06A3B
:107C6000FAF7CEF8D4F8C800FAF7CAF8D4F8CC007E
:107C7000FAF7C6F8D4F84801FAF7C2F8D4F84C017C
:107C8000FAF7BEF8FB2040B2BDEC028B01B0BDE8B4
:107C9000F08FD4F848010028C6D0F9F7C5FDDFB34E
:107CA00007EB870005F1380805F158094FEA400A4B
:107CB0004FF0000B00270026E86A3044FEF7B6FEBE
:107CC000D4F8C80001215844B0EE480A4246FFF7F4
:107CD000C5FBD4F8CC0001215844B0EE480A4A460E
:107CE000FFF7BCFB6069D4F84811D0ED3E0AC81913
:107CF000B0EE480AFEF7ECFA6069D4F84C11D0ED0A
:107D00003F0AC819B0EE480AFEF7E2FA0A362037F1
:107D1000B2450BF13C0BCFD105F13000FEF786FEEA
:107D2000606990F8340078B1012835D104F1D000B1
:107D300005F1B8020121B0EE480AFFF78FFB04F508
:107D4000867005F1D8020CE004F1D00005F178024C
:107D50000121B0EE480AFFF781FB04F5867005F1BA
:107D600098020121B0EE480AFFF778FB6069B0EE97
:107D7000480AD0ED400A04F5A870FEF7A9FA606938
:107D8000B0EE480AD0ED410A04F5B870FEF7A0FA4B
:107D90000020C4E9270076E7FC2074E7B0B500B303
:107DA0000446406990F82020F2B194F89820032A04
:107DB00067D8DFE802F00259233A94ED0E0A9FEDEE
:107DC000421A80EE010A90ED091AB4EE410AF1EE72
:107DD00010FA68DD6268012084F89800C4F89420E5
:107DE00061E0FF2568B2B0BD0025204684F89850B8
:107DF00084F8905000F00EF968B2B0BD90ED030A1F
:107E00009FED2F1AB8EE400A81EE000A94ED1E1A7B
:107E100000206268A4F8A000032084F89800C4F849
:107E2000942031EE000A84ED310A204600F0F2F889
:107E300094ED010A94ED251A9FED222A30EE410AB5
:107E4000B4EE420AF1EE10FA30DB94ED0E0A9FED2B
:107E50001E1A002580EE010AB3EE041AB4EE410AA0
:107E6000F1EE10FAC8DA0DE094ED0E0A9FED161A45
:107E700080EE010A90ED091AB4EE410AF1EE10FA13
:107E800004DA002568B284F89850B0BD94ED010A78
:107E900094ED251A90ED0A2A30EE410AB4EE420A1A
:107EA000F1EE10FA05DA204600F0B4F8002568B2C9
:107EB000B0BD012084F89000022084F89800F5E716
:107EC000DB0FC9C09A99993E00007A4400284AD035
:107ED000F0B581B02DED028B04464069007920B3E6
:107EE000C0EB00109FED218A85000026002700BF0F
:107EF000D4F8C8003844FFF7F9FAD4F8CC00384475
:107F0000FFF7F4FAD4F84801B0EE480A3044FEF71F
:107F100031FAD4F84C01B0EE480A3044FEF72AFAA0
:107F20003C37BD4206F12006E2D104F1D000FFF754
:107F3000DDFA04F58670FFF7D9FA9FED0C8A04F597
:107F4000A870B0EE480AFEF715FA04F5B870B0EE66
:107F5000480AFEF70FFA0020BDEC028B01B0BDE825
:107F6000F04040B27047FF2040B270470000000070
:107F700010B370B504464069007980B1C0EB0010C1
:107F800085000026D4F8C8003044FFF7C5FAD4F8BD
:107F9000CC003044FFF7C0FA3C36B542F2D104F1D0
:107FA000D000FFF7B9FA04F58670FFF7B5FA0020A4
:107FB000BDE8704040B27047FF2040B270470000FB
:107FC00020B310B5416991F804C0BCF1000F14D082
:107FD000D0E92921D0E92B430439A3F1040E231F52
:107FE000043A002442F8044F41F8044F43F8044F88
:107FF000BCF1010C4EF8044FF4D10021C0E92D1161
:10800000C0F8BC10BDE8104048B27047FF2148B22C
:10801000704700002DE9F04F81B02DED048B05462F
:1080200000284FF0FF0000F02C828946002900F064
:10803000288268692978047940F2157B0029C2F208
:10804000000B00F08A80287E022800F0988001282A
:1080500000F03E81002840F0FD81002C43D004EB6D
:1080600084009FED9A8A4FEA40086FF003060027CC
:108070004FF0000A002400BFD5F8C8003844FFF7CD
:108080004BFAD5F88400D5F8C8103044D0ED010A79
:10809000D5ED041AC819B0EE480AB0EE481AFFF739
:1080A00025F9D5F8A400D5F8AC10D5F84C2130440A
:1080B00080ED010A881980ED010A02EB0A00FEF743
:1080C000C9F86969D5F8B000C96A304480ED010A81
:1080D0000819FEF707FD0A3404360AF1200AA04504
:1080E00007F13C07C8D14CF22C00C2F201009FED11
:1080F000778A90ED000AD5ED041AD5ED1E0A05F138
:10810000D000B0EE481AFFF7F1F8D5ED041AD5ED1E
:10811000230A05F58670B0EE481A85ED2D0AFFF7A3
:10812000E5F805F5B87085ED2E0AFEF793F8686955
:1081300085ED2F0A3030FEF7D5FC99F802000028B3
:1081400000F08A812846FFF7C1FE2846FFF710FF9E
:108150002846FFF735FF01207DE15CB104EB840088
:10816000440000266869C06A3044FEF7B3FC0A3652
:10817000B442F7D168693030FEF7ACFC6CE12846B8
:108180004946FFF737FC002C6CD004EB84009FEDD0
:10819000CB8A4FEA40086FF0030600274FF0000A31
:1081A000002400BF686995ED301AC16AC069097A78
:1081B000D5ED041A0139C9B200EB810090ED000A37
:1081C000D5F88400D5F8C8103044D0ED010A20EE6F
:1081D000010AC819B0EE481AFFF788F8D5F8A410BC
:1081E000D5F884003144D5F8CC2081ED010A304423
:1081F000D5ED041A95ED220AD0ED010AD019B0EEA2
:10820000481AFFF773F8D5E929203044011D80EDA5
:10821000010A90190430FFF7D1FB05F1A40207CA47
:10822000304490ED010A881990ED011AD5F84C01FF
:1082300030EE010A9119504481ED010AFEF70AF867
:108240006969D5F8B000C96A304480ED010A08199F
:10825000FEF748FC0A3404360AF1200AA04507F16B
:108260003C079FD19FED958AD5ED041AD5ED1E0AE6
:1082700095ED310A05F1D000B0EE481AFFF736F857
:10828000D5ED041AD5ED230A05F58670B0EE481A2F
:1082900085ED2D0AFFF72AF805F5B87085ED2E0A51
:1082A000FDF7D8FF686985ED2F0A3030FEF71AFC1C
:1082B00099F80300002840F0CF8001202876A86FAD
:1082C0004CF22C01C2F201010860C5E00000000080
:1082D0002846FFF7EFFB002C77D004EB84009FEDDE
:1082E000789A40F2005A9FED758A4FEA400B6FF082
:1082F00003060024C2F2000A00274FF0000800BF66
:1083000095ED300A686980EE091AC16AC069097A78
:10831000D5ED041A0139C9B200EB810090ED002AB5
:10832000D5F88400D5F8C810304422EE000A8AED52
:10833000001AD0ED010A0819B0EE481AFEF7D6FF70
:10834000D5F8A410D5F884003144D5F8CC2081EDBF
:10835000010A3044D5ED041A95ED220AD0ED010A48
:108360001019B0EE481AFEF7C1FFD5E929203044B4
:10837000011D80ED010A90190430FFF71FFB05F184
:10838000A40207CA304490ED010A881990ED011A41
:10839000D5F84C0130EE010A9119384481ED010AFB
:1083A000FDF758FF6969D5F8B000C96A304480ED1F
:1083B000010A01EB0800FEF795FB08F10A080436F4
:1083C0002037C34504F13C049AD14CF22C00C2F290
:1083D00001009FED3A8A90ED000AD5ED041AD5ED23
:1083E0001E0A05F1D000B0EE481AFEF77FFFD5ED6A
:1083F000041AD5ED230A05F58670B0EE481A85ED0E
:108400002D0AFEF773FF05F5B87085ED2E0AFDF70E
:1084100021FF686985ED2F0A3030FEF763FB99F87C
:108420000200A0B340F2157BC2F2000B9BF80000E3
:1084300090B999F8030078B1687E02210328297663
:1084400032D0022835D0012814BF00200120A5F821
:10845000A00001E0002028766869C06AFEF70EFAE5
:1084600068694168052903D3C06A2830FEF706FA17
:1084700068693030FEF702FA99F803008BF80000C3
:10848000002040B2BDEC048B01B0BDE8F08F28465F
:10849000FFF71CFD2846FFF793FD002040F2157BF7
:1084A0002876C2F2000BD7E741F60A20A5F8A00013
:1084B000D2E768694069A5F8A000CDE70000000098
:1084C00000C0DA4500280FBFFF2141760021A0F847
:1084D000A01048B27047000080B501F021FC01F007
:1084E0007DFC80BDB0B501380024B4EB106F1CBF1B
:1084F0000120B0BD4EF21005CEF2000568604FF0CD
:10850000FF300F2100F060FF0720AC60286020469C
:10851000B0BD000080B5FCF725F903F009FD012886
:1085200018BF02F0DBFE80BD70B592B006AC2046ED
:108530003021F8F72CF8002543F640000595CDE9E9
:108540000355CDE901550095C4F2020001680226E9
:1085500041F080510160006800F080500090009868
:1085600047F200000095C4F20000016841F4804128
:108570000160006800F4804000900098012006909F
:108580004FF4803007904FF480000D9006200E903D
:10859000A820CDE90F060420119020460C96FCF788
:1085A00081FA88B90F20CDE901064FF4A05004905C
:1085B0004FF48050059001A805210395FCF764F95C
:1085C000002804BF12B070BDFAF7D2FC4EF68850F6
:1085D000CEF20000016841F47001016070470000B4
:1085E00080B54CF61430C2F20100FDF7B3F980BD3E
:1085F000B0B540F6FF3E0568C4F2000E40F2004CF4
:108600007045C4F2010C0FDCB0F1804F19D040F27C
:108610000043C4F20003984213D040F60003C4F2B2
:10862000000398420DD011E040F60043C4F200036D
:10863000984206D0604504D00023C4F2010398425A
:1086400004D14B6825F0700243EA020541F6FF733E
:10865000C4F2000398420DDC70451FDCB0F1804F7E
:1086600041D040F20043C4F2000398423BD040F6B0
:10867000000321E043F6FF73C4F20103984220DCBB
:1086800042F20003C4F2000398422CD00023C4F24B
:108690000103984227D0604525D029E040F60043E9
:1086A000C4F2000398421ED041F60003C4F2000356
:1086B000984218D041F60043C4F20003984212D009
:1086C00016E044F20003C4F2010398420BD044F6D2
:1086D0000003C4F20103984205D044F20043C4F2FF
:1086E0000103984204D1CB6825F4407243EA0205A5
:1086F0000A688C684B69C46240F480648262644595
:1087000004BF09690163026825F0800142F0040298
:1087100019430260012242610160B0BD80B501F0E1
:108720001F014FF0010CD0F820E00CFA01F32EEA03
:1087300003030362036A02FA01F11943016280BD77
:10874000B0B5026A036A40F2004523F001030362F8
:10875000D0F804E0D0F818C08C6822F0020240F48F
:108760008063C4F20105AB4242EA040205D1CC6841
:1087700022F00C0224F0040422430C68AB4207D11F
:10878000D1E905532EF4407E45EA0E0545EA030E75
:108790002CF073032343C0F804E08361496841630C
:1087A0000262B0BD70B5026A036A40F2004423F071
:1087B00010030362D0F804E0D0F818C08D6822F0EE
:1087C000200240F48063C4F20104A34242EA05128D
:1087D00007D1CD686FF0400622F0C00206EA051509
:1087E0002A430D68A34207D1D1E905642EF4406302
:1087F00043EA860343EA840E2CF4E64343EA052366
:10880000C0F804E0836149688163026270BD0000C2
:1088100070B5026A036A40F2004423F48073036275
:10882000D0F804E0D0F81CC08D6822F4007240F447
:108830008063C4F20104A34242EA052207D1CD6855
:1088400040F2FF462D0222F44062B5432A430D68F0
:10885000A34207D1D1E905642EF4405343EA06133D
:1088600043EA041E2CF073032B43C0F804E0C361F9
:108870004968C163026270BD70B5D0F820C0026A59
:1088800040F2004622F4805202624268C3690C68DA
:10889000D1F808E040F48065C4F20106B54204D185
:1088A0004D6922F4804242EA851223F4E64343EA0A
:1088B00004234260C3612CF40056496846EA0E3234
:1088C0000164026270BD000010B500F0B5FF48F60B
:1088D000F1104EF2A842C0F60000C0F600020021DE
:1088E00001F022FA4DF25414C2F20104206048F65D
:1088F00061404EF21452C0F60000C0F600020021A2
:1089000001F012FA606048F699304EF2F042C0F67B
:108910000000C0F60002002101F006FAA06048F64F
:10892000D1504EF28052C0F60000C0F60002002185
:1089300001F0FAF9E06048F689604EF2A452C0F600
:108940000000C0F60002002101F0EEF9206148F6B7
:1089500031204EF2CC42C0F60000C0F600020021E9
:1089600001F0E2F9606148F611504EF25C52C0F637
:108970000000C0F60002002101F0D6F9A06102203B
:108980000A21002200F0EEFFE061022018210022FF
:1089900000F0E8FFA06202200C21002200F0E2FFBC
:1089A000E06202201821002200F0DCFF2063022098
:1089B0002821002200F0D6FF206202201821002288
:1089C00000F0D0FFA06302204FF4BC61002200F051
:1089D000C9FF606302200821002200F0C3FF606429
:1089E00000F05AFF01F09CF901F0F8F910BD000009
:1089F00000F00AFF04F0F8FF9FED0B0B53EC102B77
:108A000004F018FE04F0ACFF0446002000F0B4FEB1
:108A100000F0F0FE051900BF284600F0BDFE254419
:108A2000FAE700BF00BF00BF0000000000407F4029
:108A300082B000F0E9FE04F0D7FF9FED530B53EC3A
:108A4000102B04F0F7FD04F08BFF0646002000F029
:108A500093FE00F0CFFE40F20855C2F200054CF242
:108A600054010446C2F201012846F8F73FFC2846AB
:108A7000F8F716FC40F26C5040F21871C2F2000098
:108A8000C2F20001F7F7D4FE2846F8F709FCB7EE6A
:108A9000001A81EE000A4CF6A4304EF2FC52C2F2EB
:108AA0000100C0F600020021FEF7D8FC0020F9F713
:108AB00061FA4CF264689FED368A9FED369A4CF667
:108AC00068194DF2541AA71905F1100005F11C0B95
:108AD000C2F20108C2F20109C2F2010A0196009035
:108AE000F8F752FDF8F7C8FBF8F7D2FBF8F7E8FB08
:108AF000F8F7F4FB00F0A0FE2846F8F799FC2846AA
:108B0000F8F7E0FC40F26C54C2F20004009940F225
:108B1000187320465A46C2F20003F7F751FF404649
:108B20002146F7F717FE00F0B7FED5ED0A0A4CF61E
:108B3000A430C2F20100B0EE480AB0EE491AF0EEDD
:108B4000491AFEF7D3FB0020F9F7E6F998E8070089
:108B500005F11C0658CEC9E90301DAF8280089E8B6
:108B60005800C9F8142000F095FFDAF828004946AB
:108B70000022002300F046FF384600F00DFE019869
:108B80000744ADE700BF00BF0000000000407F4089
:108B9000000020420000000086B000F035FE04F026
:108BA00023FF9FED2B0B53EC102B04F043FD04F03F
:108BB000D7FE81460020002400F0DEFD00F01AFE02
:108BC0000646FAF7EBF84CF28005C2F201059FED7C
:108BD000220A00F52271284600F020FC4DF25417BD
:108BE00040F23C5A4E44C2F20107C2F2000AE84683
:108BF0001AE000BF28464146CDE90444CDE90244CD
:108C0000CDE90044F9F7CAFA2846F9F7B7FB786BC3
:108C100000F040FF786B29460022002300F0F2FEAE
:108C2000304600F0B9FD4E44B86B51460022002397
:108C300000F054FEB86B51460022002300F04EFEB7
:108C40000028D7D12846F9F7D3FF28465146D9E75F
:108C50000000000000407F400000FA4300000000D8
:108C600000F0D2FD04F0C0FE9FED250B53EC102B5D
:108C700004F0E0FC04F074FE8146002000F07CFD6E
:108C800000F0B8FD0646FAF789F84CF27065C2F2BA
:108C900001059FED1D0A01462846FAF7DFFA4DF25D
:108CA00054144CF6501840F280574E44C2F201045E
:108CB000C2F20108C2F2000714E000BFE06A3946C0
:108CC0000022002300F00AFE2846FAF7FDFB2846A2
:108CD0003946FAF751F92846FAF760FB304600F0BA
:108CE0005BFD4E44A06A41460022002300F0F6FDE1
:108CF0000028E3D128464146FAF746FCDEE700BFEC
:108D00000000000000407F400000FA430000000027
:108D100000F07AFD04F068FE9FED2B0B53EC102B56
:108D200004F088FC04F01CFE8146002000F024FDC5
:108D300000F060FD044601F03FFE04EB09054DF232
:108D4000001B40F2847740F2FC684DF22C144DF287
:108D500054164CF2680AC2F2010BC2F20007C2F2CA
:108D60000008C2F20104C2F20106C2F2010A00BF09
:108D700058463946424601F0E7FD2046394601F0A3
:108D800025FEF06A00F086FEF06A594600220023B4
:108D900000F038FE306A00F07DFE306A2146002285
:108DA000002300F02FFEB06B00F074FEB06B514654
:108DB0000022002300F026FE284600F0EDFC4D4482
:108DC000D6E700BF00BF00BF0000000000407F40AA
:108DD00000F01AFD04F008FE9FED270B53EC102B5A
:108DE00004F028FC04F0BCFD8046002000F0C4FC28
:108DF00000F000FD0446F9F7D7FFF9F7CFFF40F286
:108E0000A075C2F200059FED1E0A00F5C07128464C
:108E1000FEF798FE28460221FFF754FB04EB0806F4
:108E20004DF2541940F638174DF2251440F2000A5D
:108E3000C2F20109C2F20007C2F20104C4F27A5A76
:108E4000D9F8200039460022002300F047FD387889
:108E5000B98C207028466180C5F8C0A0F9F7B4FA33
:108E600028462146FEF738FE304600F095FC464481
:108E7000E6E700BF00BF00BF0000000000407F40E9
:108E80000000FA430000000000F0BEFC04F0ACFD5E
:108E90009FED190B53EC102B04F0CCFB04F060FD9C
:108EA0000446002000F068FC00F0A4FC0746F9F737
:108EB00075FF4DF20025C2F201059FED110A00F584
:108EC0004A71284600F074F840F66016C2F20006B7
:108ED00002202744307000BF284600F0ADF8284635
:108EE000314600F00FF8284600F098F8384600F0B8
:108EF00053FC2744F0E700BF0000000000407F4023
:108F00000000FA43002818BF002902D14FF0FF30BB
:108F10007047B0B52DED028B0446F9F7B5F8D4E9EA
:108F20000023801A994105F0ACF99FED1E0A01EE6D
:108F3000100A81EE000A84ED020AF9F7A5F8E2684A
:108F40009FED191A92ED000A9FED188AD4ED310AAF
:108F5000D4ED021AC4E9000120EE010A04F1540024
:108F6000B0EE481A84ED050A04F11805FEF7BEF9C3
:108F7000D4ED021AD4ED2E0A2846B0EE481AFEF7B8
:108F8000B5F9B1EE400A04F1900084ED2C0AFDF72A
:108F900061F984ED2C0ABDEC028BBDE8B0404FF0C6
:108FA000FF30704700247449DB0FC9400000000007
:108FB00080B3B0B52DED028B0446C1600120207452
:108FC00004F1540001F12C020121B0EE408A04F1B9
:108FD0001805FEF743FAE068012100F10C0228466B
:108FE000B0EE480AFEF73AFAE068B0EE480AD0ED73
:108FF000130A04F19000FDF76BF9F8F715FCE0682F
:109000000430FDF713FD0020BDEC028BBDE8B0403D
:1090100040B27047FF2040B27047000010B50446D0
:10902000C0680430FDF72AFCE06894ED2C0A043097
:10903000FDF758FD10BD0000F0B110B50446C06842
:109040000430FDF79FFDE0680430FDF7B5FC00F14A
:1090500008030ECB406904F1B40C8CE80E00C4F890
:10906000C00094ED2D0A00F031FB84ED310A0020A0
:10907000BDE8104040B27047FF2040B2704700008A
:1090800080B5806B0021C185FCF744FE80BD0000E7
:10909000016851E8031F026821F4907142E803134C
:1090A000002BF5D1016851E8051F026821F001018C
:1090B00042E80513002BF5D1016B01290AD100BF4D
:1090C000016851E8031F026821F0100142E8031310
:1090D000002BF5D1202180F8421000210163704758
:1090E00080B50168CA6822F04002CA60202180F879
:1090F0004110FDF777F880BD006841F20001C4F22D
:109100000101884204BF0020704744F60001C4F208
:109110000001884204BF0220704744F20041C4F2BB
:109120000001884214BF04200120704780B582B03E
:1091300090F8421022291ED18268B2F5805F02D1D8
:10914000016900294AD0816AB2F5805F07D00AB967
:10915000026922B10268526802F07F0201E00268EF
:1091600052680A700121826A11448162C18D0139FD
:109170000A04C18501D002B080BD0168CA6822F02E
:109180002002CA60CA6822F48072CA604A6922F06A
:1091900001024A61202180F8421000214163026BE4
:1091A000012A23D1016300BF016851E8031F02684F
:1091B00021F0100142E80313002BF5D101680A6881
:1091C000D20606D5002201920A68019249680191EF
:1091D0000199818DFCF79CFD02B080BD0168826A17
:1091E00049686FF35F2111800221BCE7FCF7E6FFBD
:1091F00002B080BD10B504460068D4E902C22369FC
:10920000016921F4405111430161626943EA0C0193
:10921000E3691143C268194349F20C639A4311434D
:10922000C1604169A26921F4407141F200431143D8
:1092300040F48062C4F201039A42416102D1FBF71B
:10924000EBFB01E0FBF7D6FBE16963681922B1F59E
:10925000004FA0FB02011CD15A00DB0FF7F73AF8D0
:1092600048F21F51C5F2EB11A0FB01235A096FF020
:10927000630302FB0300322303EBC000A0FB0101E8
:109280004FF4F87000EA111000EB0210C1F3421124
:109290001AE09A009B0FF7F71DF848F21F51C5F22C
:1092A000EB11A0FB01235A096FF0630302FB0300DB
:1092B000322303EB0010A0FB0101F02000EA511063
:1092C00000EB0210C1F3431122680843906010BD07
:1092D00090F84110212923D18168B1F5805F01D137
:1092E000016931B1016A02684B1C0362097851605F
:1092F00007E0016A036831F8022B6FF35F225A60BE
:109300000162C18C01390A04C18418BF704700682A
:10931000C16821F08001C160C16841F04001C160B5
:109320007047000010B540F2B064C2F2000420465D
:10933000FCF704FD2046F8F7CFFE10BDFEE7000065
:1093400000F0FF40B0F1FF4018BF0120704700005F
:1093500000F0FF40B0F1FF4018BF0120704700004F
:1093600020F00040A0F1FF40B0FA80F040097047C3
:10937000002848BF704700F01F01012202FA01F1E6
:109380004EF280124009CEF2000242F82010BFF3E4
:109390004F8FBFF36F8F7047002848BF704700F0B2
:1093A0001F01012202FA01F14EF200124009CEF231
:1093B000000242F8201070474EF60C50CEF200002A
:1093C0000068C0F3022070474EF6145300F00F02FD
:1093D000CEF2000309011A4400F16043B0F1FF3FEF
:1093E000C8BF03F564421170704700004EF61F506D
:1093F000CEF2000000210170704700004EF60C51C3
:10940000CEF200010A684FF6FF031A4060F30A2209
:1094100042F0806040F0FD700860704770B52DED3F
:10942000048B044600284FF0FF0018BF002900F00D
:10943000B380B5EE400AB0EE408AF1EE10FA40F388
:10944000AB800020C4F828142073F8F7EDF96025EC
:10945000D4F828042844FDF7E9FA0835802DF7D11F
:10946000802500BFD4F828042844FDF7DFFA08352A
:10947000A02DF7D14EF2C850C0F6000090E80E00C3
:10948000C06804F5836C04F5387500268CE80E007E
:10949000C4F82404D4F82814A81901F140020121C9
:1094A000B0EE480AFDF7DAFF3C36F02EF2D16FF04D
:1094B000EF0500BF6619D4F8282406F5387001219D
:1094C000B0EE480AFDF7CAFFD4F8281406F5F87084
:1094D00001F120020121B0EE480AFDF7BFFF3C3543
:1094E000E8D1B3EE049A04F24C40B0EE480AF0EE34
:1094F000490AFCF7EDFE04F26C40B0EE480AF0EECB
:10950000490AFCF7E5FE04F28C40B0EE480AF0EEA2
:10951000490AFCF7DDFE04F2AC40B0EE480AF0EE7A
:10952000490AFCF7D5FE04F2CC40B0EE480AF0EE52
:10953000490AFCF7CDFE04F2EC40B0EE480AF0EE2A
:10954000490AFCF7C5FE04F20C50B0EE480AF0EEF2
:10955000490AFCF7BDFE04F22C50B0EE480AF0EECA
:10956000490AFCF7B5FE04F24C50B0EE480AF0EEA2
:10957000490AFCF7ADFE04F26C50B0EE480AF0EE7A
:10958000490AFCF7A5FE04F28C50B0EE480AF0EE52
:10959000490AFCF79DFE002040B2BDEC048B70BD73
:1095A0007047000040F6DB7110EE100AC3F6C97177
:1095B00061F31E0000EE100A70470000F0B581B0A4
:1095C000F0B104464CF68C40C2F201000068A042A3
:1095D0001FD001F0A5FA40F27870C2F20000656970
:1095E00007684CF69840C2F20100066801F0BCFA28
:1095F000BD424FF0020018BFB5420DD101B0F0BD21
:109600004FF0500080F31188BFF36F8FBFF34F8F7F
:10961000FEE7002001B0F0BD4AF2C430C2F2010002
:1096200085420CD04AF2D8310120C2F20101002D4E
:1096300008BF04208D4208BF042001B0F0BDA06A1D
:1096400010B1022001B0F0BD94F85C100320012994
:1096500008BF022001B0F0BD4FF0FF3101FA00F069
:10966000C04302EE100A30EE600AB8EEC22A31EEB4
:10967000601A20EE020A80EE010ABDEEC00A10EE6A
:10968000100A704700207047FBF77AF8FEF74CFF8E
:10969000FDF79EFBFDF748FBFDF706FBFDF724FBFE
:1096A000FDF75AFCFDF778FCFDF796FCFDF700FD91
:1096B000FDF71AFDFDF734FDFDF7B6FC00F0A8F844
:1096C000FDF768FB00F0CEF8FEE7000040F22470E2
:1096D000C2F2000090ED001A9FED132A30EE411AFD
:1096E00080ED000AB4EE421A4CF6E430F1EE10FAC6
:1096F000C2F2010002DD4FF0FF3107E09FED0B2ABF
:10970000B4EE421AF1EE10FA03DA012102681144B4
:10971000016090ED001A9FED062AB8EEC11A21EE05
:10972000021A31EE000A7047DB0F4940DB0F49C0D7
:10973000DB0FC940401A811000EE101A9FED0B1A82
:10974000B8EEC00A30EE011A9FED0A2A0C28C8BFF5
:10975000B0EE410A9FED061AB4EE420A30EE011A4D
:10976000F1EE10FAB8BFB0EE410A7047DB0FC9C086
:10977000DB0FC940DB0F49C0EFF3058100291CBF97
:109780006FF005007047002804BF0020704780B5C7
:1097900001F0CAFA002080BD10B582B0EFF3058158
:1097A00019B16FF0050002B010BD044602F0D4FB01
:1097B000211A0129019005DB01A801F0DFFA002040
:1097C00002B010BD6FF0030002B010BD80B502F012
:1097D000AFFB022808BF80BD08B9032080BD40F25E
:1097E0009040C2F2000000680138B0FA80F04009F1
:1097F00080BD000080B5EFF3058010B102F0B2FB30
:1098000080BD02F0A9FB80BD4FF47A707047000064
:10981000EFF3058000281CBF6FF00500704740F291
:109820009040C2F200000168002911BF4FF0FF30E4
:10983000012101600020704780B5EFF3058000280A
:109840001CBF6FF0050080BD02F072FB28B102283A
:1098500005D101F03FFC002080BD012080BD4FF00C
:10986000FF3080BD10B5EFF3058000281CBF6FF0FE
:10987000050010BD40F29044C2F2000420680128A7
:109880001CBF4FF0FF3010BDFEF794F8022020609F
:1098900001F0CCFB002010BD10B5EFF3058018B12E
:1098A0006FF00504204610BD02F042FB02280ED0E6
:1098B00080B902F02FFD01284FF001040CD002F016
:1098C00037FB002808BF4FF0FF34204610BD0024AE
:1098D000204610BD4FF0FF34204610BD10B582B0B9
:1098E0001C46B0FA80F3B1FA81F25B095209EFF33A
:1098F000058CBCF1000F42EA030219D0002C18BFFE
:109900000124224315D10022019201AA01F0EAFFAD
:1099100001281AD10198A8B14EF60450CEF20000E9
:109920004FF080510160BFF34F8FBFF36F8F09E09D
:109930001AB16FF0030002B010BD224601F010FF13
:10994000012806D1002002B010BD6FF0020002B065
:1099500010BD6FF00100002C08BF6FF0020002B0D4
:1099600010BD0000B0B582B0144600294FF00005CC
:10997000EFF3058218BF002802D1284602B0B0BD1F
:10998000002AFAD19CB1A568D5B1E268502A16D355
:109990002269A2B1D4F814C001FB00F2002394455F
:1099A0004FF0000228BF012210D24DB10EE001237A
:1099B00000226AB9E3B1002201F0C6FC0EE01DB935
:1099C000E2680AB92269C2B100220023002AF1D05C
:1099D000A36822690025009501F0DAFC054655B11F
:1099E000002C14BF21680021284601F067F9C4E764
:1099F0000025002DF4D10025BFE76269B2FA82F29A
:109A00005309D5E7B0B582B01C46B0FA80F3B1FA7D
:109A100081F5EFF305825B096D09002A43EA05022F
:109A200007D0002C18BF0124224306D06FF0030595
:109A30002CE0CAB16FF0030528E00022019201AAD0
:109A4000002301F003FE01281CD10198E8B14EF675
:109A50000450CEF200004FF080510160BFF34F8FF1
:109A6000BFF36F8F002511E022460023002501F08F
:109A70001BFD01280AD06FF00105002C08BF6FF014
:109A8000020503E06FF0020500E00025284602B061
:109A9000B0BD000010B5EFF3058119B16FF00504FA
:109AA000204610BD00280FBF6FF0030400210024E2
:109AB00001F0BAFC204610BD10B50C46EFF305814D
:109AC00000291CBF6FF0050010BD014620F0010009
:109AD00050B111F001010AD1214601F059FF0128CE
:109AE00004BF002010BD09E06FF0030010BD214647
:109AF00002F032F8012804BF002010BD6FF0010011
:109B0000002C08BF6FF0020010BD000070B5EFF32D
:109B10000581B9B90028044614BF60680020010718
:109B200010D494B1A36843B1E26800214F2A4FF0EA
:109B3000000288BF01220AD84BB9E168B1FA81F16D
:109B4000490903E00025284670BD0121002200F0EC
:109B500001063AB1A168002E0CBF0120042001F0DB
:109B6000E1FB06E0C9B1002E0CBF0120042001F08A
:109B7000CDFB054635B1002C14BF216800212846D5
:109B800001F09CF8B5FA85F0400986F00101084320
:109B900008BF45F00105284670BD0025002DEAD11B
:109BA000F0E7000080B5EFF3058100291CBF6FF0DE
:109BB000050080BD014620F0010040B111F0010117
:109BC00008D100210022002301F06EFC04E06FF0B8
:109BD000030080BD01F0A2FD013818BF6FF0020044
:109BE00080BD0000B0B584B048B3B1F1FF3F26DDC1
:109BF00004464FF0FF300390EFF3058018B30025C3
:109C00000DF1080C2046012200230295CDF800C07A
:109C100002F0F2F803AB204600210022009502F08A
:109C2000EBF80298D0B14EF60450CEF200004FF09F
:109C300080510160BFF34F8FBFF36F8F0EE06FF065
:109C4000030003900AE020460122002302F056F8A8
:109C500003AB20460021002202F050F8039804B024
:109C6000B0BD00002DE9F04F83B00C46EFF3058145
:109C700029B16FF00507384603B0BDE8F08F0546FF
:109C8000002849D44FF0000B9246A00758BFAB46BE
:109C900002F062F900906FF0010804F001005446F0
:109CA0000027BAF1000F08BF6FF00208019002E030
:109CB0004746002EDFD00020594602AA234602F074
:109CC00005FA06460128F3D1029807EA050140EAA1
:109CD00001090198002809EA050007D100286FF062
:109CE000020718BF4F4607D0C5E700BFA8426FF074
:109CF000020708BF4F46BED0BAF1000FBBD002F03A
:109D00002BF900994F46401A241A4FF0000038BF33
:109D10000446002ECFD1AEE76FF00307ABE700009B
:109D200080B502F0FFF880BD70B584B08E4600218A
:109D300000280391EFF3058146D0002944D1FAB100
:109D40009369002B08BF1823382B16D81179C9073F
:109D500013D15569946811684FEA950C002D08BF1E
:109D60004FF0800CFCB1D668602E1BD3D5B11569BD
:109D7000C5B10024012555B91BE0002004B070BD19
:109D80000124002118234FF0800C00258DB1946828
:109D900012690294CDE900326246734601F072FF07
:109DA000039011E00CB9D4689CB100250024002D6B
:109DB000EDD14CB103AC00931FFA8CF273460194C1
:109DC00001F02CFF012802D1039804B070BD0020DF
:109DD000E6E71469B4FA84F46409D6E710B5EFF342
:109DE000058100291CBF6FF0050010BD044660B15D
:109DF0002046FFF7E3FB042804BF6FF0020010BD0C
:109E0000204601F00FF8002010BD6FF0030010BDD8
:109E1000F0B581B00D464EF2D4114CF68C46C2F22C
:109E20000101C2F201060F6831680446081D00F006
:109E300001FE601C0AD14DB13068011D4AF2C430E8
:109E4000C2F2010000F054FE01B0F0BD3068E41928
:109E500044600AD34CF69840C2F2010000683168B1
:109E6000043100F027FE01B0F0BD40F27870C2F27C
:109E7000000000683168043100F01CFE4AF2B03086
:109E8000C2F2010001688C4238BF046001B0F0BD2D
:109E900070B5044600F044FE4AF21030C2F20100F0
:109EA00001684CF68C4501310160C2F20105296858
:109EB0004EF2D016C2F2010641B1306860B928688E
:109EC000E16AC06A884298BF2C6005E02C60006897
:109ED000012801D100F0E0F94AF21830C2F2010085
:109EE00001680131016061644AF21C31C2F2010172
:109EF000E06A0A68904288BF08604CF69C4100EB1B
:109F00008000C2F2010101EB8000211D00F0F0FD94
:109F100000F02AFE306880B12868E16AC06A884291
:109F200028BF70BD4EF60450CEF200004FF08051B5
:109F30000160BFF34F8FBFF36F8F70BD70B582B0FC
:109F400000F0EEFD4EF2D816C2F20106306850BBAA
:109F50004AF28034C2F20104204600F09BFD4EF22A
:109F60004415C2F20105284600F094FD4CF69040DD
:109F7000C2F20100046040F27C70C2F200004CF6B4
:109F8000E83240F2287305600025C2F20102C2F2F5
:109F900000030A201021009501F0FAF9306010B199
:109FA00003A100F08BFE00F0DFFD02B070BD00BF2A
:109FB000546D725100000000F0B581B04DF6E025FF
:109FC000C2F201052868E0B14AF2D8364AF21037E9
:109FD000C2F20106C2F2010700F0A2FDF068C468F7
:109FE000201D00F027FD38680138386028680138E6
:109FF000286000F0B9FD204600F058F828680028D5
:10A00000EAD101B0F0BD000080B5026C002A08BFA3
:10A0100080BDD0E902C31344C360634524BF036815
:10A02000C360C36808461946F6F732FA80BD0000DF
:10A0300070B5866B036C0446E3B115461AB3E0684D
:10A040001A46F6F725FAE168206C2268091A91424F
:10A05000E16003D2A16840420844E060A81EB0FA63
:10A0600080F040093146002E18BF01210840361A01
:10A07000002516E02068002598B9A06802F06EF867
:10A08000A56005460DE060681A46F6F701FA216CF6
:10A09000D4E90102002508446060904224BF206892
:10A0A0006060711C2846A16370BD000010B50446B5
:10A0B00090F85D00022808BF10BD012803D030B918
:10A0C000206B00F069FD204600F066FD10BD4FF0EA
:10A0D000500080F31188BFF36F8FBFF34F8F00BF25
:10A0E000FEE70000416A00290FBF0020006B0068F6
:10A0F000C0F13800704700004CF69041C2F20101F7
:10A1000009680A68B2FA82F35B090360002A0EBF8D
:10A110000020C8680068704740F66C10C2F200006A
:10A12000C21D22F0070210F0070CA0EB020318BFBB
:10A1300010464AF2BC32C2F201020021C2E900011B
:10A1400049F69912C0F20102BCF1000F18BF1A447F
:10A150000244083A4CF6944322F00702C2F201038B
:10A160001A60C2E90011111A1A68C0E900214EF202
:10A170007010C2F2010001604AF2AC30C2F201007C
:10A1800001604AF29430C2F201000121017070476F
:10A190004CF69C444EF60455C2F20104CEF2000582
:10A1A0004FF08056FFF708FF20680228FAD32E6090
:10A1B000BFF34F8FBFF36F8FF4E70000002808BF95
:10A1C000704780B500210160C0E902110021002222
:10A1D000002301F069F9BDE880407047B0B5049DE7
:10A1E000002914BF2A602D60C5E90F01284601210E
:10A1F0001C4601F019F985F84C40B0BD2DE9F04737
:10A200000A9C8246206B16460F46DDE908599100EC
:10A21000A5229846F6F7B3F9206B00EB8600A0F173
:10A22000040020F007067FB104F13400002100BFD4
:10A230007A5C42547A5C1AB10F2901F10101F7D31B
:10A24000002084F8430002E0002084F83400002756
:10A25000201D372D28BF3725E562C4E9135700F0CC
:10A2600025FC04F1180000F021FCC5F13800A061C4
:10A27000304651464246246164626765A76584F8AA
:10A280005C7000F04BFBB9F1000F206018BFC9F8FB
:10A290000040BDE8F0870000B0B54CF69C450024B6
:10A2A000C2F20105281900F0F5FB1434B4F58C6FE7
:10A2B000F8D14AF29834C2F20104204600F0EAFBD9
:10A2C0004EF25815C2F20105284600F0E3FB4EF2AB
:10A2D0007C10C2F2010000F0DDFB4AF2D830C2F27D
:10A2E000010000F0D7FB4AF2C430C2F2010000F0D6
:10A2F000D1FB40F27870C2F2000004604CF6984046
:10A30000C2F201000560B0BD80B54AF2BC32C2F2B3
:10A31000010200BF114612688242FBD3D1F804C08B
:10A3200001EB0C03834203D1406860444860084657
:10A33000D0F804C000EB0C03934201D013460BE0AD
:10A340004CF69443C2F201031B689A4204D0D2E94E
:10A35000003E0EEB0C0242608142036018BF0860B1
:10A3600080BD000080B58C46014641F804CF94457D
:10A37000006108D99A4201D29C4511D24CF6904016
:10A38000C2F2010007E08069D21A824208D240F28C
:10A390007C70C2F20000006800F08CFB002080BDE1
:10A3A000012080BD10B5044600F0BAFBA06BB0FAE6
:10A3B00080F0440900F0D8FB204610BD10B50446DB
:10A3C00000F0AEFBA06BE16B401AB0FA80F04409DC
:10A3D00000F0CAFB204610BD08480068006880F302
:10A3E00008884FF0000080F3148862B661B6BFF3AE
:10A3F0004F8FBFF36F8F00DF00BF00BF08ED00E09D
:10A4000070B582B04CF69042C2F201021268054665
:10A41000D2680E46D468201D00F00CFB94F828008A
:10A42000410704D400F0FE0084F8280010E0A06981
:10A430003246411920462B46FFF794FF40B10026D3
:10A44000204600212A460023009602F027F820B17A
:10A45000216A2046884702B070BD4FF0500080F35B
:10A460001188BFF36F8FBFF34F8F00BFFEE700006F
:10A470002DE9F04186B04EF2D817C2F201073868D4
:10A4800002A900224FF0000801F06AF900286AD002
:10A4900001AC02AD0BE000F0FE0086F8280000BF22
:10A4A00038682946002201F05BF900285BD0029849
:10A4B000B0F1FF3F03DCDDE90320059990470298E6
:10A4C0000028EDD4049E706910B1301D00F0B2FA7E
:10A4D000204600F0B3F802990929E1D80246DFE8E6
:10A4E00001F0080808052A390808052A96F8280006
:10A4F000D1E796F82800039BB16940F0010086F887
:10A50000280019443046FFF72DFF0028C8D0316AD3
:10A510003046884796F828004007C1D50398B169AE
:10A5200000230A1830460021CDF8008001F0B6FF64
:10A530000028B5D123E096F8280040F001010398E7
:10A5400086F82810B06188B1811830461346FFF7AD
:10A5500009FFA5E796F8280081073FF59CAF304634
:10A5600000F01AFB9CE706B0BDE8F0814FF0500008
:10A5700080F31188BFF36F8FBFF34F8FFEE74FF06B
:10A58000500080F31188BFF36F8FBFF34F8F00BF70
:10A59000FEE7000070B582B00E46044600F09AFD5A
:10A5A00001A800F04BF8019919B101F0B3FE02B017
:10A5B00070BD05464EB9A54207D301F0ABFE20465B
:10A5C0002946FFF71DFF02B070BD4EB140F27C700E
:10A5D000C2F2000000680068B0FA80F0420900E0B2
:10A5E00000224EF2D810C2F201000068611B00F098
:10A5F00079FB01F08FFE0028D9D14EF60450CEF23F
:10A6000000004FF080510160BFF34F8FBFF36F8F99
:10A6100002B070BD40F27870C2F2000001680968B3
:10A6200021B10068C068C068406801E04FF0FF30A9
:10A630004AF2B031C2F201010860704770B50446B9
:10A6400001F08AFC4CF68846C2F2010631680546E4
:10A65000884203D200F008F8012000E000202060CA
:10A660002846356070BD00002DE9F04182B04CF6FF
:10A670009047C2F201073868016891B34FF00008B3
:10A6800009E000BF606038682946246100F012FAD2
:10A690003868016829B3C068C4680668251D284663
:10A6A00000F0C8F9216A2046884794F8280040073E
:10A6B000EED5A0693044B042E4D8204600213246AD
:10A6C0000023CDF8008001F0E9FE0028E0D14FF032
:10A6D000500080F31188BFF36F8FBFF34F8F00BF1F
:10A6E000FEE740F27C71C2F200010A6808603A603D
:10A6F00002B0BDE8F081000081B0002000904CF273
:10A700000400C2F2010000684FF0500181F311888B
:10A71000BFF36F8FBFF34F8F013001D0FEE700BF53
:10A7200000980028FCD001B07047000082B001AC56
:10A730002046FFF7E1FC0199FFF72CFFFFF798FE99
:10A74000F6E70000F0B581B0044600F0E9F994F9AD
:10A750004560012E0FDB04F1240500BF286850B1CD
:10A76000284601F08FFD002818BF00F0CBFB70B227
:10A77000013E0128F2DCFF2684F8456000F0F4F980
:10A7800000F0CEF994F94470012F0EDB04F11005AE
:10A79000286850B1284601F075FD002818BF00F068
:10A7A000B1FB78B2013F0128F2DC84F8446000F08C
:10A7B000DBF901B0F0BD00002DE9F04381B00446A3
:10A7C00000F088FC4CF69446C2F20106306800287E
:10A7D00008BFFFF7A1FC4AF29438C2F2010898F8CA
:10A7E0000000002818BF4FF0004020420DD0002488
:10A7F00001F090FD60071ED04FF0500080F31188EB
:10A80000BFF36F8FBFF34F8FFEE7C4B114F00700A3
:10A8100004F108011EBF081A00F108015FEA417047
:10A820000ED04FF0500080F31188BFF36F8FBFF34D
:10A830004F8F00BFFEE7204601B0BDE8F083002146
:10A840004AF2AC39C2F20109D9F800004A1E82422C
:10A85000CDD24AF2BC30C2F2010005682F4657F84B
:10A86000042F8A4211D22B685BB100BF1F4657F8F4
:10A87000042F28461D468A4207D22B68002BF5D1AB
:10A8800003E04AF2BC30C2F2010033689D42AED010
:10A8900004682B68521A112A036010D36818430702
:10A8A00009D04FF0500080F31188BFF36F8FBFF3D2
:10A8B0004F8F00BFFEE742603960FFF725FD4EF283
:10A8C00070103968D9F80020C2F201000368511AEB
:10A8D0009942C9F8001038BF016098F80000396843
:10A8E00000284FF0000018BF41F0004128604AF2F4
:10A8F000B430C2F20100026808343960511C0160B2
:10A9000076E700004CF68C40C2F20100016819B1F4
:10A9100001680A6D01320A650068704703464AF211
:10A92000F960C0F600004FF0807C21F0010103E9DE
:10A9300003106FF0020043F8240CA3F1440043F825
:10A94000202C704700000000B0B58A890446C82A50
:10A9500023D0B2F5E16F22D101202070B1F90400BB
:10A96000B1F90050A0F5437003F027F89FED0E0BEE
:10A9700053EC102B03F0C4F802F076FDA0602846DB
:10A9800003F01BF89FED0A0B53EC102B03F0B8F803
:10A9900002F06AFD60600020B0BD00202070002041
:10A9A000B0BD00BF00BF00BFEE42B24A0ADB483F65
:10A9B000FC90728EDF3F623F80B54DF20C10C2F208
:10A9C00001001921FCF7E6FD80BD000000291CBF35
:10A9D00001220270CA89B2F5E16F04BF00228284AD
:10A9E000098AB1F5E16F06D0B1F57A7F08D0C829A0
:10A9F00004D1002105E040F201118184002070475C
:10AA0000012181840020704702EE100A4FF0FF30D0
:10AA1000884030EEC01AB8EEC22AC04321EE021AB6
:10AA200002EE100AB8EEC22A81EE021A31EE000AD6
:10AA300070470000D0E9013201699A60D1F804C082
:10AA400082688445536008BF4A600022026108683A
:10AA500001380860086870474AF22033C2F20103E7
:10AA600003604DF6E420C2F201000860802010600F
:10AA7000704700004EF2E403C2F2010303604DF69A
:10AA8000E440C2F2010008604FF48070106070472B
:10AA9000704700004FF0FF31024642F8081F0021C6
:10AAA0004260C0E90322016070470000002101619B
:10AAB0007047000080B5D1F800C01CF1010207D03A
:10AAC00000F108039E465B681A686245FAD901E006
:10AAD000D0F810E0DEF8042008614A609160C1F807
:10AAE00008E0CEF8041001680131016080BD00006B
:10AAF000D0F800C0436808619A684B608A609A6821
:10AB0000996051600CF1010101607047DFF80C00A1
:10AB1000016841F470010160704700BF88ED00E0FA
:10AB20004FF0500080F31188BFF36F8FBFF34F8F4A
:10AB30004CF20400C2F2010001684A1C026001B13B
:10AB400070474EF60450CEF200000068000608BFC1
:10AB500070474FF0500080F31188BFF36F8FBFF341
:10AB60004F8F00BFFEE700004CF20400C2F201006C
:10AB7000016839B10139016018BF7047002080F3C6
:10AB8000118870474FF0500080F31188BFF36F8F2A
:10AB9000BFF34F8FFEE70000B0B5002808BFB0BD7F
:10ABA00004464AF29430C2F20100007854F8041CC2
:10ABB000002818BF4FF0004008420CD0A4F108054F
:10ABC0002A6892B14FF0500080F31188BFF36F8F65
:10ABD000BFF34F8FFEE74FF0500080F31188BFF3B3
:10ABE0006F8FBFF34F8F00BFFEE721EA000044F8EC
:10ABF000040C00F06FFA4AF2AC31C2F2010154F8D1
:10AC0000040C0A68104408602846FFF77DFB4EF2EA
:10AC10007810C2F2010001680131016001F07AFB95
:10AC2000B0BD00004EF21000CEF200000021016025
:10AC3000816040F20001C2F20001096844F6D3527B
:10AC4000C1F26202A1FB02124FF0FF3101EB92113F
:10AC50004160072101607047EFF30580102814D38D
:10AC60004EF2F031CEF20001405C4DF6D821C2F236
:10AC700001010978884208D24FF0500080F3118812
:10AC8000BFF36F8FBFF34F8FFEE74EF60C50CEF23F
:10AC900000004AF208310068C2F20101096800F4BC
:10ACA000E060884298BF70474FF0500080F31188F1
:10ACB000BFF36F8FBFF34F8FFEE700004EF2901C83
:10ACC0000022C2F2010C00BF5CF8323023B1013225
:10ACD000082A08BF7047F7E70CEBC2034CF83210A4
:10ACE0005860704770B515460E460446FFF718FFCA
:10ACF00094F84400FF2804BF002084F8440094F82E
:10AD00004500FF2804BF002084F84500FFF72CFF12
:10AD1000A06B28B904F1240031462A4600F014F94A
:10AD20002046FFF70FFD70BD10B5D8B104464AF2BA
:10AD30001430C2F20100006848B14FF0500080F3B7
:10AD40001188BFF36F8FBFF34F8F00BFFEE700F096
:10AD5000C1F920460021FFF75BF801F0DBFA00287B
:10AD600018BF10BD4EF60450CEF200004FF08051D7
:10AD70000160BFF34F8FBFF36F8F10BDB0B590B1BF
:10AD80000D46D1B104464AF21430C2F20100006807
:10AD9000E8B14FF0500080F31188BFF36F8FBFF31D
:10ADA0004F8F00BFFEE74FF0500080F31188BFF3D4
:10ADB0006F8FBFF34F8F00BFFEE74FF0500080F35F
:10ADC0001188BFF36F8FBFF34F8F00BFFEE700F016
:10ADD00081F94EF2D410C2F201000068226890425C
:10ADE00002EB050102D2914202D309E0914201D364
:10ADF000814205D92160081A0021FFF709F800E017
:10AE0000216001F087FA002818BFB0BD4EF604504B
:10AE1000CEF200004FF080510160BFF34F8FBFF3BF
:10AE20006F8FB0BD70B50446FFF77AFE4CF68C46C6
:10AE3000002CC2F2010608BF3468251D2846FFF722
:10AE4000F9FDA06A18B104F11800FFF7F3FD4AF20A
:10AE50001830C2F20100016801310160306884429B
:10AE60000CD04AF21030C2F20100016801390160D1
:10AE70002046FFF71BF9FFF7CDFB0DE04AF2D83073
:10AE8000C2F201002946FFF733FE4DF6E020C2F280
:10AE90000100016801310160FFF766FE4EF2D0103B
:10AEA000C2F201000068E8B13068844218BF70BD8A
:10AEB0004AF21430C2F20100006840B14FF0500075
:10AEC00080F31188BFF36F8FBFF34F8FFEE74EF60D
:10AED0000450CEF200004FF080510160BFF34F8F5D
:10AEE000BFF36F8F70BD00004EF27411C2F201010A
:10AEF000096801604EF2D411C2F201010968416093
:10AF0000704700004EF2DC10C2F201000121016026
:10AF10007047000010B568B10C464CF68C41C2F287
:10AF2000010109681831FFF7C5FD20460121FEF730
:10AF30006FFF10BD4FF0500080F31188BFF36F8F8B
:10AF4000BFF34F8FFEE70000B0B590B10D464CF651
:10AF50008C41C2F20101096814461831FFF7C8FD9F
:10AF6000002C18BF4FF0FF3528462146FEF750FF52
:10AF7000B0BD4FF0500080F31188BFF36F8FBFF367
:10AF80004F8F00BFFEE7000070B528B3026D044686
:10AF90001AB3E06C884238BF0846012A1CD1E16A26
:10AFA000814208BF70BD4CF68C42C2F201021268A9
:10AFB000A2421CD0A269E062002A5CBFC0F1380046
:10AFC000A0614CF69C46606901EB8101C2F201066A
:10AFD00006EB8101884214D070BD4FF0500080F321
:10AFE0001188BFF36F8FBFF34F8F00BFFEE74FF0A5
:10AFF000500080F31188BFF36F8FBFF34F8F00BFF6
:10B00000FEE7251D2846FFF715FD4AF21C31C2F266
:10B010000101E06A0A68904288BF086000EB800086
:10B0200006EB80002946FFF763FD70BD10B586B0C2
:10B03000002405A804A903AACDE90444FFF70CFDE8
:10B04000DDE9032005990023CDE901014AF29110C1
:10B05000C0F600001DA1009400F014FE4EF26C1129
:10B06000C2F20101086010B101F0DEF90446601C73
:10B0700022D0012C1ED14FF0500080F31188BFF375
:10B080006F8FBFF34F8F4AF2B030C2F201004FF022
:10B09000FF3101604EF2D010C2F2010001210160C7
:10B0A0004EF2D410C2F2010000210160FEF778FADE
:10B0B00000F08AF806B010BD4FF0500080F3118800
:10B0C000BFF36F8FBFF34F8FFEE700BF49444C457E
:10B0D000000000004AF21430C2F2010001680131A0
:10B0E00001607047B0B54AF21430C2F20100006846
:10B0F00030B14EF2DC10C2F2010001210160B0BD9E
:10B100004EF2DC10C2F2010000210160FEF7BAFA33
:10B110004AF20C31C2F201010A684CF68C459042A9
:10B12000C2F2010504D92B68821A5C6D22445A656B
:10B1300008602868006B0168B1F1A53F0BD1416838
:10B14000B1F1A53F07D18168B1F1A53F03D1C06836
:10B15000B0F1A53F04D0286829683431FFF798FC86
:10B160004AF21C30C2F2010001684CF69C4201EB2D
:10B170008103C2F2010252F823404CB902EB83036F
:10B18000143B00BFB1B153F814490139002CF9D078
:10B1900001EB810302EB830252F8043F5B68141D4C
:10B1A000A342136001D15B6813601268D2682A6001
:10B1B0000160B0BD4FF0500080F31188BFF36F8F76
:10B1C000BFF34F8FFEE7000080B582B04EF2004023
:10B1D000CEF200004CF27021C4F20F11D0F8002919
:10B1E0004B1C9A4209D14FF0500080F31188BFF3F5
:10B1F0006F8FBFF34F8F00BFFEE7D0F800298A4260
:10B2000009D14FF0500080F31188BFF36F8FBFF367
:10B210004F8F00BFFEE701784DF6D8220191FF2144
:10B2200001700178C2F201028DF803109DF803103D
:10B2300001F0500111704AF20831C2F201010722F7
:10B240000A609DF90320B2F1FF3F0CDC0A6800BFE1
:10B250009DF80330013A5B008DF803309DF903300F
:10B26000002BF5D40A600A68032A2DD14FF4E0635D
:10B2700003EA02220A6001990170D0F8201941F412
:10B280007001C0F82019D0F8201941F07041C0F8C1
:10B290002019FFF7C7FC4CF20400C2F201000021A4
:10B2A0000160FFF733FC4EF63470CEF20000016807
:10B2B00041F040410160FFF78FF8FFF713FFFFF700
:10B2C0001BFA002002B080BD4FF0500080F31188BF
:10B2D000BFF36F8FBFF34F8FFEE7000080B54FF0D5
:10B2E000500080F31188BFF36F8FBFF34F8F00F0D2
:10B2F00043FE30B14EF60450CEF200004FF08051C4
:10B300000160002080F3118880BD000010B5024666
:10B310000120002100F018F80446FEF74FFF2046F8
:10B3200010BD000010B582B00B46844601200021FC
:10B330000022CDF800C000F02BF80446FEF73EFFD7
:10B34000204602B010BD0000F0B581B0B0B1054696
:10B350004843503014460E46FFF72EFA074650B1C8
:10B36000002007F1500287F8460028463146234660
:10B370000097FEF733FF384601B0F0BD4FF05000A4
:10B3800080F31188BFF36F8FBFF34F8FFEE700008C
:10B39000B0B582B068B11D46ABB1F1B9EAB14FF0BA
:10B3A000500080F31188BFF36F8FBFF34F8F00BF42
:10B3B000FEE74FF0500080F31188BFF36F8FBFF3AB
:10B3C0004F8F00BFFEE74FF0500080F31188BFF3AE
:10B3D0006F8FBFF34F8F00BFFEE751B14AB94FF0F7
:10B3E000500080F31188BFF36F8FBFF34F8F00BF02
:10B3F000FEE750230193019B502B0AD1069B019C31
:10B40000012485F846400095FEF7E8FE284602B084
:10B41000B0BD4FF0500080F31188BFF36F8FBFF3C2
:10B420004F8F00BFFEE7000070B5F8B104460E462E
:10B43000FFF776FB2068D4E90F12002502FB010319
:10B44000013901FB0201A563C4E90103FF20E160AA
:10B4500084F8440084F8450004F110007EB1FFF741
:10B4600019FB04F12400FFF715FB18E04FF0500022
:10B4700080F31188BFF36F8FBFF34F8FFEE7016832
:10B4800069B100F0FFFE50B14EF60450CEF200005C
:10B490004FF080510160BFF34F8FBFF36F8FFFF705
:10B4A00063FB012070BD00002DE9F04F83B00292D4
:10B4B000B8B11D460E460446E9B1022D03D1E06B3A
:10B4C000012840F09A8000F033FD00BB0298F0B1F3
:10B4D0004FF0500080F31188BFF36F8FBFF34F8F91
:10B4E000FEE74FF0500080F31188BFF36F8FBFF37A
:10B4F0004F8F00BFFEE7206C0028DED04FF05000D9
:10B5000080F31188BFF36F8FBFF34F8FFEE7FFF714
:10B5100007FBA06B022D58D0E16B884255D304F194
:10B52000100801206F464FF0000B0DF108094FF095
:10B53000805A00BF0299002900F07B80C00702D02A
:10B540003846FFF7D1FCFFF70FFBFFF7C3FDFFF70E
:10B55000E7FA94F84400FF2808BF84F844B094F850
:10B560004500FF2808BF84F845B0FFF7FDFA3846CC
:10B57000494600F00FFB00285ED12046FEF71EFF73
:10B58000A0B102994046FFF7C5FC2046FFF7DAF864
:10B5900000F0C0FE78B94EF60450CEF20000C0F8BC
:10B5A00000A0BFF34F8FBFF36F8F04E02046FFF77B
:10B5B000C9F800F0AFFEFFF7B3FAA06B022D04D07C
:10B5C000E16B88424FF00000B4D2204631462A4653
:10B5D000FEF72EFD54F8241FC9B1204600F052FE9C
:10B5E00008B34EF60450CEF200004FF080510160D7
:10B5F000BFF34F8FBFF36F8F15E04FF0500080F314
:10B600001188BFF36F8FBFF34F8F00BFFEE750B1BC
:10B610004EF60450CEF200004FF080510160BFF3AF
:10B620004F8FBFF36F8FFFF79FFA012003B0BDE884
:10B63000F08FFFF799FA04E02046FFF783F800F057
:10B6400069FE002003B0BDE8F08F00002DE9F04353
:10B6500081B0E8B11E46914605460F4609B3022E59
:10B6600002D1E86B012837D1FFF7F6FAEFF3118822
:10B670004FF0500080F31188BFF36F8FBFF34F8FEF
:10B68000A86B022E19D0E96B884216D300203FE048
:10B690004FF0500080F31188BFF36F8FBFF34F8FCF
:10B6A000FEE7286C0028DAD04FF0500080F31188B4
:10B6B000BFF36F8FBFF34F8FFEE795F84540A86B40
:10B6C000284639463246FEF7B3FCFF2C0DD0601CED
:10B6D00085F8450001201BE04FF0500080F31188F1
:10B6E000BFF36F8FBFF34F8FFEE755F8240F70B194
:10B6F000284600F0C7FD0146B9F1000F4FF00100E8
:10B7000006D000291CBF0120C9F8000000E001207C
:10B7100088F3118801B0BDE8F0830000B0B5A8B18E
:10B720008568044600F0FEFB85421CBF0020B0BDCA
:10B73000E0680138E0601CBF0120B0BD2046002158
:10B7400000220023FFF7B0FE0120B0BD4FF05000F3
:10B7500080F31188BFF36F8FBFF34F8FFEE70000B8
:10B760002DE9F04F85B0049298B10C4605460029AA
:10B7700000F0A58000F0DCFBA8B9049898B14FF068
:10B78000500080F31188BFF36F8FBFF34F8F00BF5E
:10B79000FEE74FF0500080F31188BFF36F8FBFF3C7
:10B7A0004F8F00BFFEE705F1240005F1100901905D
:10B7B00002AF0DF1100A4FF000080AE02846FEF72C
:10B7C000C1FF00F0A7FD2846FEF7ECFD002840F081
:10B7D0008480FFF7A5F9D5F838B0BBF1000F1DD074
:10B7E00028462146FEF710FCABF10100A86328694A
:10B7F00070B1484600F046FD50B14EF60450CEF20E
:10B8000000004FF080510160BFF34F8FBFF36F8F87
:10B81000FFF7AAF900200126A0B95FE0049850B113
:10B82000B8F1000F02D13846FFF75EFB4FF0010878
:10B83000012038B952E0FFF797F9002600200028D0
:10B840004CD000BFFFF790F9FFF744FCFFF768F911
:10B8500095F84400FF2804BF002085F8440095F8BF
:10B860004500FF2804BF002085F84500FFF77CF95C
:10B870003846514600F08EF900289FD12846FEF741
:10B8800091FDB0B104990198FFF744FB2846FEF7FB
:10B8900059FF00F03FFD00289BD14EF60450CEF238
:10B8A00000004FF080510160BFF34F8FBFF36F8FE7
:10B8B0008FE72846FEF746FF00F02CFD89E7286C4D
:10B8C00000283FF457AF4FF0500080F31188BFF3CA
:10B8D0006F8FBFF34F8F00BFFEE70026304605B0E5
:10B8E000BDE8F08F2DE9F04381B000B391460546E5
:10B8F0000E4631B3FFF7B0F9EFF311884FF0500067
:10B9000080F31188BFF36F8FBFF34F8FAC6B24B3FD
:10B9100095F8447028463146FEF776FB601EFF2FEF
:10B92000A8631CD0781C85F8440001202AE04FF061
:10B93000500080F31188BFF36F8FBFF34F8F00BFAC
:10B94000FEE7286C0028D5D04FF0500080F3118816
:10B95000BFF36F8FBFF34F8FFEE7002012E055F863
:10B96000100F70B1284600F08DFC0146B9F1000FB0
:10B970004FF0010006D000291CBF0120C9F80000CB
:10B9800000E0012088F3118801B0BDE8F0830000D9
:10B990002DE9F04F85B0049158B10446006C90B188
:10B9A0004FF0500080F31188BFF36F8FBFF34F8FBC
:10B9B000FEE74FF0500080F31188BFF36F8FBFF3A5
:10B9C0004F8F00BFFEE700F0B3FA50B9049840B1C2
:10B9D0004FF0500080F31188BFF36F8FBFF34F8F8C
:10B9E000FEE704F1240004F1100501904FF0000877
:10B9F00002AF0DF1100A4FF000094FF0000B0AE002
:10BA00002046FEF79FFE00F085FC2046FEF7CAFCAC
:10BA1000002840F07F80FFF783F8A06BF0B1013879
:10BA2000A063206810B9FEF76DFFA060286870B1B0
:10BA3000284600F027FC50B14EF60450CEF200002C
:10BA40004FF080510160BFF34F8FBFF36F8FFFF74F
:10BA50008BF801260020B8B96FE000BF049850B100
:10BA6000BBF1000F02D13846FFF73EFA4FF0010B51
:10BA7000012048B961E0B9F1000F62D1FFF774F815
:10BA800000200026002858D0FFF76EF8FFF722FBB1
:10BA9000FFF746F894F84400FF2808BF84F8448074
:10BAA00094F84500FF2808BF84F84580FFF75CF84C
:10BAB0003846514600F06EF80028A1D12046FEF726
:10BAC00071FC28B92046FEF73DFE00F023FCA2E7FA
:10BAD000206838B9FFF724F8A06800F089FB814698
:10BAE000FFF742F804990198FFF714FA2046FEF791
:10BAF00029FE00F00FFC00287FF48DAF4EF60450B5
:10BB0000CEF200004FF080510160BFF34F8FBFF3C2
:10BB10006F8F80E7B9F1000F0ED0FFF701F82046D4
:10BB2000FEF7E0FAA168024608461146FFF72CFA34
:10BB3000FFF71AF8002600E00026304605B0BDE801
:10BB4000F08F4FF0500080F31188BFF36F8FBFF379
:10BB50004F8F00BFFEE7000070B568B186680446ED
:10BB60000D4600F0DFF986420FD020462946FFF748
:10BB70000FFF58B9002070BD4FF0500080F31188BE
:10BB8000BFF36F8FBFF34F8FFEE70120E1680131F4
:10BB9000E16070BDB0B5D0B10D4611B30446FEF7FB
:10BBA000BFFF4EF2D410C2F2010001682868421CA7
:10BBB00021D04EF274136268C2F20103D3F800C0C0
:10BBC00091421AD323689C4517D0012422E04FF0FC
:10BBD000500080F31188BFF36F8FBFF34F8F00BF0A
:10BBE000FEE74FF0500080F31188BFF36F8FBFF373
:10BBF0004F8F00BFFEE700240CE0891A884206D967
:10BC0000401A28602046FFF76FF9002402E0002068
:10BC100001242860FEF7A8FF2046B0BD2DE9F043BF
:10BC200083B007469000984615468946FEF7C4FD46
:10BC300078B106466020FEF7BFFD38B104460663C2
:10BC400054B94FF0FF3003B0BDE8F0833046FEF743
:10BC5000A3FF0024002CF4D0DDE90A10002284F8B0
:10BC60005D20CDE90010384649462A4643460294F5
:10BC7000FEF7C4FA2046FEF70BF9012003B0BDE839
:10BC8000F083000070B586B00B9CCCB10C9E06B35F
:10BC900060250495049D602D25D1049DDDF828C004
:10BCA000022586F85D5005AD3463CDE900C50296E6
:10BCB000FEF7A4FA3046FEF7EBF8059806B070BD23
:10BCC0004FF0500080F31188BFF36F8FBFF34F8F99
:10BCD000FEE74FF0500080F31188BFF36F8FBFF382
:10BCE0004F8F00BFFEE74FF0500080F31188BFF385
:10BCF0006F8FBFF34F8F00BFFEE70000F0B581B03C
:10BD0000D0B11D46174604460E46FEF709FF002D2A
:10BD10001CBFA06D286094F85C000221042F84F8F9
:10BD20005C1012D80125DFE807F023031C26200051
:10BD3000A16D3143A1651FE04FF0500080F31188E1
:10BD4000BFF36F8FBFF34F8FFEE7A16D013113D0AB
:10BD50004FF0500080F31188BFF36F8FBFF34F8F08
:10BD6000FEE7A16D0131A16506E0022803D100259F
:10BD700001283CD103E0A6650125012837D1261D05
:10BD80003046FEF757FE4AF21C31C2F20101E06A6A
:10BD90000A68904288BF08604CF69C4100EB800026
:10BDA000C2F2010101EB80003146FEF7A1FEA06A5C
:10BDB00048B14FF0500080F31188BFF36F8FBFF38D
:10BDC0004F8F00BFFEE74CF68C41C2F20101E06AE2
:10BDD0000968C96A88420AD94EF60450CEF20000BA
:10BDE0004FF080510160BFF34F8FBFF36F8FFEF7AD
:10BDF000BBFE284601B0F0BD2DE9F04120B31D4641
:10BE0000174604460E46FEF727FFEFF311884FF062
:10BE1000500080F31188BFF36F8FBFF34F8F002D59
:10BE20001CBFA06D286094F85C000221042F84F8E8
:10BE30005C1012D80125DFE807F023031C26200040
:10BE4000A16D3143A1651FE04FF0500080F31188D0
:10BE5000BFF36F8FBFF34F8FFEE7A16D013113D09A
:10BE60004FF0500080F31188BFF36F8FBFF34F8FF7
:10BE7000FEE7A16D0131A16506E0022803D100258E
:10BE8000012849D103E0A6650125012844D1A06A13
:10BE900048B14FF0500080F31188BFF36F8FBFF3AC
:10BEA0004F8F00BFFEE74AF21430C2F20100006873
:10BEB00030B14EF27C1004F11801C2F2010015E01D
:10BEC000261D3046FEF7B6FD4AF21C31C2F20101D2
:10BED000E06A0A68904288BF08604CF69C4100EB1B
:10BEE0008000C2F2010101EB80003146FEF700FE46
:10BEF0004CF68C41C2F20101E06A0968C96A8842C5
:10BF00000AD9069800281CBF012101604EF2DC10FE
:10BF1000C2F201000121016088F311882846BDE8C2
:10BF2000F08100004CF68C40C2F2010000687047BE
:10BF30004EF2D010C2F201000068002804BF0120B8
:10BF400070474AF21430C2F201000068B0FA80F083
:10BF500040094000704700004EF2D410C2F20100C8
:10BF60000068704780B5FEF777FE4EF2D410C2F23B
:10BF70000100006880BD00002DE9F04F81B04AF259
:10BF80001430C2F20100006840B14AF2B830C2F287
:10BF90000100016800240131016092E04EF2D410EA
:10BFA000C2F2010001684E1C066021D340F2787095
:10BFB000C2F200000168096849B14FF0500080F3F7
:10BFC0001188BFF36F8FBFF34F8F00BFFEE74CF6B2
:10BFD0009842C2F201020168136803604EF27410C5
:10BFE0001160C2F20100016801310160FEF712FB2D
:10BFF0004AF2B031C2F2010108684CF68C4A4CF6A4
:10C000009C488642C2F2010AC2F2010801D2002411
:10C0100045E040F27877C2F20007386800240068F3
:10C0200098B34AF21C3BC2F2010B19E0D9F82C007C
:10C03000DBF80010884288BFCBF8000000EB8000DE
:10C0400008EB80002946FEF753FDD9F82C00DAF8FA
:10C050000010C96A3A68884228BF01241068B8B144
:10C060003868C068D0F80C904D4655F8040F8642E9
:10C0700010D32846FEF7DEFCD9F828000028D5D0DA
:10C0800009F11800FEF7D6FCD0E74FF0FF3005E0CD
:10C090004FF0FF304AF2B031C2F201010860DAF825
:10C0A0000000C06A00EB800058F8200001284EF222
:10C0B000DC10C2F2010088BF01240068002818BF0C
:10C0C0000124204601B0BDE8F08F00002DE9F041C9
:10C0D0001E46154688460746FEF722FD4CF68C4460
:10C0E000C2F20104206890F85C00022819D0206890
:10C0F000816D21EA0701816520684FF0010180F818
:10C100005C1076B130460121FDF782FE4EF60450F8
:10C11000CEF200004FF080510160BFF34F8FBFF3AC
:10C120006F8FFEF721FDFEF7FBFC15B12068806DD7
:10C1300028602068002590F85C100020022905D1B5
:10C14000216801258A6D22EA08028A65216881F842
:10C150005C00FEF709FD2846BDE8F081B0B580B16E
:10C1600004464CF68C40C2F201000068A0420AD09E
:10C170004FF0500080F31188BFF36F8FBFF34F8FE4
:10C18000FEE70020B0BD206D38B3013820654FF0C8
:10C19000000018BFB0BDE16AE26C91421CD0251DC1
:10C1A0002846FEF747FCE06CC0F13801A1614AF275
:10C1B0001C31E062C2F201010A68904288BF086047
:10C1C0004CF69C4100EB8000C2F2010101EB8000C3
:10C1D0002946FEF78DFC0120B0BD4FF0500080F3E2
:10C1E0001188BFF36F8FBFF34F8F00BFFEE70000D2
:10C1F000F0B581B000B34CF68C46C2F2010604469D
:10C20000C06A3168C96A884219D2A169002904D478
:10C210003168C96AC1F13801A1614CF69C47616976
:10C2200000EB8000C2F2010707EB800081420FD0D3
:10C230003068C06AE06221E0002001B0F0BDE16C2E
:10C240003068C26A0020914238BF012001B0F0BDC1
:10C25000251D2846FEF7EEFB30684AF21C31C06A05
:10C26000C2F20101E0620A68904288BF086000EBF8
:10C27000800007EB80002946FEF73AFC012001B060
:10C28000F0BD0000B0B5C068C5687DB105F1180407
:10C290002046FEF7CFFB4AF21430C2F201000068DC
:10C2A00068B14EF27C10C2F201001DE04FF0500068
:10C2B00080F31188BFF36F8FBFF34F8FFEE72C1D04
:10C2C0002046FEF7B7FB4AF21C31C2F20101E86AD0
:10C2D0000A68904288BF08604CF69C4100EB8000E1
:10C2E000C2F2010101EB80002146FEF701FC4CF691
:10C2F0008C41C2F20101E86A0968C96A884291BFAB
:10C3000000204EF2DC11C2F20101012088BF08605A
:10C31000B0BD00002DE9F04F81B04AF21434C2F2F2
:10C320000104206868B1FEF7FBFB2068013820603B
:10C33000206880B10024FEF717FC204601B0BDE85C
:10C34000F08F4FF0500080F31188BFF36F8FBFF371
:10C350004F8F00BFFEE74AF21030C2F201000068C2
:10C3600000285DD04EF27C16C2F2010630684EF213
:10C37000DC18C2F2010890B34AF21C374CF69C4913
:10C380004CF68C4BC2F20107C2F20109C2F2010B5A
:10C390004FF0010AF068C56805F11800FEF74AFB86
:10C3A0002C1D2046FEF746FBE86A3968884288BFA4
:10C3B000386000EB800009EB80002146FEF798FB17
:10C3C000E86ADBF80010C96A884228BFC8F800A0F4
:10C3D00030680028DED1002D18BFFEF71BF94AF2A5
:10C3E000B834C2F20104256855B10126FFF7C4FD37
:10C3F000002818BFC8F80060013DF7D10020206078
:10C40000D8F8000070B14EF60450CEF200004FF0A4
:10C4100080510160BFF34F8F0124BFF36F8F8AE714
:10C42000002488E7002486E780B586B0FDF786FD06
:10C430004EF2D810C2F20100006808B30020CDE926
:10C44000040005A804A903AAFEF714FBDDE90320F4
:10C450000221DDF814C0CDE900104AF22D70C0F6BB
:10C4600000000CA10023CDF808C0FFF70BFC4AF236
:10C47000EC31C2F20101086010B1012006B080BDAC
:10C480004FF0500080F31188BFF36F8FBFF34F8FD1
:10C49000FEE700BF546D72205376630010B584B080
:10C4A000A8B14EF2D814C2F2010484462068C0B18B
:10C4B0000529CDE90012CDF808C015DCFFF738FDDD
:10C4C00001462068022916D1069A694615E04FF008
:10C4D000500080F31188BFF36F8FBFF34F8F00BF01
:10C4E000FEE7002004B010BD69461A460023FFF79E
:10C4F000ADF804B010BD694600220023FEF7D4FF5A
:10C5000004B010BD03B401984100009850EAC12066
:10C5100018BF04204A0D18BF40F0010040F2FF721E
:10C52000B2EB515F08BF40F00200012808BF0520B0
:10C5300002B070474100080218BF04200A0E18BF5D
:10C5400040F001004FF07F4232EA010108BF40F0A5
:10C550000200012808BF05207047000010B54FF009
:10C560000E402DED028BB0EE408A18EE104A00EB23
:10C570004400B0F1506F4AD84FF0FC40B0EB440F8C
:10C5800022D2B0EEC80AF7EE000A30EEC00AF6EE8C
:10C59000000A60EE208A18EE900A00F039FF01EEE2
:10C5A000100A14F0004F1DBFDFED2D0A9FED2D0A7C
:10C5B000B1EE411ADFED2C0A08BF9FED2C0AF8EE10
:10C5C000001A21EE218A05E0DFED290A68EE088ACB
:10C5D000B0EE600A9FED271ADFED271A30EE080A49
:10C5E00048EE811A9FED251A08EEA11ADFED241AF4
:10C5F00048EE811A9FED231A08EEA11A68EE281A58
:10C60000BDEC028B01EE810A30EE200A10BD4FF026
:10C61000E440B0EB440F0CD918EE100AFFF78AFF84
:10C62000042808BF00F02EFEB0EE480ABDEC028BD5
:10C6300010BD4FF07F40B0EB440F07D2B0EE480A78
:10C64000BDEC028BBDE8104000F00EBE0120F3F7F8
:10C65000CDFFBDEC028BBDE8104000F00BBE00002A
:10C660000000C9BF22AAFDB90000C93F22AAFD39B6
:10C670000000000024FE1C3DC78AD83C1E67383DE0
:10C680001B93993DAFAA2A3E70B59B482DED020B36
:10C690002DED068B079D25F00044A04218DC97483D
:10C6A000844202DC0AD1069840B19DED060BBDEC38
:10C6B000068B02B0BDE8704000F0A2BD002DCCBFDB
:10C6C0009FED8F0B9FED900BBDEC068B02B070BD04
:10C6D0008F48A04215DD8F48A042D8BF4FF0FF34ED
:10C6E00058DD9DED060B51EC100BFFF70BFF0428F6
:10C6F00008BF00F0A9FD9DED060BBDEC068B02B056
:10C7000070BD9DED060B51EC100B00F075FECDE9F0
:10C71000060181489FED828BA0423CDD8248A04209
:10C720001FDD00249FED82AB9DED060B53EC1A2B11
:10C7300051EC100B00F0CAFE9DED060B41EC190BFD
:10C7400053EC1A2B51EC100B01F0DAF953EC182BC7
:10C7500001F054FC53EC192B00F06CFFCDE90601FD
:10C7600049E09DED060B012453EC182B51EC100B06
:10C7700000F0ACFE9DED060B41EC190B53EC182BB1
:10C7800051EC100B01F03AFC53EC192B00F052FF66
:10C79000CDE906012FE06848A0421FDD02249FED8D
:10C7A000689B9DED060B53EC192B51EC100B01F01F
:10C7B000A7F953EC182B00F089FE9DED060B41EC18
:10C7C000180B53EC192B51EC100B01F017FC53EC28
:10C7D000182B00F02FFFCDE906010CE09DED060BB4
:10C7E000032453EC102B9FED580B51EC100B00F071
:10C7F00021FFCDE906019DED060B53EC102B51EC0A
:10C80000100B01F07DF941EC180B53EC182B01F0E3
:10C8100077F941EC190B4E480621B0EE490AF0EECB
:10C82000690A784400F070FC53EC182B51EC100BA3
:10C8300001F066F941EC180B4648B0EE490AF0EEFB
:10C84000690A0521784400F05FFC53EC192B51EC88
:10C85000100B01F055F941EC100B51EC180B53EC97
:10C86000102B002C0EDA00F031FE9DED061B53EC70
:10C87000112B01F045F99DED061B53EC112B01F036
:10C88000E5FA35E000F022FE9DED061B53EC112B7E
:10C8900001F036F941EC100B2F48784400EBC4004E
:10C8A00090ED001B51EC100B53EC112B01F0A6FB8B
:10C8B0009DED061B53EC112B01F0A0FB41EC100B7E
:10C8C0002648784400EBC40090ED001B51EC100B9F
:10C8D00053EC112B01F0BAFA41EC100B002DA2BF62
:10C8E000BDEC068B02B070BD51EC100B00F0AFFD3B
:10C8F00041EC100B01E70000000010440000F07F45
:10C90000182D4454FB21F93F182D4454FB21F9BF45
:10C910000000DC3F0000203E0000F33F000000006C
:10C92000000000000000F03F0000E63F00000000B3
:10C9300000000000000000400080034000000000F4
:10C94000000000000000F83F000000000000F0BF01
:10C95000DA1B0000901B00001A1B0000D21A000016
:10C9600070B56F4E2DED040B2DED048B82B0DDF80C
:10C9700024C0DDE907235C422CF000411C4341EA5E
:10C98000D474069D22F00040B44205D86C422C437A
:10C9900040EAD474B4420BD99DED081B9DED060B03
:10C9A00002B0BDEC048B04B0BDE8704000F032BCB6
:10C9B000ACF14054A4F17F641C430BD0022404EA80
:10C9C000AC7444EAD27405439FED578B9FED582B0E
:10C9D00007D015E09DED060B51EC100B00F004FDA7
:10C9E00042E0002C11BF012C9DED060B02B0BDEC06
:10C9F000048B04BF04B070BD022C38D0032C3BD094
:10CA00000B439FED4D1B9FED4E0B0AD0B14218D149
:10CA1000B04209D121F0804120F080400991079077
:10CA20000FE0002A15DA10E0474B7B44002C08BFCA
:10CA300093ED000B0DD0012C10D0022C17D0032C3D
:10CA40001AD0B0421DD1002A03DAB0EE410AF0EE4E
:10CA5000610A02B0BDEC048B04B070BD93ED000B15
:10CA600051EC100B00F0F3FC41EC100BF1E7B0EED1
:10CA7000480AF0EE680AECE7B0EE420AF0EE620A0D
:10CA8000E7E7401A00159FED329B3C28C8BF8DEDAB
:10CA9000000B17DCBCF1000FBCBF10F13C0F8DED9B
:10CAA000009B0FDB9DED080B53EC102B9DED060B4F
:10CAB00051EC100B00F0BEFD00F09EFC00F094FC69
:10CAC000CDE90001B4B1012C10D0022C9FED220B56
:10CAD00053EC102B9DED000B51EC100B19D001F015
:10CAE0008DFA53EC182B01F089FABDE7019880F01C
:10CAF000004001909DED000B53EC192B51EC100BF5
:10CB000000F0F2FE04BF0220F3F770FD9DED000B74
:10CB10009FE701F073FA53EC182B01F097F9A3E7A4
:10CB20000000F07F00000000182D4454FB21094054
:10CB3000182D4454FB2109C0182D4454FB21F9BF82
:10CB4000182D4454FB21F93F021A00000000000098
:10CB50000000000000000000075C143326A6A13C82
:10CB600070B54FF068422DED048BF0EE408A18EE60
:10CB7000900AB0EE608A18EE101A02EB4003B3F18F
:10CB8000654F3CBF02EB4102B2F1654F7DD200BF61
:10CB9000C0F3C753C1F3C7529A1A1B2A09DD10F01C
:10CBA000004F14BF9FED830A9FED830ABDEC048BF9
:10CBB00070BD12F11A0F36DA11F0004F09D010F0E3
:10CBC000004F0CBF9FED7D0A9FED7D0ABDEC048BED
:10CBD00070BD88EE889A19EE100AFFF7ABFC0428A6
:10CBE00008BF00F04FFB18EE900AFFF7A3FC0546C4
:10CBF00018EE100AFFF79EFC044619EE100AFFF724
:10CC000099FC042D18BF052D08D1042C18BF052C44
:10CC100004D1002804BF0220F3F7E8FCB0EE490A73
:10CC2000BDEC048B70BD4200B2EB410F3AD910F05D
:10CC3000004F19BFDFED630A9FED630ADFED630A62
:10CC40009FED630AB0EE481A0A46B1EE688A80F09A
:10CC50000041F0EE418A10460A1A5200B2F1807F7C
:10CC600034D2484010F0004FDFED5A1A9FED5A2A97
:10CC70001DBFBEEE001A70EEE10A30EE420AB6EEBB
:10CC8000001A08BF70EEA10A00E040E008BF30EED5
:10CC9000020AB0EE682A01EE482A08EE818AC2EE46
:10CCA000081A15E011F0004F04BF9FED4C0AF0EE9A
:10CCB000400AD1D010F0004F19BFDFED490A9FEDB7
:10CCC000490ADFED490A9FED490AC5E7C8EE881A0F
:10CCD00021EEA11A9FED462ADFED462A41EE022AF7
:10CCE0009FED452A01EE222ADFED442A41EE022A79
:10CCF0009FED432ABDEC048B01EE222A21EE811A1E
:10CD000001EE020A30EE210A30EE200A70BD4FF02B
:10CD10007F42B2EB400F28BFB2EB410F09D2F0EED9
:10CD2000480AB0EE680ABDEC048BBDE8704000F024
:10CD30009EBA40EA01035B0008BF41F0FF410BD0FF
:10CD4000B2EB400F08BFB2EB410F08D120F080409A
:10CD500008EE900A21F0804108EE101A18E7B2EBB5
:10CD6000400F12BF5FEA410340F0FF4001F0004175
:10CD70003FF40EAFB2EB410F12BF5FEA400200F08A
:10CD8000004041F0FF413FF403AF4A0092EA400304
:10CD90003FF5FEAE002AACBF9FED1A0A9FED1A0ABE
:10CDA00068EE808A28EE008A18EE900A18EE101AB3
:10CDB000EEE60000DB0FC9BFDB0FC93FDB0F4940C8
:10CDC000DB0F49C00000C9BF22AAFDB90000C93F5E
:10CDD00022AAFD390060ED3EC30ACE3700000000F4
:10CDE000000049C022AA7DBA0000494022AA7D3A2B
:10CDF0002DAD65BD8FB8D53D0FB511BE61C84C3E98
:10CE0000A8AAAABE0000804F0000802F10B52DED0B
:10CE1000040B86B09DED060B10EE100A10EE901A72
:10CE20008DED000B002818BF0120084320F00040C2
:10CE3000C0F17F6000F1E040C00F21D19DED080BF3
:10CE400010EE101A10EE900A8DED000B002918BF9D
:10CE50000121084320F00040C0F17F6000F1E04074
:10CE6000C00F0DD129490798B1EB400F04BF0698B8
:10CE7000002842D00998400004BF089800283CD000
:10CE80009DED080B53EC102B9DED060B51EC100B98
:10CE900000F02EFFCDE902019DED020B40F2FF7183
:10CEA00010EE900A8DED000B31EA105021D007985A
:10CEB000039900F0004001F00041884219D09DED37
:10CEC000080B8DED040B9DED020B8DED000B10EEAC
:10CED000900A059961F31E0005909DED041B9DEDE0
:10CEE000020B51EC110B53EC102B00F0AFFFCDE90E
:10CEF00002019DED020B0AB010BD0120F3F776FB95
:10CF00000AB0BDE8104000F08FB900000000E0FF5B
:10CF100000B52DED048BB0EE409AF0EE609A83B030
:10CF200051EC190B00F09EFF41EC180B18EE100AA3
:10CF300018EE901A8DED008B002818BF01200843D1
:10CF400020F00040C0F17F6000F1E040C00F14D03D
:10CF500019EE101A19EE900A8DED009B002918BFEA
:10CF60000121084320F00040C0F17F6000F1E04063
:10CF7000C00F04BF0120F3F739FBB0EE480A03B03D
:10CF8000F0EE680ABDEC048B00BD000000B510EEA9
:10CF9000101A2DED028B81B04D4A6846B2EB410F5D
:10CFA0003CD94FF0E640B0EB410F94BF00204FF06A
:10CFB000FF3000900098B0EE408A00285FDB28EE3A
:10CFC000080ADFED440A9FED441A00EE201ADFED57
:10CFD000430A40EE010A9FED421A00EE201ADFEDEF
:10CFE000410A10F0010F40EE010A9FED3F1A00EEDA
:10CFF000201A61EE000AB0EE480A08EE200A02BFCD
:10D0000001B0BDEC028B00BDBFEE001A01B0C1EE55
:10D01000000ABDEC028BB0EE600A00BD334B21F07C
:10D020000042934228D911F0004FDFED310A20EE83
:10D03000201ADFED300A19BF31EE601A71EE200AB6
:10D0400031EE201A71EE600ABDEEE01A11EE100A00
:10D050009FED291A00F0030000EEC10A9FED271A88
:10D06000009000EEC10A9FED261A00EEC10A9FED66
:10D07000251A00EEC10A9DE700F00CF99AE718EEB8
:10D08000100A4000B0F17F4F0DD218EE100AFFF7E2
:10D0900051FA042808BF00F0F5F8B0EE480A01B0D4
:10D0A000BDEC028B00BD09D10120F3F79FFA01B05E
:10D0B000BDEC028B5DF804EB00F0DCB801B0B0EE23
:10D0C000480ABDEC028B5DF804EB00F0CDB800001F
:10D0D000B61F927EBCE9223C0B6D063B8A76CE3CA5
:10D0E000ACB5593D35A1083E29AAAA3E490E49468C
:10D0F00083F9223F0000004B0000C93F00A0FD392A
:10D100000020A2331A61342C70B504462DED028B39
:10D110004D1E00EBC500B0EE408AF0EE608A90ED47
:10D12000000B35F0060017D053EC182B51EC100B08
:10D1300000F0E6FC41EC100B6D1E04EBC50090ED19
:10D14000001B51EC100B53EC112B00F0BFF941EC1C
:10D15000100B35F00600E7D1022D36D0042D1CD07F
:10D16000062D1CBFBDEC028B70BD53EC182B51EC8F
:10D17000100B00F0C5FC94ED0A1B53EC112B00F0D2
:10D18000A5F953EC182B00F0BBFC94ED081B53ECF5
:10D19000112B00F09BF941EC100B53EC182B51ECC8
:10D1A000100B00F0ADFC94ED061B53EC112B00F0BE
:10D1B0008DF953EC182B00F0A3FC94ED040B53EC09
:10D1C000102B00F083F941EC100B53EC182B51ECB1
:10D1D000100B00F095FC94ED021B53EC112B00F0AA
:10D1E00075F953EC182B00F08BFC94ED001B53ECFD
:10D1F000112B00F06BF9BDEC028B41EC100B70BDF4
:10D2000010B553EC102B51EC100B00F05FF941EC12
:10D21000100B10BD10B553EC112B51EC100B00F09E
:10D2200055F941EC100B10BD9FED050B10B553ECFB
:10D23000102B51EC100B00F0FDF941EC100B10BD60
:10D2400000000000000000009FED050B10B553EC3E
:10D25000102B51EC100B00F053FC41EC100B10BDE7
:10D26000000000000000001030EE000A704730EEB1
:10D27000200A7047DFED020A80EEA00A7047000026
:10D28000000000009FED020A20EE000A7047000037
:10D29000000000102DE9F0014FF07F42B2EB410F8A
:10D2A0009FBF4FF0FF310160BDE8F00170474FF0C4
:10D2B000004242EA0123C1F3C752783A551112F0F5
:10D2C0001F0C434CCCF120067C44C1F3C752A2F1A1
:10D2D00078024FEA621204EB820254F8254008BF3C
:10D2E000D2E9015612D0556804FA0CF425FA06F773
:10D2F0003C43976805FA0CF527FA06F8D26807FA56
:10D300000CFCF24045EA08054CEA0206A4FB034C7B
:10D31000A5FB0352A6FB03631D449D4234BF0126B7
:10D3200000261319334416B1934202D903E0934205
:10D3300001D2012200E00022624402F1200C920698
:10D34000DC0C42EA443200EE102A5B03DFED210AD6
:10D35000F8EEC01A00EE103A4FEA9C1C11F0004F94
:10D36000B8EE400AC0F800C020EE201A00EE105AB5
:10D37000DFED190AB8EE400A20EE200A71EE810AAC
:10D3800070EE800A10EE902A02F500626FF30B0235
:10D3900000EE902A70EEE11A31EEC11ADFED101A9C
:10D3A00030EE411A9FED0D0A20EE800A01EE210AAF
:10D3B0009FED0C1A00EE810A04BFBDE8F001704732
:10D3C000CCF180510160BDE8F001B1EE400A704738
:10D3D0006C110000000000360000802C22AAFD29FC
:10D3E000DB0FC92F0000C92F10B541EC100BFFF760
:10D3F0004BF951EC100B10BD82B0CDE9000121F0CA
:10D40000004001909DED000B02B051EC100B7047F5
:10D4100010B500EE100A2DED028BB1EEC08A18EEA9
:10D42000100A20F00040C0F1FF40C00F0AD010EEFB
:10D43000100A20F00040C0F1FF40C00F04BF0120DF
:10D44000F3F7D4F818EE100ABDEC028B10BD81F092
:10D450000041704780F00040704721F00041704764
:10D4600020F000407047000021F0004201F000432E
:10D47000A2F16052B2F5801F28BFD2F17F6C0BD9A8
:10D480005FEA001C43EAC20242EB507018BF7047CB
:10D4900028BF20F001007047B2F5801FBCBF1846BE
:10D4A00070474FEA410C1CF5001F02D2084600F0FD
:10D4B0006BBF70B500F0CEFB00000089FFF7F6BF30
:10D4C0004FF00040A0F580007047000010B591EAD1
:10D4D000030F48BF83F0004300F19885841A71EB75
:10D4E000030C05D2121943EB0C03001B61EB0C017A
:10D4F0004FEA1154A4EB135CDFF81CE11EEA430F62
:10D5000018BF9EEA445F00F0748021EA045123EAC8
:10D510000E0343F48013DCF1200E32D322FA0CFE0A
:10D5200010EB0E0023FA0CFE41EB0E01CCF1200EA5
:10D5300003FA0EFE10EB0E00CCF1200E51F10001AB
:10D54000B1F5801F32D201EB045112FA0EF2BDE8A0
:10D55000104058BF7047401C38BF5FEA420218BFF6
:10D560007047002814BF20F0010041F100014FEA8C
:10D57000410313F5001F38BF7047A1F1C04100F00F
:10D580005FBC012A43EB0302ACF1200CDCF11F0E5F
:10D5900032BF4FF0000E23FA0CF310EB030041EB07
:10D5A0000451B4EB115FD0D0A1EB045101F580110F
:10D5B000490801EB04515FEA30000ED350F100003E
:10D5C00038BF12FA0EFE08D1BDE81040C9E7401C72
:10D5D00038BF5FEA4202CAD1C3E7BDE810404FEA54
:10D5E000410313F5001F38BF7047A1F1C04100F09F
:10D5F00027BC9EEA445F08D011EA5E0FBDE81040E8
:10D6000004BF01F0004100207047BDE8104070B534
:10D6100000F020FB64FBBE3E0000E0FF491058BF55
:10D62000C1F140415B1058BFC3F140438B42EFF35F
:10D63000008070472DE9C04130B4DFF8A4C23CEA55
:10D64000111418BF3CEA131400F0ED801CEA111409
:10D6500081EA030544EAD57418BF1CEA131500F0EB
:10D66000C880A4EB050404F17F7404F500344FF086
:10D67000004545EAC12145EAC32341EA505143EA46
:10D6800052534FEAC0204FEAC222994208BF90424B
:10D6900000F09D804FEA13650FF24416765D4FEA65
:10D6A000134506FB05F7C7F1807706FB07F74FEA3E
:10D6B000D737A7FB03687642A7FB06CEC8F58038AC
:10D6C00038BFA8F1010807FB08E6A6FB028C4FF063
:10D6D000000EE6FB03CEDCF1000CCEF1004E38BFAD
:10D6E000AEF1010EA6FB0C584FF00007E6FB0E87CB
:10D6F000A1FB08C6A0FB07CE16EB0E064FF00005F7
:10D7000045F10005E1FB076515F1E04E7EBFA4F58C
:10D7100080345FEA46066D4116F1800745F1000549
:10D720004FEA172747EA05674FEA15254FEA0666CD
:10D73000A6F1DE46B6F1805F20D9384605EBC4710C
:10D7400024F0010C01EB0C11BCF1FE6F02D8F0BC0F
:10D75000BDE8008124425CBF01F5801E9EEAC47FC3
:10D7600002D4F0BCBDE80081244200F13980A1F16F
:10D77000C041F0BCBDE8004100F062BB4FEAD020E0
:10D7800040EA41504FEAD1214FEAD22242EA4352C5
:10D790004FEAD323A7FB028607FB036605FB02665D
:10D7A0001EEA0E0F58BFA6EB0056B6EB00564FEA26
:10D7B000520E4EEAC37E18EB0E0E56EB530EBCD53E
:10D7C00018EB02085E417F1C55F10005B5E74FF4E8
:10D7D00080154FF000074FF000064FF00008ACE74F
:10D7E00001F1C04101F000414FF00000F0BCBDE884
:10D7F00000810CEA131511EA0C1F00D00CE013EAAB
:10D800000C1F00F026804FF0000081EA030101F0B8
:10D810000041F0BCBDE80081F0BCBDE8004181EAF8
:10D82000030100F00DBBF0BCBDE8004170B500F095
:10D8300011FA00BF097EFC3E00F007B84FF000006F
:10D8400081EA030101F00041704781EA030100F021
:10D85000F7BAF0BCBDE8004122494FF00000704724
:10D86000FFFDFBF9F7F5F4F2F0EEEDEBE9E8E6E4A5
:10D87000E3E1E0DEDDDBDAD8D7D5D4D3D1D0CFCD2C
:10D88000CCCBCAC8C7C6C5C4C2C1C0BFBEBDBCBB65
:10D89000BAB9B8B7B6B5B4B3B2B1B0AFAEADACAB60
:10D8A000AAA9A8A8A7A6A5A4A3A3A2A1A09F9F9E3A
:10D8B0009D9C9C9B9A9999989797969595949393EC
:10D8C000929191908F8F8E8E8D8C8C8B8B8A898983
:10D8D0008888878786858584848383828281818006
:10D8E0000000FF070000F87F51EA030C17D41CF575
:10D8F000801F58BFBCF5801F00F10680994218BFF9
:10D90000704708BF9042704707D711F5801F58BF76
:10D9100013F5801F19D499427047894270471CF54E
:10D92000801F08D5BCF5801FF7D58B4218BF704704
:10D9300008BF824270474FF4001C1CEB410F38BFF8
:10D940001CEB430F01D28B42704770B500F082F997
:10D95000922449004FF000514FF08053FFF75EBE14
:10D960004FEA1153A3F58063D3F11E03A8BFD3F18F
:10D97000200C08DB4FF0004242EAC12252EA50522A
:10D9800032FA03F0704709420BD4102BC4BF0020B9
:10D99000704703F5787CBCF1FF3F05D04FF0FF30B6
:10D9A00070474FF00000704770B500F053F900BFAA
:10D9B0004992248000207047F0E710F0004248BFF1
:10D9C0004042B0FA80F310FA03F10AD0C3F11D030C
:10D9D00003F5806302EB03524FEA415002EBD12181
:10D9E00070474FF000007047B0FA80F310FA03F16F
:10D9F0000AD0C3F11D0303F580634FEA03524FEAD7
:10DA0000415002EBD12170474FF0000070470000F9
:10DA100051EA030C17D41CF5801F58BFBCF5801FBA
:10DA200000F10680994218BF704708BF90427047C6
:10DA300007D711F5801F58BF13F5801F19D49942DD
:10DA40007047894270471CF5801F08D5BCF5801FC0
:10DA5000F7D58B4218BF704708BF824270474FF41A
:10DA6000001C1CEB410F38BF1CEB430F01D28B4253
:10DA7000704770B500F0EEF8922449004FF08051E5
:10DA80004FF00053FFF7CABD51EA030C17D41CF541
:10DA9000801F58BFBCF5801F00F10680994218BF57
:10DAA000704708BF9042704707D711F5801F58BFD5
:10DAB00013F5801F19D499427047894270471CF5AD
:10DAC000801F08D5BCF5801FF7D58B4218BF704763
:10DAD00008BF824270474FF4001C1CEB410F38BF57
:10DAE0001CEB430F01D28B42704770B500F0B2F8C7
:10DAF000922449004FF000514FF08053FFF78EBD44
:10DB000070B5DFF848C11CEA111E1EBF1CEA1315D0
:10DB10009EEA0C0F95EA0C0F00F06F8081EA030477
:10DB20004EEAD47EAE4421EA4C1123EA4C1341F470
:10DB3000801143F48013AEF17F7EA1FB024CA0FB69
:10DB40000365361955EB0C05A1FB034C4CF10003A2
:10DB5000A0FB021C16EB0C06654153F100030942C1
:10DB600018BF46F0010613F4007F0BD14FEA0331D2
:10DB70004FEA053041EA155140EA165034036FF080
:10DB800003020AE04FEAC3214FEAC52041EA55519A
:10DB900040EA5650F4026FF0020202EB2E4201EB13
:10DBA000025585EACE710AD05FEA440C18BF24F012
:10DBB000004450F1000041F1000120EAD47040F22D
:10DBC000FE7C624500D270BDA84214BF4FF0804475
:10DBD0004FF04044002E08BF0024BEF1806FA8BF64
:10DBE000A1F1C041BDE8704080F22A8101F1C0413D
:10DBF00001F000414FF0000070470CEA13159EEA57
:10DC00000C0F18BF95EA0C0F06D081EA030E4FF0F7
:10DC100000000EF0004170BD00F01CF88900013ECC
:10DC200000F007B800F009B84FEA430C5FEA5C5C0B
:10DC300008D081EA030100F003B94FEA410C5FEA22
:10DC40005C5CF6D102494FF0000070470000FF070E
:10DC50000000F87F0EF1020E2EF0030E5EF8046B4A
:10DC6000364205D4012A43EB030515F5001F12D8EF
:10DC7000012841EB010C1CF5001F0CD80ED14FEA16
:10DC8000D17C0CEB4C0C0CF1020C15F5001F08BFFD
:10DC90004CEBD37C04E04FF0080C01E04FEAD37C5E
:10DCA0000CEB4C0526FA05F606F00706B6F1040C57
:10DCB00006D20EEB860CBDE870404CF0010C6047BC
:10DCC000DFE80CF0090B02024FF00041A1F5002142
:10DCD0004FF0000070BD19461046012851EB0104B9
:10DCE00018BFD4F5001484BF002001F0004170BDBE
:10DCF00070B5DFF844C13CEA111418BF3CEA1315B3
:10DD000000F08F8011F1004F0CEA11141CEA13157A
:10DD100068BF45F0050518BF11EA0C1F00F07980B7
:10DD200021EA4C1123EA4C1341F4801143F480138F
:10DD30002E46A5F58035AC423DDDA4F58036801A2F
:10DD4000994109D54042C1F1000134BFB1F101014F
:10DD5000B1F1000185F0010511F4F01F08D011F4B4
:10DD6000801FE8D1400041EB0101A4F58034F6E7C3
:10DD700021F00041B1FA81F6202E04BFB0FA80FEF6
:10DD80000EF12006A6F10B06A4EB0644B6F1200E18
:10DD90000CD2C6F1200E01FA06F120FA0EF641EA85
:10DDA0000601CEF1200600FA06F003E000FA0EF1BB
:10DDB0004FF00000BFE750EA410E23D04FEA244E57
:10DDC000BEEB254F0FDB994208BF904204D00AD327
:10DDD000520043EB0303B0E74FEA1646B6EB144F8D
:10DDE00008BF85F00105B4F5803401EB041181EA28
:10DDF000C57100DB70BD01F1C04101F000414FF081
:10DE0000000070BD4FEA45714FF0000001F0004185
:10DE100070BD1CEA131F09D04FF0000001F0004153
:10DE200070BDFFF717FF00BFEDFFFF3EBDE870407C
:10DE300002494FF0000070470000FF070000F87F24
:10DE40000808A0F500114FEA3101704710B591EABA
:10DE5000030F81F000413FF541AB83F0004300F038
:10DE6000D5B800002DE9F04101F5801CBCF5001F7C
:10DE7000C0F2A9804FEA115C21EA0C5141F48011F3
:10DE80000CF1FD0C5FEA5C0C0CF5C07C01D340008A
:10DE90004941890241EA905187022EA48E0EA45D69
:10DEA0000A0C04FB04F602FB06F6C6F14046A4FB8E
:10DEB0000662F60D46EA422606FB06F4A4FB0123A1
:10DEC0005242C3F1404338BF5B1EA6FB024200240E
:10DED000E6FB0324D20B42EA4446A6FB0623A1FB41
:10DEE00002E2A3FB07E4E3FB61426442C2F1404E5D
:10DEF00038BFAEF1010EA6FB04234FF00002E6FB93
:10DF00000E32A2FB03463400E2FB6264A1FB06E68C
:10DF1000A4FB07E8E4FB61687642C8F1405838BFCB
:10DF2000A8F10108A2FB06E4A3FB08E5E2FB6854A4
:10DF3000A1FB05E6A7FB04E8E1FB648618F12005D8
:10DF400056F10006A80940EA8660B109A8F11B084D
:10DF500008F03F08B8F10A0F1CD901EB0C51BDE8DD
:10DF6000F08100BFFCF5EEE8E2DDD8D3CFCBC7C32C
:10DF7000C0BDB9B6B4B1AEACA9A7A5A3A19F9D9BE6
:10DF80009A9896959392908F8D8C8B8988878685A9
:10DF900084838281A0FB006800FB01F208EB420849
:10DFA000B8EB872807D5341858EB0104D5D5401CA9
:10DFB00051F10001D1E7341A78EB0104CDD4401EB1
:10DFC00071F10001C9E75FEA4C0C5FEA9C5C0DD17E
:10DFD00005D301F000414FF00000BDE8F081BDE83D
:10DFE000F04170B5FFF736FE6DDBFFBEBDE8F041D6
:10DFF00001494FF0000070470000F87F10B591EA2A
:10E00000030F48BF83F000433FF568AA841A71EB01
:10E01000030C07D28CF0004C121943EB0C03001BCD
:10E0200061EB0C014FEA1154A4EB135CDFF8A4E19F
:10E030001EEA430F18BF9EEA445F00F0B48021EA55
:10E04000045123EA6E035242C3EB6E0338BF5B1EDA
:10E05000DCF1200E25D322FA0CFE10EB0E0043FA61
:10E060000CFE41EB0E01CCF1200E03FA0EFE10EB7C
:10E070000E00CCF1200E51F1000129D401EB045126
:10E0800012FA0EF2BDE8104058BF7047401C1CBF8A
:10E09000B2F1004F704700280CBF491C20F001006E
:10E0A000704712EB020E43EB030218BF4FF0010E54
:10E0B0004EEA4202ACF1200CDCF11E0E56D943FAB6
:10E0C0000CFE10EB0E00CCF11E0E51F1FF31D5D538
:10E0D0000EF1010E12FA0EFE404141EB010101EB7F
:10E0E000445C5FEA5C5C10D901EB045110EBDE701C
:10E0F00038BFBEF1004FBDE8104018BF7047002880
:10E100000CBF491C20F00100704734D24FEAD42CD8
:10E1100024F4006411F500111BD0B1FA81F20B3A1E
:10E12000A41AA41ED2F12003914030FA03F319433C
:10E13000904001EBCC7101EB0451002CBDE8104084
:10E14000A8BF704701F1C04101F000414FF000004D
:10E150007047B0FA80F310FA03F102D1BDE8104025
:10E160007047E41A173C4805C90AE2E701EB04517D
:10E17000BDE81040704749104FEA300001EB0451F0
:10E18000BDE8104002E04FF0000170474A0008BFB0
:10E190000042F8D0B2F5001F28BF704701F00041DF
:10E1A0004FF0000070479EEA445F07D011EA5E0F0F
:10E1B000BDE8104004BF002100207047BDE81040BA
:10E1C00070B5FFF747FD00BF40DFF63E104683F015
:10E1D000004170470000E0FF43004FEAD30C4FEAD4
:10E1E0003C0C43401FBF40070CF1605113F0FE4F41
:10E1F00070471CF0006F03D10CF000410020704705
:10E200000CF0004343EA507040EACC0010B500F037
:10E2100068F800BF000000924FEA0001FFF710BE4F
:10E220004FF00041A1F500214FF00000704710B5FC
:10E23000FFF75AFB0CBF0120002010BD10B5FFF7FF
:10E2400053FB14BF0120002010BD10B5FFF7E0FB09
:10E250008CBF0120002010BD10B5FFF7D9FB2CBFEB
:10E260000120002010BD10B5FFF70EFC94BF012067
:10E27000002010BD10B5FFF707FC34BF01200020BF
:10E2800010BD4FF07E5209E011F0004204D540422B
:10E29000C1F1000138BF491E42F07E5202F17062A6
:10E2A0000B0012BF20235FEA00017047B1FA81FC26
:10E2B00001FA0CF1A3EB0C0320FA03FC41EA0C0178
:10E2C00002EBC352C3F1200310FA03FC5CEA416C79
:10E2D00042EB112018BF5FF0806C28BF20F00100D6
:10E2E00070470EF1020E2EF0030E5EF8044B24422E
:10E2F00004D44FEA4102B2F17F4F11D84FEA4003F4
:10E30000B3F17F4F0CD80ED14FEAD07C0CEB4C0C04
:10E310000CF1020CB2F17F4F08BF4CEBD17C04E052
:10E320004FF0080C01E04FEAD17C0CEB4C0324FACF
:10E3300003F404F00704B4F1040C06D20EEB840CD1
:10E34000BDE810404CF0010C6047DFE80CF0070816
:10E3500002024FF00040A0F5800010BD08464200C8
:10E3600018BFD2F1807288BF00F0004010BDF1EEFE
:10E37000100A4FF6FF71C0F2C03120EA010040F0F0
:10E380004070E1EE100A7047FF2141EAD050C0050D
:10E3900070470000000000004FBB610567ACDD3F27
:10E3A000182D4454FB21E93F9BF681D20B73EF3FBC
:10E3B000182D4454FB21F93FE2652F227F2B7A3C34
:10E3C000075C143326A6813CBDCBF07A8807703CED
:10E3D000075C143326A6913CC4EB98999999C9BF60
:10E3E000711623FEC671BCBF6D9A74AFF2B0B3BF95
:10E3F0009AFDDE522DDEADBF2F6C6A2C44B4A2BF55
:10E400000D5555555555D53FFF8300922449C23FC0
:10E410006E204CC5CD45B73F513DD0A0660DB13FF4
:10E42000EB0D76244B7BA93F11DA22E33AAD903F06
:10E430000000000000000000000000006E83F9A250
:10E440002915444ED15727FCC0DD34F5999562DB80
:10E450004190433CAB6351FE00000000000000000F
:10E46000010203040607080900000000010203047A
:10E470000100000000000240100000000000024007
:10E4800001000000000402401000000000080240EB
:10E4900020000000000802400800000000180240B0
:10E4A000400000000018024033E6000800000000B1
:10E4B0000000000000000000000000000004000058
:10E4C00018000000000000000000000036E6000810
:10E4D000000000000000000000000000000000003C
:10E4E0000004000018000000000000000000000010
:10E4F00058E60008000000000000000000000000D6
:10E5000000000000000400001800000000000000EF
:10E51000000000004CE600080000000000000000C1
:10E5200000000000000000000004000018000000CF
:10E53000000000000000000070E60008000000007D
:10E5400000000000000000000000000000040000C7
:10E5500030000000000000000000000040E600085D
:10E5600000000000000000000000000000000000AB
:10E57000000400001800000000000000000000007F
:10E5800065E6000800000000000000000000000038
:10E59000000000000004000018000000000000005F
:10E5A0000000000028E60008000000000000000055
:10E5B000000000000000000000040000180000003F
:10E5C000000000000000000080E9334320949643DF
:10E5D000002CF14209B896431CE600080000000038
:10E5E0000000000000000000000000000002000029
:10E5F0001800000000000000000000009A99193E79
:10E600000000803F00000000000000000000803F8C
:10E610000000803F000000000000000064656661AB
:10E62000756C745461736B0074656C65636F7069AD
:10E630006E6700616900617474695F657374690075
:10E6400072656D6F74655F6374726C0067696D628B
:10E65000616C5F6374726C00636861737369735F8C
:10E660006374726C0073686F6F745F6374726C00B4
:10E670005461736B5F496E6974000000C0E6000866
:10E680000000002088030000C401000800E8000822
:10E6900000C00120080000002002000800E8000877
:10E6A0008803002068A201003C02000808E8000876
:10E6B00008C00120D82500003C020008000000002E
:10E6C000112324F41A0102F112013C0A0202083A51
:10E6D0000908256666E63E23803F4FC04017B751C4
:10E6E0003A0C39044ABF04332041E24029141E8009
:10E6F000BFDB0FC9185A8040210C11FA2AF9400ECD
:10E7000019404166660640019429B8880B7A44D7BF
:10E71000A3303FD7A3F0BED0E11C9A9999FCF93CF5
:10E72000192C1119E03AA0DC5A0414520234A04109
:10E730000AD20133F042293419181307022A011EA4
:10E740003E803F6666E614811C666666101AF058C5
:10E7500029883990180A40CDCCCC3E0AD7233D0CED
:10E76000198829041A204C29201A207C1B803F205C
:10E770002A3D20292869C43CDB0FC91C215BC03F0E
:10E78000C019287A4C2059E83980292029440C11D5
:10E790009A99194039E8D9F8694029A8A904392C6F
:10E7A0003990992C793029803C3D0A576C89206931
:10E7B000EC5BB443A0D920A970540102015A0208AD
:10E7C0005A03085A0408540502023A060812015A6C
:10E7D00007085A0818237AC44A080BD9DC597C99CF
:10E7E0006C290C1EC8419A999918111A4094123E2E
:10E7F0004C409C461C412BF04174721000000000FC
:08E80000022B073DAAAAAAAAF7
:040000050800018965
:00000001FF
